BL51 BANKED LINKER/LOCATER V6.22                                                        06/21/2022  07:40:42  PAGE 1


BL51 BANKED LINKER/LOCATER V6.22, INVOKED BY:
C:\KEIL_V5\C51\BIN\BL51.EXE .\output\Main.obj, .\output\Initial.obj, .\output\InterruptApp.obj, .\output\Led.obj, .\outp
>> ut\KeyApp.obj, .\output\LowPower.obj, .\output\UartApp.obj, .\output\Memory.obj, .\output\AFE.obj, .\output\Balance.o
>> bj, .\output\Calculate.obj, .\output\Calibrate.obj, .\output\ChargerLoad.obj, .\output\ExtE2PRom.obj, .\output\Interr
>> upt.obj, .\output\KeyScan.obj, .\output\McuFlash.obj, .\output\McuLib.obj, .\output\MosCtrl.obj, .\output\PorSelfTest
>> .obj, .\output\Protect.obj, .\output\RTC.obj, .\output\TWI.obj, .\output\Uart.obj, .\output\Thermistor.obj, .\output\
>> STARTUP.obj, .\output\GasGauge.obj, .\code_gasguage\GasGaugeLib.LIB, .\output\BootApp.obj, .\output\DataFlash.obj TO 
>> .\output\McuFlash_IAP REGFILE (.\output\McuFlash_IAP.ORC) PRINT (.\output\McuFlash_IAP.m51) RAMSIZE (256) DISABLEWARN
>> ING (16) CODE (0X1000-0X87FF, ?CO?DATAFLASH (0X8400)) XDATA (0X0200-0X0AFE)


MEMORY MODEL: LARGE WITH FLOATING POINT ARITHMETIC


INPUT MODULES INCLUDED:
  .\output\Main.obj (MAIN)
  .\output\Initial.obj (INITIAL)
  .\output\InterruptApp.obj (INTERRUPTAPP)
  .\output\Led.obj (LED)
  .\output\KeyApp.obj (KEYAPP)
  .\output\LowPower.obj (LOWPOWER)
  .\output\UartApp.obj (UARTAPP)
  .\output\Memory.obj (MEMORY)
  .\output\AFE.obj (AFE)
  .\output\Balance.obj (BALANCE)
  .\output\Calculate.obj (CALCULATE)
  .\output\Calibrate.obj (CALIBRATE)
  .\output\ChargerLoad.obj (CHARGERLOAD)
  .\output\ExtE2PRom.obj (EXTE2PROM)
  .\output\Interrupt.obj (INTERRUPT)
  .\output\KeyScan.obj (KEYSCAN)
  .\output\McuFlash.obj (MCUFLASH)
  .\output\McuLib.obj (MCULIB)
  .\output\MosCtrl.obj (MOSCTRL)
  .\output\PorSelfTest.obj (PORSELFTEST)
  .\output\Protect.obj (PROTECT)
  .\output\RTC.obj (RTC)
  .\output\TWI.obj (TWI)
  .\output\Uart.obj (UART)
  .\output\Thermistor.obj (THERMISTOR)
  .\output\STARTUP.obj (?C_STARTUP)
  .\output\GasGauge.obj (GASGAUGE)
  .\code_gasguage\GasGaugeLib.LIB (GASGAUGELIB)
  .\output\BootApp.obj (BOOTAPP)
  .\output\DataFlash.obj (DATAFLASH)
  C:\KEIL_V5\C51\LIB\C51FPL.LIB (?C?FPADD)
  C:\KEIL_V5\C51\LIB\C51FPL.LIB (?C?FPMUL)
  C:\KEIL_V5\C51\LIB\C51FPL.LIB (?C?FPDIV)
  C:\KEIL_V5\C51\LIB\C51FPL.LIB (?C?FCAST)
  C:\KEIL_V5\C51\LIB\C51FPL.LIB (?C?CASTF)
  C:\KEIL_V5\C51\LIB\C51FPL.LIB (?C?FPGETOPN)
  C:\KEIL_V5\C51\LIB\C51L.LIB (?C?CLDPTR)
  C:\KEIL_V5\C51\LIB\C51L.LIB (?C?IMUL)
  C:\KEIL_V5\C51\LIB\C51L.LIB (?C?UIDIV)
  C:\KEIL_V5\C51\LIB\C51L.LIB (?C?IILDX)
  C:\KEIL_V5\C51\LIB\C51L.LIB (?C?LADD)
  C:\KEIL_V5\C51\LIB\C51L.LIB (?C?LSUB)
  C:\KEIL_V5\C51\LIB\C51L.LIB (?C?LMUL)
BL51 BANKED LINKER/LOCATER V6.22                                                      06/21/2022  07:40:42  PAGE 2


  C:\KEIL_V5\C51\LIB\C51L.LIB (?C?ULDIV)
  C:\KEIL_V5\C51\LIB\C51L.LIB (?C?SLDIV)
  C:\KEIL_V5\C51\LIB\C51L.LIB (?C?LOR)
  C:\KEIL_V5\C51\LIB\C51L.LIB (?C?LNEG)
  C:\KEIL_V5\C51\LIB\C51L.LIB (?C?SLCMP)
  C:\KEIL_V5\C51\LIB\C51L.LIB (?C?ULCMP)
  C:\KEIL_V5\C51\LIB\C51L.LIB (?C?ULSHR)
  C:\KEIL_V5\C51\LIB\C51L.LIB (?C?SLSHR)
  C:\KEIL_V5\C51\LIB\C51L.LIB (?C?LSHL)
  C:\KEIL_V5\C51\LIB\C51L.LIB (?C?LLDXDATA)
  C:\KEIL_V5\C51\LIB\C51L.LIB (?C?LLDXDATA0)
  C:\KEIL_V5\C51\LIB\C51L.LIB (?C?LSTXDATA)
  C:\KEIL_V5\C51\LIB\C51L.LIB (?C?LSTKXDATA)
  C:\KEIL_V5\C51\LIB\C51L.LIB (?C?OFFXADD)
  C:\KEIL_V5\C51\LIB\C51L.LIB (?C?CCASE)
  C:\KEIL_V5\C51\LIB\C51L.LIB (?C?LIMUL)
  C:\KEIL_V5\C51\LIB\C51L.LIB (LABS)


LINK MAP OF MODULE:  .\output\McuFlash_IAP (MAIN)


            TYPE    BASE      LENGTH    RELOCATION   SEGMENT NAME
            -----------------------------------------------------

            * * * * * * *   D A T A   M E M O R Y   * * * * * * *
            REG     0000H     0008H     ABSOLUTE     "REG BANK 0"
            DATA    0008H     0007H     UNIT         ?DT?KEYSCAN
            DATA    000FH     0006H     UNIT         ?DT?AFE
            DATA    0015H     0002H     UNIT         _DATA_GROUP_
            IDATA   0017H     0007H     UNIT         ?ID?GASGAUGE
            IDATA   001EH     0002H     UNIT         _IDATA_GROUP_
            DATA    0020H     0007H     BIT_ADDR     ?BA?MEMORY
            BIT     0027H.0   0001H.5   UNIT         ?BI?EXTE2PROM
            BIT     0028H.5   0000H.6   UNIT         _BIT_GROUP_
            BIT     0029H.3   0000H.5   UNIT         ?BI?AFE
            BIT     002AH.0   0000H.5   UNIT         ?BI?BALANCE
            BIT     002AH.5   0000H.4   UNIT         ?BI?LOWPOWER
            BIT     002BH.1   0000H.4   UNIT         ?BI?UARTAPP
            BIT     002BH.5   0000H.4   UNIT         ?BI?CHARGERLOAD
            BIT     002CH.1   0000H.4   UNIT         ?BI?GASGAUGE
            BIT     002CH.5   0000H.3   UNIT         ?BI?INTERRUPTAPP
            BIT     002DH.0   0000H.3   UNIT         ?BI?MCUFLASH
            BIT     002DH.3   0000H.2   UNIT         ?BI?LED
            BIT     002DH.5   0000H.2   UNIT         ?BI?MOSCTRL
            BIT     002DH.7   0000H.2   UNIT         ?BI?PROTECT
            BIT     002EH.1   0000H.2   UNIT         ?BI?RTC
            BIT     002EH.3   0000H.1   UNIT         ?BI?CALIBRATE
            BIT     002EH.4   0000H.1   UNIT         ?BI?KEYSCAN
            BIT     002EH.5   0000H.1   UNIT         ?BI?PORSELFTEST
                    002EH.6   0000H.2                *** GAP ***
            IDATA   002FH     0001H     UNIT         ?ID?EXTE2PROM
                    0030H     0070H                  *** GAP ***
            IDATA   00A0H     0060H     ABSOLUTE     

            * * * * * * *  X D A T A   M E M O R Y  * * * * * * *
            XDATA   0000H     0002H     ABSOLUTE     
BL51 BANKED LINKER/LOCATER V6.22                                                      06/21/2022  07:40:42  PAGE 3


            XDATA   0002H     0014H     ABSOLUTE     
            XDATA   0016H     0004H     ABSOLUTE     
            XDATA   001AH     0004H     ABSOLUTE     
            XDATA   001EH     0004H     ABSOLUTE     
            XDATA   0022H     0002H     ABSOLUTE     
            XDATA   0024H     0002H     ABSOLUTE     
            XDATA   0026H     0002H     ABSOLUTE     
            XDATA   0028H     0002H     ABSOLUTE     
            XDATA   002AH     0001H     ABSOLUTE     
            XDATA   002BH     0001H     ABSOLUTE     
            XDATA   002CH     0002H     ABSOLUTE     
            XDATA   002EH     0001H     ABSOLUTE     
            XDATA   002FH     0001H     ABSOLUTE     
            XDATA   0030H     0002H     ABSOLUTE     
            XDATA   0032H     0002H     ABSOLUTE     
            XDATA   0034H     0001H     ABSOLUTE     
            XDATA   0035H     000CH     ABSOLUTE     
            XDATA   0041H     0004H     ABSOLUTE     
            XDATA   0045H     0002H     ABSOLUTE     
            XDATA   0047H     000CH     ABSOLUTE     
            XDATA   0053H     000CH     ABSOLUTE     
            XDATA   005FH     0002H     ABSOLUTE     
            XDATA   0061H     0001H     ABSOLUTE     
            XDATA   0062H     0002H     ABSOLUTE     
            XDATA   0064H     0002H     ABSOLUTE     
            XDATA   0066H     0001H     ABSOLUTE     
            XDATA   0067H     0001H     ABSOLUTE     
            XDATA   0068H     0005H     ABSOLUTE     
            XDATA   006DH     0004H     ABSOLUTE     
            XDATA   0071H     0001H     ABSOLUTE     
            XDATA   0072H     0001H     ABSOLUTE     
            XDATA   0073H     0001H     ABSOLUTE     
            XDATA   0074H     0001H     ABSOLUTE     
            XDATA   0075H     0002H     ABSOLUTE     
            XDATA   0077H     0002H     ABSOLUTE     
            XDATA   0079H     0001H     ABSOLUTE     
            XDATA   007AH     0001H     ABSOLUTE     
            XDATA   007BH     0003H     ABSOLUTE     
            XDATA   007EH     0004H     ABSOLUTE     
            XDATA   0082H     0001H     ABSOLUTE     
            XDATA   0083H     0004H     ABSOLUTE     
            XDATA   0087H     0001H     ABSOLUTE     
            XDATA   0088H     0001H     ABSOLUTE     
            XDATA   0089H     0001H     ABSOLUTE     
            XDATA   008AH     0002H     ABSOLUTE     
            XDATA   008CH     0001H     ABSOLUTE     
            XDATA   008DH     0001H     ABSOLUTE     
            XDATA   008EH     0001H     ABSOLUTE     
            XDATA   008FH     0002H     ABSOLUTE     
            XDATA   0091H     0002H     ABSOLUTE     
            XDATA   0093H     0002H     ABSOLUTE     
            XDATA   0095H     0002H     ABSOLUTE     
            XDATA   0097H     0001H     ABSOLUTE     
            XDATA   0098H     0001H     ABSOLUTE     
            XDATA   0099H     0001H     ABSOLUTE     
            XDATA   009AH     0002H     ABSOLUTE     
            XDATA   009CH     0002H     ABSOLUTE     
BL51 BANKED LINKER/LOCATER V6.22                                                      06/21/2022  07:40:42  PAGE 4


            XDATA   009EH     0002H     ABSOLUTE     
            XDATA   00A0H     0002H     ABSOLUTE     
            XDATA   00A2H     0001H     ABSOLUTE     
            XDATA   00A3H     0002H     ABSOLUTE     
            XDATA   00A5H     0002H     ABSOLUTE     
            XDATA   00A7H     0002H     ABSOLUTE     
            XDATA   00A9H     0001H     ABSOLUTE     
            XDATA   00AAH     0001H     ABSOLUTE     
            XDATA   00ABH     0002H     ABSOLUTE     
            XDATA   00ADH     0002H     ABSOLUTE     
            XDATA   00AFH     0001H     ABSOLUTE     
            XDATA   00B0H     0001H     ABSOLUTE     
            XDATA   00B1H     0002H     ABSOLUTE     
            XDATA   00B3H     0002H     ABSOLUTE     
            XDATA   00B5H     0001H     ABSOLUTE     
            XDATA   00B6H     0004H     ABSOLUTE     
            XDATA   00BAH     0004H     ABSOLUTE     
            XDATA   00BEH     0004H     ABSOLUTE     
            XDATA   00C2H     0004H     ABSOLUTE     
            XDATA   00C6H     0004H     ABSOLUTE     
            XDATA   00CAH     0002H     ABSOLUTE     
            XDATA   00CCH     0001H     ABSOLUTE     
            XDATA   00CDH     0001H     ABSOLUTE     
            XDATA   00CEH     0002H     ABSOLUTE     
            XDATA   00D0H     0001H     ABSOLUTE     
            XDATA   00D1H     0002H     ABSOLUTE     
            XDATA   00D3H     0002H     ABSOLUTE     
            XDATA   00D5H     0002H     ABSOLUTE     
            XDATA   00D7H     0002H     ABSOLUTE     
            XDATA   00D9H     0002H     ABSOLUTE     
            XDATA   00DBH     0001H     ABSOLUTE     
            XDATA   00DCH     0001H     ABSOLUTE     
            XDATA   00DDH     0121H     ABSOLUTE     
            XDATA   01FEH     0002H     ABSOLUTE     
            XDATA   0200H     00B5H     UNIT         ?XD?AFE
            XDATA   02B5H     0070H     UNIT         _XDATA_GROUP_
            XDATA   0325H     0022H     UNIT         ?XD?PROTECT
            XDATA   0347H     0012H     UNIT         ?XD?CALIBRATE
            XDATA   0359H     000FH     UNIT         ?XD?EXTE2PROM
            XDATA   0368H     000FH     UNIT         ?XD?GASGAUGE
            XDATA   0377H     0008H     UNIT         ?XD?RTC
            XDATA   037FH     0007H     UNIT         ?XD?UARTAPP
            XDATA   0386H     0006H     UNIT         ?XD?BALANCE
            XDATA   038CH     0003H     UNIT         ?XD?LED
            XDATA   038FH     0003H     UNIT         ?XD?LOWPOWER
            XDATA   0392H     0003H     UNIT         ?XD?_MCUPWM0SET?MCULIB
            XDATA   0395H     0003H     UNIT         ?XD?_MCUPWM1SET?MCULIB
            XDATA   0398H     0002H     UNIT         ?XD?INTERRUPTAPP
            XDATA   039AH     0002H     UNIT         ?XD?CALCULATE
            XDATA   039CH     0002H     UNIT         ?XD?CHARGERLOAD
            XDATA   039EH     0002H     UNIT         ?XD?MCUFLASH
            XDATA   03A0H     0001H     UNIT         ?XD?KEYAPP
            XDATA   03A1H     0001H     UNIT         ?XD?PORSELFTEST
                    03A2H     065EH                  *** GAP ***
            XDATA   0A00H     0096H     ABSOLUTE     

            * * * * * * *   C O D E   M E M O R Y   * * * * * * *
BL51 BANKED LINKER/LOCATER V6.22                                                      06/21/2022  07:40:42  PAGE 5


                    0000H     1000H                  *** GAP ***
            CODE    1000H     0003H     ABSOLUTE     
            CODE    1003H     0020H     UNIT         ?PR?INTERRUPTTIMER3?INTERRUPT
            CODE    1023H     0003H     ABSOLUTE     
                    1026H     0005H                  *** GAP ***
            CODE    102BH     0003H     ABSOLUTE     
            CODE    102EH     0025H     UNIT         ?PR?INITGPIO?INITIAL
            CODE    1053H     0003H     ABSOLUTE     
            CODE    1056H     065BH     UNIT         ?C?LIB_CODE
            CODE    16B1H     04DAH     UNIT         ?PR?DATAFILTER?GASGAUGELIB
            CODE    1B8BH     045EH     UNIT         ?PR?CORRECTDSGSOC?GASGAUGELIB
            CODE    1FE9H     0326H     UNIT         ?PR?GASGAUGEMANAGE?GASGAUGE
            CODE    230FH     025CH     UNIT         ?PR?GASGAUGEINIT?GASGAUGE
            CODE    256BH     0255H     UNIT         ?PR?CORRECTCHGSOC?GASGAUGELIB
            CODE    27C0H     01F0H     UNIT         ?PR?_CALCUTEMP?CALCULATE
            CODE    29B0H     01D8H     UNIT         ?PR?_TWIREAD?TWI
            CODE    2B88H     01C2H     UNIT         ?PR?_RTCREADTIME?RTC
            CODE    2D4AH     01B3H     UNIT         ?PR?_E2PROMBKDATA?EXTE2PROM
            CODE    2EFDH     0178H     UNIT         ?PR?AFECALCUCURR?CALCULATE
            CODE    3075H     0167H     UNIT         ?PR?IAPCHECKHANDSHAKE?UARTAPP
            CODE    31DCH     0148H     UNIT         ?PR?UARTRDCMDPROCESS?UARTAPP
            CODE    3324H     0147H     UNIT         ?PR?_TWIWRITE?TWI
            CODE    346BH     0144H     UNIT         ?PR?BALTURNONCHECK?BALANCE
            CODE    35AFH     0142H     UNIT         ?CO?THERMISTOR
            CODE    36F1H     0139H     UNIT         ?PR?_MCUTIMER3SET?MCULIB
            CODE    382AH     0138H     UNIT         ?PR?AFECALCUVOL?CALCULATE
            CODE    3962H     0100H     UNIT         ?CO?TWI
            CODE    3A62H     00EEH     UNIT         ?PR?AFECALCUTEMPE?CALCULATE
            CODE    3B50H     00D3H     UNIT         ?PR?E2PROMBKCHECK?EXTE2PROM
            CODE    3C23H     00C1H     UNIT         ?PR?MCUFLASHPROCESS?MCUFLASH
            CODE    3CE4H     00BDH     UNIT         ?PR?UARTCALICURRENT?UARTAPP
            CODE    3DA1H     00BCH     UNIT         ?PR?PROTECTOV?PROTECT
            CODE    3E5DH     00BCH     UNIT         ?PR?PROTECTUV?PROTECT
            CODE    3F19H     00BCH     UNIT         ?PR?PROTECTOTC?PROTECT
            CODE    3FD5H     00BCH     UNIT         ?PR?PROTECTUTC?PROTECT
            CODE    4091H     00BCH     UNIT         ?PR?PROTECTOTD?PROTECT
            CODE    414DH     00BCH     UNIT         ?PR?PROTECTUTD?PROTECT
            CODE    4209H     00BAH     UNIT         ?PR?BALPROCESS?BALANCE
            CODE    42C3H     00B3H     UNIT         ?PR?OFFSETCALCULATE?CALCULATE
            CODE    4376H     00B2H     UNIT         ?PR?_AFEWRITEREG?AFE
            CODE    4428H     00ADH     UNIT         ?PR?LEDDISPLAY?LED
            CODE    44D5H     00ABH     UNIT         ?PR?INTERRUPTUARTAPPTX?UARTAPP
            CODE    4580H     00A7H     UNIT         ?PR?UARTWRCMDPROCESS?UARTAPP
            CODE    4627H     00A2H     UNIT         ?PR?KEYSCAN?KEYSCAN
            CODE    46C9H     00A1H     UNIT         ?PR?SYSPARAINIT?INITIAL
            CODE    476AH     009CH     UNIT         ?PR?_RTCMODIFYTIME?RTC
            CODE    4806H     0097H     UNIT         ?PR?_INTERRUPTUARTAPPRX?UARTAPP
            CODE    489DH     0097H     UNIT         ?PR?_MCUFLASHWRITE?MCUFLASH
            CODE    4934H     0091H     UNIT         ?PR?_UART0INIT?UART
            CODE    49C5H     008DH     UNIT         ?PR?_RTCINITTIME?RTC
            CODE    4A52H     008CH     UNIT         ?PR?_MCUFLASHWRSECTOR?MCUFLASH
            CODE    4ADEH     0088H     UNIT         ?PR?LOWPOWERCHECK?LOWPOWER
            CODE    4B66H     0086H     UNIT         ?PR?_UARTWRITEINFO?UARTAPP
            CODE    4BECH     0086H     UNIT         ?PR?AFEINITREG?AFE
            CODE    4C72H     0081H     UNIT         ?PR?_MCUPWM0SET?MCULIB
            CODE    4CF3H     0081H     UNIT         ?PR?_MCUPWM1SET?MCULIB
            CODE    4D74H     0081H     UNIT         ?PR?_MCUPWM2SET?MCULIB
BL51 BANKED LINKER/LOCATER V6.22                                                      06/21/2022  07:40:42  PAGE 6


            CODE    4DF5H     007DH     UNIT         ?PR?E2PROMINIT?EXTE2PROM
            CODE    4E72H     0079H     UNIT         ?PR?_UARTREADINFO?UARTAPP
            CODE    4EEBH     0078H     UNIT         ?PR?MAIN?MAIN
            CODE    4F63H     0076H     UNIT         ?PR?PROTECTOCRECOVER?PROTECT
            CODE    4FD9H     006FH     UNIT         ?PR?_AFEREADREG?AFE
            CODE    5048H     006DH     UNIT         ?PR?CALIVOLTAGE?CALIBRATE
            CODE    50B5H     006CH     UNIT         ?PR?E2PROMERASE?EXTE2PROM
            CODE    5121H     006BH     UNIT         ?PR?INTERRUPTINT4?INTERRUPT
            CODE    518CH     0069H     UNIT         ?PR?UARTRDE2PROM?EXTE2PROM
            CODE    51F5H     0066H     UNIT         ?PR?RAMCHECKPROCESS?MCULIB
            CODE    525BH     005FH     UNIT         ?PR?_E2PROMWRITE?EXTE2PROM
            CODE    52BAH     005FH     UNIT         ?PR?_E2PROMREAD?EXTE2PROM
            CODE    5319H     005FH     UNIT         ?PR?_MCUFLASHREAD?MCUFLASH
            CODE    5378H     005DH     UNIT         ?PR?AFERAMCHECK?AFE
            CODE    53D5H     005CH     UNIT         ?PR?KEYSWITCHSPEED?KEYAPP
            CODE    5431H     005BH     UNIT         ?PR?_RTCWRITE?RTC
            CODE    548CH     005BH     UNIT         ?PR?_RTCREAD?RTC
            CODE    54E7H     005AH     UNIT         ?PR?_MCUFLASHDATACHECK?MCUFLASH
            CODE    5541H     0059H     UNIT         ?PR?PROTECTOCC?PROTECT
            CODE    559AH     0059H     UNIT         ?PR?PROTECTOCD1?PROTECT
            CODE    55F3H     0059H     UNIT         ?PR?PROTECTOCD2?PROTECT
            CODE    564CH     0056H     UNIT         ?PR?E2PROMBKPROCESS?EXTE2PROM
            CODE    56A2H     0055H     UNIT         ?PR?INITIAL?INITIAL
            CODE    56F7H     0054H     UNIT         ?PR?UARTCALIRTC?UARTAPP
            CODE    574BH     0052H     UNIT         ?PR?UARTCALIVOLTAGE?UARTAPP
            CODE    579DH     0051H     UNIT         ?PR?_MCUCLOCKSET?MCULIB
            CODE    57EEH     0051H     UNIT         ?PR?INTERRUPTUART0?UART
            CODE    583FH     004FH     UNIT         ?PR?CALIPROCESS?CALIBRATE
            CODE    588EH     004FH     UNIT         ?PR?PORPROTECTOTC?PORSELFTEST
            CODE    58DDH     004FH     UNIT         ?PR?PORPROTECTUTC?PORSELFTEST
            CODE    592CH     004FH     UNIT         ?PR?PORPROTECTOTD?PORSELFTEST
            CODE    597BH     004FH     UNIT         ?PR?PORPROTECTUTD?PORSELFTEST
            CODE    59CAH     004EH     UNIT         ?PR?LOADCHECK?CHARGERLOAD
            CODE    5A18H     004CH     UNIT         ?PR?E2PROMBKRTC?EXTE2PROM
            CODE    5A64H     004AH     UNIT         ?PR?AFEGETVOL?CALCULATE
            CODE    5AAEH     004AH     UNIT         ?PR?MOSSTATUSCHECK?MOSCTRL
            CODE    5AF8H     0049H     UNIT         ?PR?UARTCALITS1?UARTAPP
            CODE    5B41H     0049H     UNIT         ?PR?UARTCALITS2?UARTAPP
            CODE    5B8AH     0048H     UNIT         ?CO?UARTAPP
            CODE    5BD2H     0048H     UNIT         ?PR?AFEGETTEMPE?CALCULATE
            CODE    5C1AH     0048H     UNIT         ?PR?_DELAY1MS?MCULIB
            CODE    5C62H     0048H     UNIT         ?PR?PORPROTECTOV?PORSELFTEST
            CODE    5CAAH     0048H     UNIT         ?PR?PORPROTECTUV?PORSELFTEST
            CODE    5CF2H     0046H     UNIT         ?PR?UARTRDRTC?EXTE2PROM
            CODE    5D38H     0045H     UNIT         ?PR?WRITEMANUFACTURE?UARTAPP
            CODE    5D7DH     0045H     UNIT         ?PR?CALITS1?CALIBRATE
            CODE    5DC2H     0045H     UNIT         ?PR?CALITS2?CALIBRATE
            CODE    5E07H     0044H     UNIT         ?PR?CALIRTCTIME?CALIBRATE
            CODE    5E4BH     0044H     UNIT         ?PR?CHGERCHECK?CHARGERLOAD
            CODE    5E8FH     0044H     UNIT         ?C?LDIV
            CODE    5ED3H     0043H     UNIT         ?PR?SYSTEMINTOSLEEP?LOWPOWER
            CODE    5F16H     0042H     UNIT         ?PR?INITVAR?INITIAL
            CODE    5F58H     0041H     UNIT         ?PR?E2PROMBKBOOT?EXTE2PROM
            CODE    5F99H     003FH     UNIT         ?PR?_LEDGETDISNUM?LED
            CODE    5FD8H     003FH     UNIT         ?PR?_AFEBALCTL?AFE
            CODE    6017H     003CH     UNIT         ?PR?AFECLRFLG?AFE
            CODE    6053H     003BH     UNIT         ?PR?LOWPOWERPROCESS?LOWPOWER
BL51 BANKED LINKER/LOCATER V6.22                                                      06/21/2022  07:40:42  PAGE 7


            CODE    608EH     003BH     UNIT         ?PR?CALICURRENTGAIN?CALIBRATE
            CODE    60C9H     003BH     UNIT         ?PR?PORSELFTEST?PORSELFTEST
            CODE    6104H     0039H     UNIT         ?PR?_TWIINIT?TWI
            CODE    613DH     0038H     UNIT         ?PR?WAKEUPPROCESS?LOWPOWER
            CODE    6175H     0037H     UNIT         ?PR?READSUBCLASSID?UARTAPP
            CODE    61ACH     0036H     UNIT         ?PR?UARTCALICUROFFSET?UARTAPP
            CODE    61E2H     0035H     UNIT         ?PR?CTOCHECKVOL?BALANCE
            CODE    6217H     0035H     UNIT         ?PR?_MCUFLASHWRONEBYTE?MCUFLASH
            CODE    624CH     0034H     UNIT         ?CO?CALCULATE
            CODE    6280H     0033H     UNIT         ?PR?AFERDFLG?AFE
            CODE    62B3H     0033H     UNIT         ?PR?CLRRAM?MCULIB
            CODE    62E6H     0033H     UNIT         ?PR?_MEMORYCOPY?MCULIB
            CODE    6319H     0030H     UNIT         ?PR?KEYPROCESS?KEYAPP
            CODE    6349H     002DH     UNIT         ?PR?MOSCTRL?MOSCTRL
            CODE    6376H     002AH     UNIT         ?PR?_MEMORYSET?MCULIB
            CODE    63A0H     0027H     UNIT         ?PR?_MCUFLASHCHECKFLG?MCUFLASH
            CODE    63C7H     0027H     UNIT         ?PR?_TWICHECKSTATUS?TWI
            CODE    63EEH     0026H     UNIT         ?PR?AFEENTERPD?AFE
            CODE    6414H     0026H     UNIT         ?PR?CTOTURNONCHECK?BALANCE
            CODE    643AH     0026H     UNIT         ?PR?_MCUFLASHBLANKCHECK?MCUFLASH
            CODE    6460H     0025H     UNIT         ?PR?SYSTEMRESETPROCESS?MCULIB
            CODE    6485H     0024H     UNIT         ?PR?_INTERRUPTINT4APP?INTERRUPTAPP
            CODE    64A9H     0024H     UNIT         ?PR?INTERRUPTTIMER3APP?INTERRUPTAPP
            CODE    64CDH     001FH     UNIT         ?PR?SYSTEMINTOPD?LOWPOWER
            CODE    64ECH     001FH     UNIT         ?PR?PROTECTPROCESS?PROTECT
            CODE    650BH     001EH     UNIT         ?PR?INITIRQ?INITIAL
            CODE    6529H     001DH     UNIT         ?PR?E2PROMTWICHECK?EXTE2PROM
            CODE    6546H     001DH     UNIT         ?PR?RTCTWICHECK?RTC
            CODE    6563H     001CH     UNIT         ?PR?_CRC8CAL?TWI
            CODE    657FH     001AH     UNIT         ?PR?AFETWICHECK?AFE
            CODE    6599H     0018H     UNIT         ?PR?AFERDSTATUS?AFE
            CODE    65B1H     0017H     UNIT         ?PR?_AFEALARMDIS?AFE
            CODE    65C8H     0015H     UNIT         ?PR?_AFEMOSCTL?AFE
            CODE    65DDH     0015H     UNIT         ?PR?MCUFLASHWRWAITCHECK?MCUFLASH
            CODE    65F2H     0014H     UNIT         ?PR?UARTCHECK?UARTAPP
            CODE    6606H     0014H     UNIT         ?PR?AFEINFOPROCESS?CALCULATE
            CODE    661AH     0014H     UNIT         ?C_C51STARTUP
            CODE    662EH     0013H     UNIT         ?PR?LEDAUTOOFF?LED
            CODE    6641H     0013H     UNIT         ?PR?AFECHGERCHECKEN?AFE
            CODE    6654H     0013H     UNIT         ?PR?AFECHGERCHECKDIS?AFE
            CODE    6667H     0013H     UNIT         ?PR?AFELOADCHECKEN?AFE
            CODE    667AH     0013H     UNIT         ?PR?AFELOADCHECKDIS?AFE
            CODE    668DH     0013H     UNIT         ?PR?AFEWDTEN?AFE
            CODE    66A0H     0013H     UNIT         ?PR?AFEWDTDIS?AFE
            CODE    66B3H     0013H     UNIT         ?PR?AFEADCEN?AFE
            CODE    66C6H     0013H     UNIT         ?PR?AFEADCDIS?AFE
            CODE    66D9H     0013H     UNIT         ?PR?AFECADCEN?AFE
            CODE    66ECH     0013H     UNIT         ?PR?AFECADCDIS?AFE
            CODE    66FFH     0013H     UNIT         ?PR?AFETEMPADCEN?AFE
            CODE    6712H     0013H     UNIT         ?PR?AFETEMPADCDIS?AFE
            CODE    6725H     0013H     UNIT         ?PR?ISPPROCESS?BOOTAPP
            CODE    6738H     0012H     UNIT         ?PR?UARTHANDSHAKE?UARTAPP
            CODE    674AH     0012H     UNIT         ?PR?_AFEALARMEN?AFE
            CODE    675CH     0010H     UNIT         ?PR?AFEINIT?AFE
            CODE    676CH     0010H     UNIT         ?PR?CALICURZERO?CALIBRATE
            CODE    677CH     000CH     UNIT         ?PR?MCUINTOIDLE?MCULIB
            CODE    6788H     000CH     UNIT         ?PR?MCUINTOPD?MCULIB
BL51 BANKED LINKER/LOCATER V6.22                                                      06/21/2022  07:40:42  PAGE 8


            CODE    6794H     000AH     UNIT         ?PR?BALANCEPROCESS?BALANCE
            CODE    679EH     0008H     UNIT         ?PR?_LABS?LABS
                    67A6H     1C5AH                  *** GAP ***
            CODE    8400H     0400H     UNIT         ?CO?DATAFLASH



OVERLAY MAP OF MODULE:   .\output\McuFlash_IAP (MAIN)


SEGMENT                                        BIT_GROUP          DATA_GROUP          IDATA_GROUP         XDATA_GROUP
  +--> CALLED SEGMENT                       START    LENGTH     START    LENGTH     START    LENGTH     START    LENGTH
-----------------------------------------------------------------------------------------------------------------------
?PR?INTERRUPTINT4?INTERRUPT                 -----    -----      -----    -----      -----    -----      -----    -----
  +--> ?PR?_INTERRUPTINT4APP?INTERRUPTAPP

?PR?_INTERRUPTINT4APP?INTERRUPTAPP          -----    -----      -----    -----      -----    -----      -----    -----
  +--> ?PR?_MCUCLOCKSET?MCULIB

*** NEW ROOT ***************************************************

?PR?INTERRUPTTIMER3?INTERRUPT               -----    -----      -----    -----      -----    -----      -----    -----
  +--> ?PR?INTERRUPTTIMER3APP?INTERRUPTAPP

?PR?INTERRUPTTIMER3APP?INTERRUPTAPP         -----    -----      -----    -----      -----    -----      -----    -----
  +--> ?PR?KEYSCAN?KEYSCAN

*** NEW ROOT ***************************************************

?PR?INTERRUPTUART0?UART                     -----    -----      -----    -----      -----    -----      -----    -----
  +--> ?PR?_INTERRUPTUARTAPPRX?UARTAPP
  +--> ?PR?INTERRUPTUARTAPPTX?UARTAPP

?PR?_INTERRUPTUARTAPPRX?UARTAPP             -----    -----      -----    -----      -----    -----      -----    -----
  +--> ?PR?UARTRDCMDPROCESS?UARTAPP
  +--> ?PR?UARTWRCMDPROCESS?UARTAPP
  +--> ?PR?IAPCHECKHANDSHAKE?UARTAPP

?PR?UARTRDCMDPROCESS?UARTAPP                -----    -----      -----    -----      -----    -----      02B5H    0002H
  +--> ?PR?_UARTREADINFO?UARTAPP
  +--> ?CO?UARTAPP

?PR?_UARTREADINFO?UARTAPP                   -----    -----      -----    -----      -----    -----      -----    -----
  +--> ?PR?_CRC8CAL?TWI

?PR?_CRC8CAL?TWI                            -----    -----      -----    -----      -----    -----      -----    -----
  +--> ?CO?TWI

?PR?UARTWRCMDPROCESS?UARTAPP                -----    -----      -----    -----      -----    -----      02B5H    0002H
  +--> ?PR?WRITEMANUFACTURE?UARTAPP
  +--> ?PR?READSUBCLASSID?UARTAPP
  +--> ?PR?UARTCALICURRENT?UARTAPP
  +--> ?PR?UARTCALIVOLTAGE?UARTAPP
  +--> ?PR?UARTCALICUROFFSET?UARTAPP
  +--> ?PR?UARTCALITS1?UARTAPP
  +--> ?PR?UARTCALITS2?UARTAPP
  +--> ?PR?UARTCALIRTC?UARTAPP
BL51 BANKED LINKER/LOCATER V6.22                                                      06/21/2022  07:40:42  PAGE 9


  +--> ?CO?UARTAPP
  +--> ?PR?_UARTWRITEINFO?UARTAPP

?PR?WRITEMANUFACTURE?UARTAPP                -----    -----      -----    -----      -----    -----      -----    -----
  +--> ?PR?_CRC8CAL?TWI

?PR?READSUBCLASSID?UARTAPP                  -----    -----      -----    -----      -----    -----      -----    -----
  +--> ?PR?_CRC8CAL?TWI

?PR?UARTCALICURRENT?UARTAPP                 -----    -----      -----    -----      -----    -----      -----    -----
  +--> ?PR?_CRC8CAL?TWI

?PR?UARTCALIVOLTAGE?UARTAPP                 -----    -----      -----    -----      -----    -----      -----    -----
  +--> ?PR?_CRC8CAL?TWI

?PR?UARTCALICUROFFSET?UARTAPP               -----    -----      -----    -----      -----    -----      -----    -----
  +--> ?PR?_CRC8CAL?TWI

?PR?UARTCALITS1?UARTAPP                     -----    -----      -----    -----      -----    -----      -----    -----
  +--> ?PR?_CRC8CAL?TWI

?PR?UARTCALITS2?UARTAPP                     -----    -----      -----    -----      -----    -----      -----    -----
  +--> ?PR?_CRC8CAL?TWI

?PR?UARTCALIRTC?UARTAPP                     -----    -----      -----    -----      -----    -----      -----    -----
  +--> ?PR?_CRC8CAL?TWI

?PR?_UARTWRITEINFO?UARTAPP                  -----    -----      -----    -----      -----    -----      02B7H    0002H
  +--> ?PR?_CRC8CAL?TWI

?PR?IAPCHECKHANDSHAKE?UARTAPP               -----    -----      -----    -----      -----    -----      02B5H    0002H

*** NEW ROOT ***************************************************

?C_C51STARTUP                               -----    -----      -----    -----      -----    -----      -----    -----
  +--> ?PR?MAIN?MAIN

?PR?MAIN?MAIN                               -----    -----      -----    -----      -----    -----      -----    -----
  +--> ?PR?INITIAL?INITIAL
  +--> ?PR?KEYPROCESS?KEYAPP
  +--> ?PR?AFEINFOPROCESS?CALCULATE
  +--> ?PR?BALANCEPROCESS?BALANCE
  +--> ?PR?PROTECTPROCESS?PROTECT
  +--> ?PR?PORSELFTEST?PORSELFTEST
  +--> ?PR?LOADCHECK?CHARGERLOAD
  +--> ?PR?CHGERCHECK?CHARGERLOAD
  +--> ?PR?MOSCTRL?MOSCTRL
  +--> ?PR?PROTECTOCRECOVER?PROTECT
  +--> ?PR?LEDDISPLAY?LED
  +--> ?PR?UARTCHECK?UARTAPP
  +--> ?PR?GASGAUGEMANAGE?GASGAUGE
  +--> ?PR?AFERAMCHECK?AFE
  +--> ?PR?AFETWICHECK?AFE
  +--> ?PR?E2PROMTWICHECK?EXTE2PROM
  +--> ?PR?RTCTWICHECK?RTC
  +--> ?PR?RAMCHECKPROCESS?MCULIB
  +--> ?PR?SYSPARAINIT?INITIAL
BL51 BANKED LINKER/LOCATER V6.22                                                      06/21/2022  07:40:42  PAGE 10


  +--> ?PR?MCUFLASHWRWAITCHECK?MCUFLASH
  +--> ?PR?E2PROMBKCHECK?EXTE2PROM
  +--> ?PR?LOWPOWERCHECK?LOWPOWER
  +--> ?PR?SYSTEMRESETPROCESS?MCULIB
  +--> ?PR?ISPPROCESS?BOOTAPP
  +--> ?PR?CALIPROCESS?CALIBRATE
  +--> ?PR?MCUFLASHPROCESS?MCUFLASH
  +--> ?PR?E2PROMBKPROCESS?EXTE2PROM
  +--> ?PR?LOWPOWERPROCESS?LOWPOWER

?PR?INITIAL?INITIAL                         -----    -----      -----    -----      -----    -----      -----    -----
  +--> ?PR?_MCUCLOCKSET?MCULIB
  +--> ?PR?INITGPIO?INITIAL
  +--> ?PR?CLRRAM?MCULIB
  +--> ?PR?SYSPARAINIT?INITIAL
  +--> ?PR?INITVAR?INITIAL
  +--> ?PR?_MCUTIMER3SET?MCULIB
  +--> ?PR?_UART0INIT?UART
  +--> ?PR?_TWIINIT?TWI
  +--> ?PR?_MCUPWM2SET?MCULIB
  +--> ?PR?AFEINITREG?AFE
  +--> ?PR?AFEINIT?AFE
  +--> ?PR?AFECLRFLG?AFE
  +--> ?PR?E2PROMINIT?EXTE2PROM
  +--> ?PR?_RTCINITTIME?RTC
  +--> ?PR?INITIRQ?INITIAL

?PR?CLRRAM?MCULIB                           -----    -----      -----    -----      001EH    0002H      -----    -----

?PR?SYSPARAINIT?INITIAL                     -----    -----      -----    -----      -----    -----      -----    -----
  +--> ?PR?_MCUFLASHCHECKFLG?MCUFLASH
  +--> ?PR?_MCUFLASHREAD?MCUFLASH
  +--> ?PR?_MCUFLASHWRITE?MCUFLASH

?PR?_MCUFLASHCHECKFLG?MCUFLASH              0028H.5  0000H.1    -----    -----      -----    -----      -----    -----

?PR?_MCUFLASHREAD?MCUFLASH                  0028H.5  0000H.1    0015H    0002H      -----    -----      02B9H    0004H

?PR?_MCUFLASHWRITE?MCUFLASH                 0028H.7  0000H.1    -----    -----      -----    -----      02BBH    0004H
  +--> ?PR?_MCUFLASHBLANKCHECK?MCUFLASH
  +--> ?PR?_MCUFLASHWRSECTOR?MCUFLASH
  +--> ?PR?_MCUFLASHDATACHECK?MCUFLASH

?PR?_MCUFLASHBLANKCHECK?MCUFLASH            0029H.0  0000H.1    -----    -----      -----    -----      -----    -----

?PR?_MCUFLASHWRSECTOR?MCUFLASH              0029H.0  0000H.1    -----    -----      -----    -----      02BFH    0004H

?PR?_MCUFLASHDATACHECK?MCUFLASH             0029H.0  0000H.1    -----    -----      -----    -----      02BFH    0004H

?PR?INITVAR?INITIAL                         -----    -----      -----    -----      -----    -----      -----    -----
  +--> ?PR?_MEMORYSET?MCULIB

?PR?_MEMORYSET?MCULIB                       -----    -----      -----    -----      -----    -----      02C5H    0002H

?PR?_MCUTIMER3SET?MCULIB                    -----    -----      -----    -----      -----    -----      02B9H    0005H

?PR?_UART0INIT?UART                         -----    -----      -----    -----      -----    -----      02B9H    0002H
BL51 BANKED LINKER/LOCATER V6.22                                                      06/21/2022  07:40:42  PAGE 11



?PR?_MCUPWM2SET?MCULIB                      -----    -----      -----    -----      -----    -----      02B9H    0003H

?PR?AFEINIT?AFE                             0028H.5  0000H.1    -----    -----      -----    -----      -----    -----
  +--> ?PR?_AFEWRITEREG?AFE

?PR?_AFEWRITEREG?AFE                        0028H.6  0000H.1    -----    -----      -----    -----      02BDH    0006H
  +--> ?PR?_TWIWRITE?TWI
  +--> ?PR?_DELAY1MS?MCULIB
  +--> ?PR?_TWIINIT?TWI

?PR?_TWIWRITE?TWI                           0029H.1  0000H.1    -----    -----      -----    -----      02F5H    000EH
  +--> ?PR?_CRC8CAL?TWI
  +--> ?PR?_TWICHECKSTATUS?TWI

?PR?_TWICHECKSTATUS?TWI                     0029H.2  0000H.1    -----    -----      -----    -----      -----    -----

?PR?AFECLRFLG?AFE                           -----    -----      -----    -----      -----    -----      -----    -----
  +--> ?PR?_AFEREADREG?AFE
  +--> ?PR?_AFEWRITEREG?AFE

?PR?_AFEREADREG?AFE                         0028H.6  0000H.1    -----    -----      -----    -----      02C3H    0005H
  +--> ?PR?_TWIREAD?TWI
  +--> ?PR?_DELAY1MS?MCULIB
  +--> ?PR?_TWIINIT?TWI

?PR?_TWIREAD?TWI                            0029H.0  0000H.1    -----    -----      -----    -----      02EBH    003AH
  +--> ?PR?_TWICHECKSTATUS?TWI
  +--> ?PR?_CRC8CAL?TWI

?PR?E2PROMINIT?EXTE2PROM                    0028H.5  0000H.1    -----    -----      -----    -----      02B9H    0008H
  +--> ?PR?_E2PROMREAD?EXTE2PROM

?PR?_E2PROMREAD?EXTE2PROM                   0028H.6  0000H.1    -----    -----      -----    -----      02C5H    0006H
  +--> ?PR?_TWIREAD?TWI
  +--> ?PR?_DELAY1MS?MCULIB

?PR?_RTCINITTIME?RTC                        0028H.5  0000H.1    -----    -----      -----    -----      02B9H    000CH
  +--> ?PR?_MEMORYSET?MCULIB
  +--> ?PR?_E2PROMREAD?EXTE2PROM
  +--> ?PR?_MEMORYCOPY?MCULIB
  +--> ?PR?_RTCREADTIME?RTC

?PR?_MEMORYCOPY?MCULIB                      -----    -----      -----    -----      -----    -----      02DBH    0002H

?PR?_RTCREADTIME?RTC                        0028H.6  0000H.1    -----    -----      -----    -----      02DBH    000BH
  +--> ?PR?_RTCREAD?RTC
  +--> ?PR?_RTCMODIFYTIME?RTC

?PR?_RTCREAD?RTC                            0028H.7  0000H.1    -----    -----      -----    -----      02E6H    0005H
  +--> ?PR?_TWIREAD?TWI
  +--> ?PR?_DELAY1MS?MCULIB

?PR?_RTCMODIFYTIME?RTC                      0028H.7  0000H.1    -----    -----      -----    -----      02E6H    000AH
  +--> ?PR?_RTCWRITE?RTC

?PR?_RTCWRITE?RTC                           0029H.0  0000H.1    -----    -----      -----    -----      02F0H    0005H
BL51 BANKED LINKER/LOCATER V6.22                                                      06/21/2022  07:40:42  PAGE 12


  +--> ?PR?_TWIWRITE?TWI
  +--> ?PR?_DELAY1MS?MCULIB

?PR?KEYPROCESS?KEYAPP                       -----    -----      -----    -----      -----    -----      -----    -----
  +--> ?PR?KEYSWITCHSPEED?KEYAPP

?PR?KEYSWITCHSPEED?KEYAPP                   -----    -----      -----    -----      -----    -----      -----    -----
  +--> ?PR?_MCUPWM2SET?MCULIB

?PR?AFEINFOPROCESS?CALCULATE                -----    -----      -----    -----      -----    -----      -----    -----
  +--> ?PR?AFERDFLG?AFE
  +--> ?PR?AFECALCUVOL?CALCULATE
  +--> ?PR?AFECALCUTEMPE?CALCULATE
  +--> ?PR?AFECALCUCURR?CALCULATE

?PR?AFERDFLG?AFE                            -----    -----      -----    -----      -----    -----      -----    -----
  +--> ?PR?_AFEREADREG?AFE
  +--> ?PR?AFEINIT?AFE

?PR?AFECALCUVOL?CALCULATE                   -----    -----      -----    -----      -----    -----      02B9H    0009H
  +--> ?PR?AFEGETVOL?CALCULATE

?PR?AFEGETVOL?CALCULATE                     0028H.5  0000H.1    -----    -----      -----    -----      02C2H    0001H
  +--> ?PR?_AFEREADREG?AFE

?PR?AFECALCUTEMPE?CALCULATE                 -----    -----      -----    -----      -----    -----      -----    -----
  +--> ?PR?AFEGETTEMPE?CALCULATE
  +--> ?PR?_CALCUTEMP?CALCULATE

?PR?AFEGETTEMPE?CALCULATE                   0028H.5  0000H.1    -----    -----      -----    -----      -----    -----
  +--> ?PR?_AFEREADREG?AFE

?PR?_CALCUTEMP?CALCULATE                    -----    -----      -----    -----      -----    -----      02B9H    0007H
  +--> ?CO?THERMISTOR

?PR?AFECALCUCURR?CALCULATE                  -----    -----      -----    -----      -----    -----      02B9H    0005H
  +--> ?PR?_AFEREADREG?AFE
  +--> ?PR?OFFSETCALCULATE?CALCULATE

?PR?OFFSETCALCULATE?CALCULATE               -----    -----      -----    -----      -----    -----      02BEH    0003H
  +--> ?CO?CALCULATE

?PR?BALANCEPROCESS?BALANCE                  -----    -----      -----    -----      -----    -----      -----    -----
  +--> ?PR?BALTURNONCHECK?BALANCE
  +--> ?PR?CTOTURNONCHECK?BALANCE
  +--> ?PR?BALPROCESS?BALANCE

?PR?BALPROCESS?BALANCE                      -----    -----      -----    -----      -----    -----      02B9H    0002H
  +--> ?PR?_AFEBALCTL?AFE
  +--> ?PR?CTOCHECKVOL?BALANCE

?PR?_AFEBALCTL?AFE                          -----    -----      -----    -----      -----    -----      02BBH    0002H
  +--> ?PR?_AFEWRITEREG?AFE

?PR?CTOCHECKVOL?BALANCE                     0028H.5  0000H.1    -----    -----      -----    -----      -----    -----

?PR?PROTECTPROCESS?PROTECT                  -----    -----      -----    -----      -----    -----      -----    -----
BL51 BANKED LINKER/LOCATER V6.22                                                      06/21/2022  07:40:42  PAGE 13


  +--> ?PR?PROTECTOV?PROTECT
  +--> ?PR?PROTECTUV?PROTECT
  +--> ?PR?PROTECTOTC?PROTECT
  +--> ?PR?PROTECTUTC?PROTECT
  +--> ?PR?PROTECTOTD?PROTECT
  +--> ?PR?PROTECTUTD?PROTECT
  +--> ?PR?PROTECTOCC?PROTECT
  +--> ?PR?PROTECTOCD1?PROTECT
  +--> ?PR?PROTECTOCD2?PROTECT

?PR?PORSELFTEST?PORSELFTEST                 -----    -----      -----    -----      -----    -----      -----    -----
  +--> ?PR?AFECALCUVOL?CALCULATE
  +--> ?PR?AFECALCUTEMPE?CALCULATE
  +--> ?PR?PORPROTECTOV?PORSELFTEST
  +--> ?PR?PORPROTECTUV?PORSELFTEST
  +--> ?PR?PORPROTECTOTC?PORSELFTEST
  +--> ?PR?PORPROTECTUTC?PORSELFTEST
  +--> ?PR?PORPROTECTOTD?PORSELFTEST
  +--> ?PR?PORPROTECTUTD?PORSELFTEST
  +--> ?PR?GASGAUGEINIT?GASGAUGE

?PR?GASGAUGEINIT?GASGAUGE                   -----    -----      -----    -----      -----    -----      02B9H    0001H

?PR?LOADCHECK?CHARGERLOAD                   -----    -----      -----    -----      -----    -----      -----    -----
  +--> ?PR?AFELOADCHECKEN?AFE
  +--> ?PR?AFERDSTATUS?AFE
  +--> ?PR?AFELOADCHECKDIS?AFE
  +--> ?PR?AFECLRFLG?AFE

?PR?AFELOADCHECKEN?AFE                      -----    -----      -----    -----      -----    -----      -----    -----
  +--> ?PR?_AFEWRITEREG?AFE

?PR?AFERDSTATUS?AFE                         -----    -----      -----    -----      -----    -----      02B9H    0002H
  +--> ?PR?_AFEREADREG?AFE

?PR?AFELOADCHECKDIS?AFE                     -----    -----      -----    -----      -----    -----      -----    -----
  +--> ?PR?_AFEWRITEREG?AFE

?PR?CHGERCHECK?CHARGERLOAD                  -----    -----      -----    -----      -----    -----      -----    -----
  +--> ?PR?AFECHGERCHECKEN?AFE
  +--> ?PR?AFERDSTATUS?AFE
  +--> ?PR?AFECHGERCHECKDIS?AFE

?PR?AFECHGERCHECKEN?AFE                     -----    -----      -----    -----      -----    -----      -----    -----
  +--> ?PR?_AFEWRITEREG?AFE

?PR?AFECHGERCHECKDIS?AFE                    -----    -----      -----    -----      -----    -----      -----    -----
  +--> ?PR?_AFEWRITEREG?AFE

?PR?MOSCTRL?MOSCTRL                         -----    -----      -----    -----      -----    -----      -----    -----
  +--> ?PR?MOSSTATUSCHECK?MOSCTRL
  +--> ?PR?_AFEMOSCTL?AFE

?PR?_AFEMOSCTL?AFE                          -----    -----      -----    -----      -----    -----      -----    -----
  +--> ?PR?_AFEWRITEREG?AFE

?PR?PROTECTOCRECOVER?PROTECT                -----    -----      -----    -----      -----    -----      -----    -----
BL51 BANKED LINKER/LOCATER V6.22                                                      06/21/2022  07:40:42  PAGE 14


  +--> ?PR?AFECLRFLG?AFE

?PR?LEDDISPLAY?LED                          -----    -----      -----    -----      -----    -----      -----    -----
  +--> ?PR?_LEDGETDISNUM?LED
  +--> ?PR?LEDAUTOOFF?LED

?PR?GASGAUGEMANAGE?GASGAUGE                 -----    -----      -----    -----      -----    -----      02B9H    0002H
  +--> ?PR?CORRECTCHGSOC?GASGAUGELIB
  +--> ?PR?CORRECTDSGSOC?GASGAUGELIB
  +--> ?PR?DATAFILTER?GASGAUGELIB

?PR?CORRECTCHGSOC?GASGAUGELIB               -----    -----      -----    -----      -----    -----      02BBH    0001H

?PR?CORRECTDSGSOC?GASGAUGELIB               -----    -----      -----    -----      -----    -----      02BBH    0009H
  +--> ?PR?_LABS?LABS

?PR?DATAFILTER?GASGAUGELIB                  -----    -----      -----    -----      -----    -----      02BBH    000CH

?PR?AFERAMCHECK?AFE                         -----    -----      -----    -----      -----    -----      02B9H    0003H
  +--> ?PR?_AFEREADREG?AFE
  +--> ?PR?AFEINIT?AFE

?PR?E2PROMBKCHECK?EXTE2PROM                 -----    -----      -----    -----      -----    -----      -----    -----
  +--> ?PR?_RTCREADTIME?RTC
  +--> ?PR?_MEMORYCOPY?MCULIB

?PR?ISPPROCESS?BOOTAPP                      -----    -----      -----    -----      -----    -----      -----    -----
  +--> ?PR?AFEWDTDIS?AFE

?PR?AFEWDTDIS?AFE                           -----    -----      -----    -----      -----    -----      -----    -----
  +--> ?PR?_AFEWRITEREG?AFE

?PR?CALIPROCESS?CALIBRATE                   -----    -----      -----    -----      -----    -----      -----    -----
  +--> ?PR?CALIVOLTAGE?CALIBRATE
  +--> ?PR?CALICURRENTGAIN?CALIBRATE
  +--> ?PR?CALICURZERO?CALIBRATE
  +--> ?PR?CALITS1?CALIBRATE
  +--> ?PR?CALITS2?CALIBRATE
  +--> ?PR?CALIRTCTIME?CALIBRATE

?PR?CALIVOLTAGE?CALIBRATE                   -----    -----      -----    -----      -----    -----      02B9H    0002H

?PR?CALITS1?CALIBRATE                       -----    -----      -----    -----      -----    -----      -----    -----
  +--> ?PR?_CALCUTEMP?CALCULATE

?PR?CALITS2?CALIBRATE                       -----    -----      -----    -----      -----    -----      -----    -----
  +--> ?PR?_CALCUTEMP?CALCULATE

?PR?CALIRTCTIME?CALIBRATE                   -----    -----      -----    -----      -----    -----      -----    -----
  +--> ?PR?_RTCMODIFYTIME?RTC

?PR?MCUFLASHPROCESS?MCUFLASH                0028H.5  0000H.2    -----    -----      -----    -----      02B9H    0002H
  +--> ?PR?_MCUFLASHWRITE?MCUFLASH
  +--> ?PR?_MCUFLASHWRONEBYTE?MCUFLASH

?PR?E2PROMBKPROCESS?EXTE2PROM               -----    -----      -----    -----      -----    -----      02B9H    0001H
  +--> ?PR?E2PROMERASE?EXTE2PROM
BL51 BANKED LINKER/LOCATER V6.22                                                      06/21/2022  07:40:42  PAGE 15


  +--> ?PR?UARTRDE2PROM?EXTE2PROM
  +--> ?PR?UARTRDRTC?EXTE2PROM
  +--> ?PR?E2PROMBKRTC?EXTE2PROM
  +--> ?PR?_E2PROMBKDATA?EXTE2PROM

?PR?E2PROMERASE?EXTE2PROM                   -----    -----      -----    -----      -----    -----      02BAH    000AH
  +--> ?PR?_MEMORYSET?MCULIB
  +--> ?PR?_E2PROMWRITE?EXTE2PROM

?PR?_E2PROMWRITE?EXTE2PROM                  0028H.5  0000H.1    -----    -----      -----    -----      02E3H    0006H
  +--> ?PR?_TWIWRITE?TWI
  +--> ?PR?_DELAY1MS?MCULIB

?PR?UARTRDE2PROM?EXTE2PROM                  -----    -----      -----    -----      -----    -----      -----    -----
  +--> ?PR?_E2PROMREAD?EXTE2PROM
  +--> ?PR?_CRC8CAL?TWI

?PR?UARTRDRTC?EXTE2PROM                     -----    -----      -----    -----      -----    -----      -----    -----
  +--> ?PR?_RTCREADTIME?RTC
  +--> ?PR?_MEMORYCOPY?MCULIB
  +--> ?PR?_CRC8CAL?TWI

?PR?E2PROMBKRTC?EXTE2PROM                   -----    -----      -----    -----      -----    -----      02BAH    000AH
  +--> ?PR?_RTCREADTIME?RTC
  +--> ?PR?_MEMORYCOPY?MCULIB
  +--> ?PR?_E2PROMWRITE?EXTE2PROM

?PR?_E2PROMBKDATA?EXTE2PROM                 -----    -----      -----    -----      -----    -----      02BAH    0021H
  +--> ?PR?_MEMORYCOPY?MCULIB
  +--> ?PR?_RTCREADTIME?RTC
  +--> ?PR?_E2PROMWRITE?EXTE2PROM
  +--> ?PR?E2PROMBKBOOT?EXTE2PROM

?PR?E2PROMBKBOOT?EXTE2PROM                  -----    -----      -----    -----      -----    -----      02DBH    0008H
  +--> ?PR?_E2PROMWRITE?EXTE2PROM

?PR?LOWPOWERPROCESS?LOWPOWER                -----    -----      -----    -----      -----    -----      -----    -----
  +--> ?PR?MCUINTOIDLE?MCULIB
  +--> ?PR?SYSTEMINTOPD?LOWPOWER
  +--> ?PR?SYSTEMINTOSLEEP?LOWPOWER
  +--> ?PR?WAKEUPPROCESS?LOWPOWER

?PR?SYSTEMINTOPD?LOWPOWER                   -----    -----      -----    -----      -----    -----      -----    -----
  +--> ?PR?_AFEMOSCTL?AFE
  +--> ?PR?AFEENTERPD?AFE

?PR?AFEENTERPD?AFE                          -----    -----      -----    -----      -----    -----      -----    -----
  +--> ?PR?_AFEWRITEREG?AFE

?PR?SYSTEMINTOSLEEP?LOWPOWER                -----    -----      -----    -----      -----    -----      -----    -----
  +--> ?PR?AFEWDTDIS?AFE
  +--> ?PR?AFETEMPADCDIS?AFE
  +--> ?PR?_AFEALARMEN?AFE
  +--> ?PR?_DELAY1MS?MCULIB
  +--> ?PR?_MCUCLOCKSET?MCULIB
  +--> ?PR?MCUINTOPD?MCULIB

BL51 BANKED LINKER/LOCATER V6.22                                                      06/21/2022  07:40:42  PAGE 16


?PR?AFETEMPADCDIS?AFE                       -----    -----      -----    -----      -----    -----      -----    -----
  +--> ?PR?_AFEWRITEREG?AFE

?PR?_AFEALARMEN?AFE                         -----    -----      -----    -----      -----    -----      -----    -----
  +--> ?PR?_AFEWRITEREG?AFE

?PR?WAKEUPPROCESS?LOWPOWER                  -----    -----      -----    -----      -----    -----      -----    -----
  +--> ?PR?_MCUCLOCKSET?MCULIB
  +--> ?PR?_DELAY1MS?MCULIB
  +--> ?PR?_AFEALARMDIS?AFE
  +--> ?PR?AFETEMPADCEN?AFE
  +--> ?PR?AFEWDTEN?AFE

?PR?_AFEALARMDIS?AFE                        -----    -----      -----    -----      -----    -----      -----    -----
  +--> ?PR?_AFEWRITEREG?AFE

?PR?AFETEMPADCEN?AFE                        -----    -----      -----    -----      -----    -----      -----    -----
  +--> ?PR?_AFEWRITEREG?AFE

?PR?AFEWDTEN?AFE                            -----    -----      -----    -----      -----    -----      -----    -----
  +--> ?PR?_AFEWRITEREG?AFE



SYMBOL TABLE OF MODULE:  .\output\McuFlash_IAP (MAIN)

  VALUE           TYPE          NAME
  ----------------------------------

  -------         MODULE        MAIN
  C:0000H         SYMBOL        _ICE_DUMMY_
  D:0080H         PUBLIC        P0
  D:0090H         PUBLIC        P1
  D:00A0H         PUBLIC        P2
  D:00B0H         PUBLIC        P3
  D:00C0H         PUBLIC        P4
  D:0080H         PUBLIC        P5
  C:4EEBH         PUBLIC        main
  D:00B1H         PUBLIC        RSTSTAT
  -------         PROC          MAIN
  C:4EEBH         LINE#         21
  C:4EEBH         LINE#         22
  C:4EEBH         LINE#         23
  C:4EEEH         LINE#         25
  C:4EEEH         LINE#         26
  C:4EEEH         LINE#         27
  C:4EF1H         LINE#         29
  C:4EF4H         LINE#         31
  C:4EF7H         LINE#         32
  C:4EF7H         LINE#         33
  C:4EF9H         LINE#         34
  C:4EFCH         LINE#         36
  C:4EFFH         LINE#         38
  C:4F02H         LINE#         40
  C:4F05H         LINE#         42
  C:4F08H         LINE#         44
  C:4F0BH         LINE#         46
BL51 BANKED LINKER/LOCATER V6.22                                                      06/21/2022  07:40:42  PAGE 17


  C:4F0EH         LINE#         48
  C:4F11H         LINE#         50
  C:4F14H         LINE#         52
  C:4F17H         LINE#         53
  C:4F17H         LINE#         55
  C:4F1AH         LINE#         56
  C:4F1AH         LINE#         57
  C:4F1CH         LINE#         58
  C:4F1FH         LINE#         60
  C:4F22H         LINE#         62
  C:4F25H         LINE#         63
  C:4F28H         LINE#         64
  C:4F2BH         LINE#         66
  C:4F30H         LINE#         67
  C:4F30H         LINE#         68
  C:4F33H         LINE#         69
  C:4F33H         LINE#         71
  C:4F36H         LINE#         73
  C:4F39H         LINE#         75
  C:4F3CH         LINE#         76
  C:4F3CH         LINE#         78
  C:4F3FH         LINE#         80
  C:4F42H         LINE#         82
  C:4F45H         LINE#         84
  C:4F48H         LINE#         86
  C:4F4BH         LINE#         88
  C:4F4EH         LINE#         90
  C:4F58H         LINE#         91
  C:4F60H         LINE#         92
  -------         ENDPROC       MAIN
  -------         ENDMOD        MAIN

  -------         MODULE        INITIAL
  C:0000H         SYMBOL        _ICE_DUMMY_
  D:0080H         PUBLIC        P0
  D:0090H         PUBLIC        P1
  D:00A0H         PUBLIC        P2
  D:00B0H         PUBLIC        P3
  C:650BH         PUBLIC        InitIRQ
  D:00C0H         PUBLIC        P4
  D:0080H         PUBLIC        P5
  B:00A8H.7       PUBLIC        EA
  D:00A9H         PUBLIC        IEN1
  D:00E8H         PUBLIC        EXF0
  D:00D8H         PUBLIC        EXF1
  D:00E1H         PUBLIC        P0CR
  D:00E2H         PUBLIC        P1CR
  D:00E3H         PUBLIC        P2CR
  D:00E4H         PUBLIC        P3CR
  D:00BAH         PUBLIC        IENC
  C:5F16H         PUBLIC        InitVar
  C:102EH         PUBLIC        InitGPIO
  B:00A8H.4       PUBLIC        ES0
  B:00A8H.5       PUBLIC        ET3
  D:0086H         PUBLIC        INSCON
  B:0088H.7       PUBLIC        TF3
  C:56A2H         PUBLIC        Initial
BL51 BANKED LINKER/LOCATER V6.22                                                      06/21/2022  07:40:42  PAGE 18


  C:46C9H         PUBLIC        SysParaInit
  D:00E9H         PUBLIC        P0PCR
  D:00EAH         PUBLIC        P1PCR
  D:00EBH         PUBLIC        P2PCR
  D:00ECH         PUBLIC        P3PCR
  -------         PROC          INITVAR
  C:5F16H         LINE#         18
  C:5F16H         LINE#         19
  C:5F16H         LINE#         20
  C:5F1CH         LINE#         21
  C:5F27H         LINE#         22
  C:5F31H         LINE#         23
  C:5F3BH         LINE#         24
  C:5F43H         LINE#         26
  C:5F45H         LINE#         27
  C:5F47H         LINE#         28
  C:5F4DH         LINE#         29
  C:5F4FH         LINE#         30
  C:5F51H         LINE#         32
  C:5F57H         LINE#         33
  -------         ENDPROC       INITVAR
  -------         PROC          SYSPARAINIT
  C:46C9H         LINE#         41
  C:46C9H         LINE#         42
  C:46C9H         LINE#         43
  C:46D2H         LINE#         44
  C:46D2H         LINE#         45
  C:46DEH         LINE#         46
  C:46E7H         LINE#         47
  C:46E7H         LINE#         48
  C:46EFH         LINE#         49
  C:46EFH         LINE#         50
  C:46F1H         LINE#         51
  C:46FAH         LINE#         52
  C:46FAH         LINE#         53
  C:4707H         LINE#         54
  C:470EH         LINE#         55
  C:4710H         LINE#         57
  C:4710H         LINE#         58
  C:4713H         LINE#         60
  C:4713H         LINE#         62
  C:471DH         LINE#         63
  C:4727H         LINE#         64
  C:4733H         LINE#         65
  C:4742H         LINE#         67
  C:474AH         LINE#         69
  C:4753H         LINE#         70
  C:4753H         LINE#         71
  C:4756H         LINE#         72
  C:4757H         LINE#         73
  C:4762H         LINE#         74
  C:4762H         LINE#         75
  C:4765H         LINE#         76
  C:4766H         LINE#         78
  C:4766H         LINE#         79
  C:4769H         LINE#         80
  C:4769H         LINE#         81
BL51 BANKED LINKER/LOCATER V6.22                                                      06/21/2022  07:40:42  PAGE 19


  -------         ENDPROC       SYSPARAINIT
  -------         PROC          INITIRQ
  C:650BH         LINE#         89
  C:650BH         LINE#         90
  C:650BH         LINE#         91
  C:650DH         LINE#         93
  C:650FH         LINE#         95
  C:6518H         LINE#         96
  C:651AH         LINE#         98
  C:651DH         LINE#         99
  C:6520H         LINE#         100
  C:6523H         LINE#         101
  C:6526H         LINE#         103
  C:6528H         LINE#         104
  -------         ENDPROC       INITIRQ
  -------         PROC          INITGPIO
  C:102EH         LINE#         131
  C:102EH         LINE#         132
  C:102EH         LINE#         133
  C:1031H         LINE#         134
  C:1034H         LINE#         135
  C:1037H         LINE#         137
  C:103AH         LINE#         138
  C:103DH         LINE#         139
  C:1040H         LINE#         141
  C:1043H         LINE#         142
  C:1046H         LINE#         143
  C:1049H         LINE#         145
  C:104CH         LINE#         146
  C:104FH         LINE#         147
  C:1052H         LINE#         148
  -------         ENDPROC       INITGPIO
  -------         PROC          INITIAL
  C:56A2H         LINE#         156
  C:56A2H         LINE#         157
  C:56A2H         LINE#         158
  C:56A7H         LINE#         160
  C:56AAH         LINE#         162
  C:56ADH         LINE#         164
  C:56B0H         LINE#         166
  C:56B3H         LINE#         168
  C:56BCH         LINE#         170
  C:56C3H         LINE#         172
  C:56C8H         LINE#         174
  C:56D1H         LINE#         176
  C:56D4H         LINE#         177
  C:56D9H         LINE#         178
  C:56D9H         LINE#         179
  C:56DBH         LINE#         180
  C:56DBH         LINE#         181
  C:56DEH         LINE#         183
  C:56E1H         LINE#         184
  C:56E1H         LINE#         185
  C:56E6H         LINE#         186
  C:56E6H         LINE#         187
  C:56E8H         LINE#         188
  C:56E8H         LINE#         190
BL51 BANKED LINKER/LOCATER V6.22                                                      06/21/2022  07:40:42  PAGE 20


  C:56F1H         LINE#         191
  C:56F1H         LINE#         192
  C:56F3H         LINE#         193
  C:56F3H         LINE#         194
  C:56F3H         LINE#         196
  C:56F6H         LINE#         197
  -------         ENDPROC       INITIAL
  -------         ENDMOD        INITIAL

  -------         MODULE        INTERRUPTAPP
  C:0000H         SYMBOL        _ICE_DUMMY_
  D:0080H         PUBLIC        P0
  D:0090H         PUBLIC        P1
  D:00A0H         PUBLIC        P2
  X:0398H         PUBLIC        ucTimer1s
  D:00B0H         PUBLIC        P3
  D:00C0H         PUBLIC        P4
  D:0080H         PUBLIC        P5
  C:6485H         PUBLIC        _InterruptINT4App
  B:002CH.5       PUBLIC        bTimer5msFlg
  X:0399H         PUBLIC        ucTimer50ms
  B:002CH.6       PUBLIC        bTimer1sFlg
  C:64A9H         PUBLIC        InterruptTimer3App
  B:002CH.7       PUBLIC        bTimer50msFlg
  -------         PROC          _INTERRUPTINT4APP
  D:0007H         SYMBOL        IntSource
  C:6485H         LINE#         24
  C:6485H         LINE#         25
  C:6485H         LINE#         26
  C:6489H         LINE#         27
  C:6489H         LINE#         28
  C:648FH         LINE#         29
  C:648FH         LINE#         30
  C:6494H         LINE#         31
  C:6496H         LINE#         32
  C:6496H         LINE#         33
  C:6497H         LINE#         34
  C:649BH         LINE#         35
  C:649BH         LINE#         36
  C:64A1H         LINE#         37
  C:64A1H         LINE#         38
  C:64A6H         LINE#         39
  C:64A8H         LINE#         40
  C:64A8H         LINE#         41
  C:64A8H         LINE#         42
  -------         ENDPROC       _INTERRUPTINT4APP
  -------         PROC          INTERRUPTTIMER3APP
  C:64A9H         LINE#         51
  C:64A9H         LINE#         52
  C:64A9H         LINE#         53
  C:64ABH         LINE#         55
  C:64B6H         LINE#         56
  C:64B6H         LINE#         57
  C:64B8H         LINE#         58
  C:64BAH         LINE#         59
  C:64BAH         LINE#         61
  C:64C5H         LINE#         62
BL51 BANKED LINKER/LOCATER V6.22                                                      06/21/2022  07:40:42  PAGE 21


  C:64C5H         LINE#         63
  C:64C7H         LINE#         64
  C:64C9H         LINE#         65
  C:64C9H         LINE#         67
  C:64CCH         LINE#         68
  -------         ENDPROC       INTERRUPTTIMER3APP
  -------         ENDMOD        INTERRUPTAPP

  -------         MODULE        LED
  C:0000H         SYMBOL        _ICE_DUMMY_
  D:0080H         PUBLIC        P0
  D:0090H         PUBLIC        P1
  D:00A0H         PUBLIC        P2
  D:00B0H         PUBLIC        P3
  D:00C0H         PUBLIC        P4
  D:0080H         PUBLIC        P5
  C:5F99H         PUBLIC        _LedGetDisNum
  B:00A0H.0       PUBLIC        P2_0
  B:00A0H.1       PUBLIC        P2_1
  B:00A0H.2       PUBLIC        P2_2
  B:00A0H.3       PUBLIC        P2_3
  B:00A0H.4       PUBLIC        P2_4
  X:038CH         PUBLIC        ucLedChgFlickCnt
  B:00B0H.5       PUBLIC        P3_5
  X:038DH         PUBLIC        ucLedBleFlickCnt
  X:038EH         PUBLIC        ucLedTimeCnt
  B:002DH.3       PUBLIC        bLedDisFlg
  B:002DH.4       PUBLIC        bLedDisBleFlg
  C:662EH         PUBLIC        LedAutoOff
  C:4428H         PUBLIC        LedDisplay
  -------         PROC          _LEDGETDISNUM
  D:0006H         SYMBOL        Rsoc
  C:5F99H         LINE#         24
  C:5F99H         LINE#         25
  C:5F99H         LINE#         26
  C:5FA2H         LINE#         27
  C:5FA2H         LINE#         28
  C:5FA5H         LINE#         29
  C:5FA5H         LINE#         30
  C:5FAEH         LINE#         31
  C:5FAEH         LINE#         32
  C:5FB1H         LINE#         33
  C:5FB1H         LINE#         34
  C:5FBAH         LINE#         35
  C:5FBAH         LINE#         36
  C:5FBDH         LINE#         37
  C:5FBDH         LINE#         38
  C:5FC6H         LINE#         39
  C:5FC6H         LINE#         40
  C:5FC9H         LINE#         41
  C:5FC9H         LINE#         42
  C:5FD2H         LINE#         43
  C:5FD2H         LINE#         44
  C:5FD5H         LINE#         45
  C:5FD5H         LINE#         47
  C:5FD5H         LINE#         48
  C:5FD7H         LINE#         49
BL51 BANKED LINKER/LOCATER V6.22                                                      06/21/2022  07:40:42  PAGE 22


  C:5FD7H         LINE#         50
  -------         ENDPROC       _LEDGETDISNUM
  -------         PROC          LEDAUTOOFF
  C:662EH         LINE#         59
  C:662EH         LINE#         60
  C:662EH         LINE#         61
  C:6631H         LINE#         62
  C:6631H         LINE#         63
  C:663CH         LINE#         64
  C:663CH         LINE#         65
  C:663EH         LINE#         66
  C:6640H         LINE#         67
  C:6640H         LINE#         68
  C:6640H         LINE#         69
  -------         ENDPROC       LEDAUTOOFF
  -------         PROC          LEDDISPLAY
  -------         DO            
  D:0007H         SYMBOL        LedDisNum
  -------         ENDDO         
  C:4428H         LINE#         80
  C:4428H         LINE#         81
  C:4428H         LINE#         84
  C:442BH         LINE#         85
  C:442BH         LINE#         86
  C:4436H         LINE#         87
  C:4436H         LINE#         88
  C:4438H         LINE#         89
  C:443DH         LINE#         90
  C:443DH         LINE#         91
  C:443FH         LINE#         93
  C:443FH         LINE#         94
  C:4441H         LINE#         95
  C:4441H         LINE#         97
  C:4444H         LINE#         98
  C:4444H         LINE#         99
  C:444FH         LINE#         100
  C:444FH         LINE#         101
  C:4451H         LINE#         102
  C:4456H         LINE#         103
  C:4456H         LINE#         104
  C:4458H         LINE#         106
  C:4458H         LINE#         107
  C:445AH         LINE#         108
  C:445AH         LINE#         110
  C:445DH         LINE#         111
  C:445DH         LINE#         112
  C:4468H         LINE#         113
  C:446BH         LINE#         114
  C:446BH         LINE#         115
  C:4478H         LINE#         116
  C:4478H         LINE#         117
  C:447CH         LINE#         118
  C:447CH         LINE#         119
  C:4481H         LINE#         120
  C:4483H         LINE#         121
  C:4487H         LINE#         122
  C:4487H         LINE#         123
BL51 BANKED LINKER/LOCATER V6.22                                                      06/21/2022  07:40:42  PAGE 23


  C:448CH         LINE#         124
  C:448EH         LINE#         125
  C:4490H         LINE#         126
  C:4494H         LINE#         127
  C:4494H         LINE#         128
  C:4499H         LINE#         129
  C:449BH         LINE#         130
  C:449DH         LINE#         131
  C:449FH         LINE#         132
  C:44A3H         LINE#         133
  C:44A3H         LINE#         134
  C:44A8H         LINE#         135
  C:44AAH         LINE#         136
  C:44ACH         LINE#         137
  C:44AEH         LINE#         138
  C:44B0H         LINE#         139
  C:44B5H         LINE#         140
  C:44B5H         LINE#         141
  C:44C2H         LINE#         142
  C:44C2H         LINE#         143
  C:44C4H         LINE#         145
  C:44C4H         LINE#         146
  C:44D1H         LINE#         147
  C:44D1H         LINE#         149
  C:44D4H         LINE#         150
  -------         ENDPROC       LEDDISPLAY
  -------         ENDMOD        LED

  -------         MODULE        KEYAPP
  C:0000H         SYMBOL        _ICE_DUMMY_
  D:0080H         PUBLIC        P0
  D:0090H         PUBLIC        P1
  D:00A0H         PUBLIC        P2
  D:00B0H         PUBLIC        P3
  D:00C0H         PUBLIC        P4
  D:0080H         PUBLIC        P5
  D:00B7H         PUBLIC        PWM2CON
  C:6319H         PUBLIC        KeyProcess
  B:0080H.3       PUBLIC        P0_3
  C:53D5H         PUBLIC        KeySwitchSpeed
  X:03A0H         PUBLIC        ucDsgingSpeed
  -------         PROC          KEYSWITCHSPEED
  C:53D5H         LINE#         20
  C:53D5H         LINE#         21
  C:53D5H         LINE#         22
  C:53D7H         LINE#         23
  C:53D9H         LINE#         24
  C:53DBH         LINE#         26
  C:53E1H         LINE#         27
  C:53E1H         LINE#         28
  C:53E3H         LINE#         29
  C:53E5H         LINE#         30
  C:53F5H         LINE#         31
  C:53F8H         LINE#         32
  C:53F9H         LINE#         33
  C:5400H         LINE#         34
  C:5400H         LINE#         35
BL51 BANKED LINKER/LOCATER V6.22                                                      06/21/2022  07:40:42  PAGE 24


  C:5403H         LINE#         36
  C:5405H         LINE#         37
  C:5412H         LINE#         38
  C:5415H         LINE#         39
  C:5416H         LINE#         41
  C:5416H         LINE#         42
  C:541BH         LINE#         43
  C:541DH         LINE#         44
  C:542DH         LINE#         45
  C:5430H         LINE#         46
  C:5430H         LINE#         47
  -------         ENDPROC       KEYSWITCHSPEED
  -------         PROC          KEYPROCESS
  C:6319H         LINE#         56
  C:6319H         LINE#         57
  C:6319H         LINE#         58
  C:631CH         LINE#         59
  C:631CH         LINE#         60
  C:631EH         LINE#         61
  C:632FH         LINE#         62
  C:632FH         LINE#         63
  C:632FH         LINE#         64
  C:6332H         LINE#         65
  C:6333H         LINE#         67
  C:6333H         LINE#         68
  C:6335H         LINE#         69
  C:633AH         LINE#         70
  C:633BH         LINE#         72
  C:633BH         LINE#         73
  C:633DH         LINE#         74
  C:633EH         LINE#         76
  C:633EH         LINE#         77
  C:6340H         LINE#         78
  C:6343H         LINE#         79
  C:6343H         LINE#         80
  C:6345H         LINE#         81
  C:6346H         LINE#         83
  C:6346H         LINE#         84
  C:6348H         LINE#         85
  C:6348H         LINE#         86
  C:6348H         LINE#         88
  C:6348H         LINE#         89
  C:6348H         LINE#         90
  C:6348H         LINE#         91
  C:6348H         LINE#         92
  -------         ENDPROC       KEYPROCESS
  -------         ENDMOD        KEYAPP

  -------         MODULE        LOWPOWER
  C:0000H         SYMBOL        _ICE_DUMMY_
  D:0080H         PUBLIC        P0
  D:0090H         PUBLIC        P1
  X:038FH         PUBLIC        ucSleepTimerCnt
  D:00A0H         PUBLIC        P2
  D:00B0H         PUBLIC        P3
  D:00C0H         PUBLIC        P4
  D:0080H         PUBLIC        P5
BL51 BANKED LINKER/LOCATER V6.22                                                      06/21/2022  07:40:42  PAGE 25


  B:00A8H.7       PUBLIC        EA
  B:00C8H.6       PUBLIC        ENTWI
  D:00B7H         PUBLIC        PWM2CON
  B:002AH.5       PUBLIC        bPDFlg
  B:00A0H.0       PUBLIC        P2_0
  B:0080H.3       PUBLIC        P0_3
  B:00A0H.1       PUBLIC        P2_1
  B:00A0H.2       PUBLIC        P2_2
  B:00A0H.3       PUBLIC        P2_3
  D:00D8H         PUBLIC        EXF1
  B:00A0H.4       PUBLIC        P2_4
  B:00A0H.5       PUBLIC        P2_5
  X:0390H         PUBLIC        ucPDTimerCnt
  C:5ED3H         PUBLIC        SystemIntoSleep
  C:4ADEH         PUBLIC        LowPowerCheck
  B:002AH.6       PUBLIC        bPCEnterPDFlg
  C:6053H         PUBLIC        LowPowerProcess
  C:613DH         PUBLIC        WakeUpProcess
  D:00B1H         PUBLIC        RSTSTAT
  C:64CDH         PUBLIC        SystemIntoPD
  B:00A8H.4       PUBLIC        ES0
  B:00A8H.5       PUBLIC        ET3
  X:0391H         PUBLIC        ucResetFlag
  B:002AH.7       PUBLIC        bWakeupFlg
  B:002BH.0       PUBLIC        bSleepFlg
  -------         PROC          WAKEUPPROCESS
  C:613DH         LINE#         26
  C:613DH         LINE#         27
  C:613DH         LINE#         28
  C:6140H         LINE#         29
  C:6140H         LINE#         30
  C:6142H         LINE#         31
  C:6145H         LINE#         32
  C:6145H         LINE#         33
  C:614AH         LINE#         34
  C:614CH         LINE#         36
  C:614EH         LINE#         37
  C:6153H         LINE#         38
  C:6158H         LINE#         40
  C:615AH         LINE#         41
  C:615CH         LINE#         42
  C:615EH         LINE#         44
  C:6163H         LINE#         45
  C:6166H         LINE#         46
  C:6169H         LINE#         47
  C:6169H         LINE#         48
  C:616EH         LINE#         49
  C:6170H         LINE#         50
  C:6174H         LINE#         51
  C:6174H         LINE#         52
  -------         ENDPROC       WAKEUPPROCESS
  -------         PROC          SYSTEMINTOPD
  C:64CDH         LINE#         61
  C:64CDH         LINE#         62
  C:64CDH         LINE#         63
  C:64CDH         LINE#         64
  C:64CDH         LINE#         65
BL51 BANKED LINKER/LOCATER V6.22                                                      06/21/2022  07:40:42  PAGE 26


  C:64D0H         LINE#         67
  C:64D2H         LINE#         68
  C:64DFH         LINE#         69
  C:64E1H         LINE#         70
  C:64E6H         LINE#         72
  C:64E9H         LINE#         73
  -------         ENDPROC       SYSTEMINTOPD
  -------         PROC          SYSTEMINTOSLEEP
  C:5ED3H         LINE#         83
  C:5ED3H         LINE#         84
  C:5ED3H         LINE#         85
  C:5EE0H         LINE#         86
  C:5EE2H         LINE#         87
  C:5EE4H         LINE#         89
  C:5EE7H         LINE#         90
  C:5EEAH         LINE#         91
  C:5EEFH         LINE#         92
  C:5EF1H         LINE#         93
  C:5EF4H         LINE#         94
  C:5EF7H         LINE#         95
  C:5EF7H         LINE#         96
  C:5EF9H         LINE#         97
  C:5EFBH         LINE#         99
  C:5EFBH         LINE#         100
  C:5EFDH         LINE#         101
  C:5EFDH         LINE#         102
  C:5F02H         LINE#         104
  C:5F04H         LINE#         105
  C:5F06H         LINE#         106
  C:5F08H         LINE#         107
  C:5F0BH         LINE#         108
  C:5F10H         LINE#         109
  C:5F12H         LINE#         111
  C:5F15H         LINE#         112
  -------         ENDPROC       SYSTEMINTOSLEEP
  -------         PROC          LOWPOWERCHECK
  C:4ADEH         LINE#         123
  C:4ADEH         LINE#         124
  C:4ADEH         LINE#         125
  C:4AE4H         LINE#         126
  C:4AE4H         LINE#         127
  C:4AE6H         LINE#         128
  C:4AE8H         LINE#         129
  C:4AE9H         LINE#         130
  C:4AECH         LINE#         131
  C:4AECH         LINE#         132
  C:4AFBH         LINE#         133
  C:4AFBH         LINE#         134
  C:4AFDH         LINE#         135
  C:4AFFH         LINE#         136
  C:4AFFH         LINE#         137
  C:4B00H         LINE#         138
  C:4B03H         LINE#         139
  C:4B03H         LINE#         140
  C:4B09H         LINE#         141
  C:4B09H         LINE#         142
  C:4B0CH         LINE#         143
BL51 BANKED LINKER/LOCATER V6.22                                                      06/21/2022  07:40:42  PAGE 27


  C:4B0CH         LINE#         144
  C:4B1BH         LINE#         145
  C:4B1BH         LINE#         146
  C:4B1DH         LINE#         147
  C:4B1FH         LINE#         148
  C:4B1FH         LINE#         149
  C:4B20H         LINE#         151
  C:4B20H         LINE#         152
  C:4B25H         LINE#         153
  C:4B3DH         LINE#         154
  C:4B3DH         LINE#         155
  C:4B4BH         LINE#         156
  C:4B4BH         LINE#         157
  C:4B4DH         LINE#         158
  C:4B4FH         LINE#         159
  C:4B4FH         LINE#         160
  C:4B50H         LINE#         162
  C:4B50H         LINE#         163
  C:4B55H         LINE#         164
  C:4B55H         LINE#         165
  C:4B55H         LINE#         166
  C:4B56H         LINE#         168
  C:4B56H         LINE#         169
  C:4B5BH         LINE#         170
  C:4B5DH         LINE#         171
  C:4B5DH         LINE#         172
  C:4B5EH         LINE#         174
  C:4B5EH         LINE#         175
  C:4B63H         LINE#         176
  C:4B65H         LINE#         177
  C:4B65H         LINE#         178
  -------         ENDPROC       LOWPOWERCHECK
  -------         PROC          LOWPOWERPROCESS
  C:6053H         LINE#         187
  C:6053H         LINE#         188
  C:6053H         LINE#         189
  C:6059H         LINE#         190
  C:6059H         LINE#         191
  C:605BH         LINE#         192
  C:6073H         LINE#         193
  C:6073H         LINE#         194
  C:6075H         LINE#         195
  C:6078H         LINE#         196
  C:6078H         LINE#         197
  C:607AH         LINE#         198
  C:607CH         LINE#         199
  C:607FH         LINE#         200
  C:607FH         LINE#         201
  C:6082H         LINE#         202
  C:6084H         LINE#         203
  C:6087H         LINE#         204
  C:6087H         LINE#         205
  C:608AH         LINE#         206
  C:608AH         LINE#         208
  C:608DH         LINE#         209
  -------         ENDPROC       LOWPOWERPROCESS
  -------         ENDMOD        LOWPOWER
BL51 BANKED LINKER/LOCATER V6.22                                                      06/21/2022  07:40:42  PAGE 28



  -------         MODULE        UARTAPP
  C:0000H         SYMBOL        _ICE_DUMMY_
  C:65F2H         PUBLIC        UartCheck
  D:0080H         PUBLIC        P0
  D:0090H         PUBLIC        P1
  D:00A0H         PUBLIC        P2
  C:3CE4H         PUBLIC        UartCaliCurrent
  D:00B0H         PUBLIC        P3
  D:00C0H         PUBLIC        P4
  C:56F7H         PUBLIC        UartCaliRTC
  D:0080H         PUBLIC        P5
  X:037FH         PUBLIC        ucUartSndLength
  C:3075H         PUBLIC        IapCheckHandshake
  X:0380H         PUBLIC        ucUartTimeoutCnt
  X:0381H         PUBLIC        ucSubClassID
  C:5D38H         PUBLIC        WriteManufacture
  X:0A00H         PUBLIC        ucUartBuf
  B:002BH.1       PUBLIC        bUartReadFlg
  X:0382H         PUBLIC        ucUartErrCode
  B:002BH.2       PUBLIC        bUartWriteFlg
  C:4E72H         PUBLIC        _UartReadInfo
  C:6738H         PUBLIC        UartHandshake
  C:5B8AH         PUBLIC        Page1WrRdFuncTable
  C:5BAEH         PUBLIC        Page2WrRdFuncTable
  D:0099H         PUBLIC        SBUF
  C:61ACH         PUBLIC        UartCaliCurOffset
  C:6175H         PUBLIC        ReadSubClassID
  D:00B1H         PUBLIC        RSTSTAT
  C:4B66H         PUBLIC        _UartWriteInfo
  X:0383H         PUBLIC        ucUartBufPT
  C:31DCH         PUBLIC        UartRdCmdProcess
  B:002BH.3       PUBLIC        bUartSndAckFlg
  C:4806H         PUBLIC        _InterruptUartAppRx
  C:4580H         PUBLIC        UartWrCmdProcess
  C:44D5H         PUBLIC        InterruptUartAppTx
  B:0098H.4       PUBLIC        REN
  B:002BH.4       PUBLIC        bISPFlg
  D:009AH         PUBLIC        SADDR
  C:574BH         PUBLIC        UartCaliVoltage
  C:5AF8H         PUBLIC        UartCaliTS1
  C:5B41H         PUBLIC        UartCaliTS2
  X:0384H         PUBLIC        uiReceCheckSum
  -------         PROC          UARTHANDSHAKE
  C:6738H         LINE#         90
  C:6738H         LINE#         91
  C:6738H         LINE#         92
  C:673EH         LINE#         93
  C:673EH         LINE#         94
  C:6743H         LINE#         95
  C:6744H         LINE#         97
  C:6744H         LINE#         98
  C:6749H         LINE#         99
  C:6749H         LINE#         100
  -------         ENDPROC       UARTHANDSHAKE
  -------         PROC          _UARTWRITEINFO
  X:02B7H         SYMBOL        ptr
BL51 BANKED LINKER/LOCATER V6.22                                                      06/21/2022  07:40:42  PAGE 29


  -------         DO            
  D:0007H         SYMBOL        i
  -------         ENDDO         
  C:4B66H         LINE#         109
  C:4B6EH         LINE#         110
  C:4B6EH         LINE#         113
  C:4B8FH         LINE#         114
  C:4B8FH         LINE#         115
  C:4B9AH         LINE#         116
  C:4B9AH         LINE#         117
  C:4B9DH         LINE#         118
  C:4BB6H         LINE#         119
  C:4BC0H         LINE#         120
  C:4BC3H         LINE#         122
  C:4BC8H         LINE#         123
  C:4BCAH         LINE#         124
  C:4BCCH         LINE#         125
  C:4BCEH         LINE#         126
  C:4BD0H         LINE#         127
  C:4BD2H         LINE#         129
  C:4BD6H         LINE#         130
  C:4BD8H         LINE#         131
  C:4BDAH         LINE#         133
  C:4BDCH         LINE#         134
  C:4BE0H         LINE#         136
  C:4BE5H         LINE#         137
  C:4BE6H         LINE#         139
  C:4BE6H         LINE#         140
  C:4BEBH         LINE#         141
  C:4BEBH         LINE#         142
  -------         ENDPROC       _UARTWRITEINFO
  -------         PROC          _UARTREADINFO
  D:0006H         SYMBOL        ptr
  -------         DO            
  D:0005H         SYMBOL        i
  -------         ENDDO         
  C:4E72H         LINE#         151
  C:4E72H         LINE#         152
  C:4E72H         LINE#         155
  C:4E7BH         LINE#         156
  C:4E7BH         LINE#         157
  C:4E7DH         LINE#         158
  C:4E7DH         LINE#         160
  C:4E82H         LINE#         161
  C:4E84H         LINE#         162
  C:4E86H         LINE#         163
  C:4E88H         LINE#         164
  C:4E8AH         LINE#         165
  C:4E8CH         LINE#         167
  C:4E90H         LINE#         168
  C:4E92H         LINE#         169
  C:4E94H         LINE#         171
  C:4E9FH         LINE#         172
  C:4E9FH         LINE#         173
  C:4EA2H         LINE#         174
  C:4EB4H         LINE#         175
  C:4EB9H         LINE#         176
BL51 BANKED LINKER/LOCATER V6.22                                                      06/21/2022  07:40:42  PAGE 30


  C:4EBCH         LINE#         177
  C:4ED8H         LINE#         179
  C:4EEAH         LINE#         180
  -------         ENDPROC       _UARTREADINFO
  -------         PROC          WRITEMANUFACTURE
  C:5D38H         LINE#         191
  C:5D38H         LINE#         192
  C:5D38H         LINE#         193
  C:5D59H         LINE#         194
  C:5D59H         LINE#         195
  C:5D61H         LINE#         196
  C:5D61H         LINE#         197
  C:5D67H         LINE#         198
  C:5D69H         LINE#         199
  C:5D6DH         LINE#         200
  C:5D6DH         LINE#         201
  C:5D6FH         LINE#         202
  C:5D6FH         LINE#         203
  C:5D71H         LINE#         204
  C:5D76H         LINE#         205
  C:5D77H         LINE#         207
  C:5D77H         LINE#         208
  C:5D7CH         LINE#         209
  C:5D7CH         LINE#         210
  -------         ENDPROC       WRITEMANUFACTURE
  -------         PROC          READSUBCLASSID
  C:6175H         LINE#         219
  C:6175H         LINE#         220
  C:6175H         LINE#         221
  C:6196H         LINE#         222
  C:6196H         LINE#         223
  C:619EH         LINE#         225
  C:61A0H         LINE#         226
  C:61A5H         LINE#         227
  C:61A6H         LINE#         229
  C:61A6H         LINE#         230
  C:61ABH         LINE#         231
  C:61ABH         LINE#         232
  -------         ENDPROC       READSUBCLASSID
  -------         PROC          UARTRDCMDPROCESS
  -------         DO            
  X:02B5H         SYMBOL        rdaddr
  -------         ENDDO         
  C:31DCH         LINE#         241
  C:31DCH         LINE#         242
  C:31DCH         LINE#         245
  C:3230H         LINE#         246
  C:3230H         LINE#         247
  C:3230H         LINE#         248
  C:3230H         LINE#         249
  C:3230H         LINE#         250
  C:3230H         LINE#         251
  C:3230H         LINE#         252
  C:3230H         LINE#         253
  C:3230H         LINE#         254
  C:3230H         LINE#         255
  C:3230H         LINE#         256
BL51 BANKED LINKER/LOCATER V6.22                                                      06/21/2022  07:40:42  PAGE 31


  C:3230H         LINE#         257
  C:3240H         LINE#         258
  C:3241H         LINE#         260
  C:3241H         LINE#         261
  C:3248H         LINE#         262
  C:3249H         LINE#         264
  C:3249H         LINE#         265
  C:3250H         LINE#         266
  C:3251H         LINE#         268
  C:3251H         LINE#         269
  C:3258H         LINE#         270
  C:3259H         LINE#         272
  C:3259H         LINE#         273
  C:3260H         LINE#         274
  C:3261H         LINE#         276
  C:3261H         LINE#         277
  C:3268H         LINE#         278
  C:3269H         LINE#         280
  C:3269H         LINE#         281
  C:3270H         LINE#         282
  C:3271H         LINE#         284
  C:3271H         LINE#         285
  C:3278H         LINE#         286
  C:3279H         LINE#         288
  C:3279H         LINE#         289
  C:3280H         LINE#         290
  C:3281H         LINE#         292
  C:3281H         LINE#         293
  C:3288H         LINE#         294
  C:3289H         LINE#         296
  C:3289H         LINE#         297
  C:3290H         LINE#         298
  C:3291H         LINE#         300
  C:3291H         LINE#         301
  C:3298H         LINE#         302
  C:3299H         LINE#         304
  C:3299H         LINE#         305
  C:32A0H         LINE#         306
  C:32A1H         LINE#         308
  C:32A1H         LINE#         309
  C:32A8H         LINE#         310
  C:32A9H         LINE#         312
  C:32A9H         LINE#         313
  C:32B0H         LINE#         314
  C:32B1H         LINE#         316
  C:32B1H         LINE#         317
  C:32BAH         LINE#         318
  C:32BAH         LINE#         319
  C:32BCH         LINE#         320
  C:32BEH         LINE#         321
  C:32BFH         LINE#         322
  C:32CDH         LINE#         323
  C:32CDH         LINE#         324
  C:32CFH         LINE#         325
  C:32D1H         LINE#         326
  C:32D2H         LINE#         327
  C:32D9H         LINE#         328
BL51 BANKED LINKER/LOCATER V6.22                                                      06/21/2022  07:40:42  PAGE 32


  C:32D9H         LINE#         329
  C:32F7H         LINE#         330
  C:32FAH         LINE#         331
  C:32FBH         LINE#         332
  C:3302H         LINE#         333
  C:3302H         LINE#         334
  C:3320H         LINE#         335
  C:3323H         LINE#         336
  C:3323H         LINE#         337
  C:3323H         LINE#         338
  C:3323H         LINE#         339
  -------         ENDPROC       UARTRDCMDPROCESS
  -------         PROC          UARTCALIVOLTAGE
  C:574BH         LINE#         348
  C:574BH         LINE#         349
  C:574BH         LINE#         350
  C:576CH         LINE#         351
  C:576CH         LINE#         352
  C:577FH         LINE#         354
  C:5782H         LINE#         355
  C:5782H         LINE#         356
  C:5787H         LINE#         357
  C:5788H         LINE#         359
  C:5788H         LINE#         360
  C:578AH         LINE#         361
  C:5791H         LINE#         362
  C:5796H         LINE#         363
  C:5796H         LINE#         364
  C:5797H         LINE#         366
  C:5797H         LINE#         367
  C:579CH         LINE#         368
  C:579CH         LINE#         369
  -------         ENDPROC       UARTCALIVOLTAGE
  -------         PROC          UARTCALICURRENT
  C:3CE4H         LINE#         378
  C:3CE4H         LINE#         379
  C:3CE4H         LINE#         380
  C:3D08H         LINE#         381
  C:3D08H         LINE#         385
  C:3D70H         LINE#         387
  C:3D86H         LINE#         388
  C:3D86H         LINE#         389
  C:3D8BH         LINE#         390
  C:3D8CH         LINE#         392
  C:3D8CH         LINE#         393
  C:3D8EH         LINE#         394
  C:3D95H         LINE#         395
  C:3D9AH         LINE#         396
  C:3D9AH         LINE#         397
  C:3D9BH         LINE#         399
  C:3D9BH         LINE#         400
  C:3DA0H         LINE#         401
  C:3DA0H         LINE#         402
  -------         ENDPROC       UARTCALICURRENT
  -------         PROC          UARTCALICUROFFSET
  C:61ACH         LINE#         405
  C:61ACH         LINE#         406
BL51 BANKED LINKER/LOCATER V6.22                                                      06/21/2022  07:40:42  PAGE 33


  C:61ACH         LINE#         407
  C:61CDH         LINE#         408
  C:61CDH         LINE#         409
  C:61CFH         LINE#         410
  C:61D6H         LINE#         412
  C:61DBH         LINE#         413
  C:61DCH         LINE#         415
  C:61DCH         LINE#         416
  C:61E1H         LINE#         417
  C:61E1H         LINE#         418
  -------         ENDPROC       UARTCALICUROFFSET
  -------         PROC          UARTCALITS1
  C:5AF8H         LINE#         427
  C:5AF8H         LINE#         428
  C:5AF8H         LINE#         429
  C:5B19H         LINE#         430
  C:5B19H         LINE#         431
  C:5B1BH         LINE#         432
  C:5B2EH         LINE#         433
  C:5B35H         LINE#         435
  C:5B3AH         LINE#         436
  C:5B3BH         LINE#         438
  C:5B3BH         LINE#         439
  C:5B40H         LINE#         440
  C:5B40H         LINE#         441
  -------         ENDPROC       UARTCALITS1
  -------         PROC          UARTCALITS2
  C:5B41H         LINE#         444
  C:5B41H         LINE#         445
  C:5B41H         LINE#         446
  C:5B62H         LINE#         447
  C:5B62H         LINE#         448
  C:5B64H         LINE#         449
  C:5B77H         LINE#         450
  C:5B7EH         LINE#         452
  C:5B83H         LINE#         453
  C:5B84H         LINE#         455
  C:5B84H         LINE#         456
  C:5B89H         LINE#         457
  C:5B89H         LINE#         458
  -------         ENDPROC       UARTCALITS2
  -------         PROC          UARTCALIRTC
  -------         DO            
  D:0007H         SYMBOL        i
  -------         ENDDO         
  C:56F7H         LINE#         467
  C:56F7H         LINE#         468
  C:56F7H         LINE#         471
  C:5718H         LINE#         472
  C:5718H         LINE#         473
  C:5719H         LINE#         474
  C:5719H         LINE#         475
  C:5731H         LINE#         476
  C:5736H         LINE#         477
  C:5738H         LINE#         478
  C:573FH         LINE#         479
  C:5744H         LINE#         480
BL51 BANKED LINKER/LOCATER V6.22                                                      06/21/2022  07:40:42  PAGE 34


  C:5745H         LINE#         482
  C:5745H         LINE#         483
  C:574AH         LINE#         484
  C:574AH         LINE#         485
  -------         ENDPROC       UARTCALIRTC
  -------         PROC          UARTWRCMDPROCESS
  -------         DO            
  X:02B5H         SYMBOL        rdaddr
  -------         ENDDO         
  C:4580H         LINE#         494
  C:4580H         LINE#         495
  C:4580H         LINE#         497
  C:45ACH         LINE#         498
  C:45ACH         LINE#         499
  C:45ACH         LINE#         500
  C:45AFH         LINE#         501
  C:45B0H         LINE#         502
  C:45B0H         LINE#         503
  C:45B3H         LINE#         504
  C:45B4H         LINE#         505
  C:45B4H         LINE#         506
  C:45B7H         LINE#         507
  C:45B8H         LINE#         508
  C:45B8H         LINE#         509
  C:45BBH         LINE#         510
  C:45BCH         LINE#         511
  C:45BCH         LINE#         512
  C:45BFH         LINE#         513
  C:45C0H         LINE#         514
  C:45C0H         LINE#         515
  C:45C3H         LINE#         516
  C:45C4H         LINE#         517
  C:45C4H         LINE#         518
  C:45C7H         LINE#         519
  C:45C8H         LINE#         521
  C:45C8H         LINE#         522
  C:45CBH         LINE#         523
  C:45CCH         LINE#         524
  C:45CCH         LINE#         525
  C:45EAH         LINE#         526
  C:45EDH         LINE#         527
  C:45EEH         LINE#         528
  C:45EEH         LINE#         529
  C:460CH         LINE#         530
  C:460FH         LINE#         531
  C:4610H         LINE#         533
  C:4610H         LINE#         534
  C:4617H         LINE#         535
  C:4617H         LINE#         536
  C:4619H         LINE#         537
  C:461BH         LINE#         538
  C:4620H         LINE#         539
  C:4621H         LINE#         541
  C:4621H         LINE#         542
  C:4626H         LINE#         543
  C:4626H         LINE#         544
  C:4626H         LINE#         545
BL51 BANKED LINKER/LOCATER V6.22                                                      06/21/2022  07:40:42  PAGE 35


  C:4626H         LINE#         546
  -------         ENDPROC       UARTWRCMDPROCESS
  -------         PROC          IAPCHECKHANDSHAKE
  -------         DO            
  D:0007H         SYMBOL        i
  D:0007H         SYMBOL        databak
  X:02B5H         SYMBOL        checksum
  -------         ENDDO         
  C:3075H         LINE#         555
  C:3075H         LINE#         556
  C:3075H         LINE#         558
  C:307CH         LINE#         560
  C:3084H         LINE#         561
  C:3084H         LINE#         562
  C:308CH         LINE#         563
  C:308CH         LINE#         564
  C:3091H         LINE#         565
  C:3092H         LINE#         567
  C:3092H         LINE#         568
  C:3099H         LINE#         569
  C:309DH         LINE#         570
  C:309DH         LINE#         571
  C:309EH         LINE#         573
  C:309EH         LINE#         574
  C:30B9H         LINE#         575
  C:30B9H         LINE#         576
  C:30CCH         LINE#         577
  C:30CCH         LINE#         578
  C:30E4H         LINE#         579
  C:30E4H         LINE#         580
  C:30ECH         LINE#         581
  C:30ECH         LINE#         582
  C:30F7H         LINE#         583
  C:30F7H         LINE#         584
  C:30FCH         LINE#         585
  C:30FCH         LINE#         586
  C:30FDH         LINE#         587
  C:3105H         LINE#         588
  C:3105H         LINE#         589
  C:3110H         LINE#         590
  C:3110H         LINE#         591
  C:3117H         LINE#         592
  C:3117H         LINE#         593
  C:3117H         LINE#         594
  C:3118H         LINE#         596
  C:3118H         LINE#         597
  C:311DH         LINE#         598
  C:314CH         LINE#         599
  C:314CH         LINE#         600
  C:3153H         LINE#         601
  C:3153H         LINE#         603
  C:315AH         LINE#         604
  C:315AH         LINE#         605
  C:315EH         LINE#         606
  C:3160H         LINE#         608
  C:3160H         LINE#         609
  C:3162H         LINE#         610
BL51 BANKED LINKER/LOCATER V6.22                                                      06/21/2022  07:40:42  PAGE 36


  C:3167H         LINE#         611
  C:3167H         LINE#         613
  C:316CH         LINE#         614
  C:3172H         LINE#         616
  C:3177H         LINE#         617
  C:317DH         LINE#         618
  C:3180H         LINE#         620
  C:3199H         LINE#         621
  C:3199H         LINE#         622
  C:31AEH         LINE#         623
  C:31B1H         LINE#         625
  C:31C5H         LINE#         626
  C:31D6H         LINE#         628
  C:31DBH         LINE#         629
  C:31DBH         LINE#         630
  C:31DBH         LINE#         631
  -------         ENDPROC       IAPCHECKHANDSHAKE
  -------         PROC          _INTERRUPTUARTAPPRX
  D:0007H         SYMBOL        RxData
  C:4806H         LINE#         645
  C:4806H         LINE#         646
  C:4806H         LINE#         647
  C:4815H         LINE#         648
  C:481BH         LINE#         649
  C:4821H         LINE#         650
  C:4821H         LINE#         651
  C:4823H         LINE#         652
  C:4823H         LINE#         653
  C:482BH         LINE#         654
  C:482BH         LINE#         655
  C:4835H         LINE#         656
  C:4835H         LINE#         657
  C:4839H         LINE#         658
  C:4839H         LINE#         659
  C:483BH         LINE#         660
  C:483DH         LINE#         661
  C:483FH         LINE#         663
  C:483FH         LINE#         664
  C:4841H         LINE#         665
  C:4843H         LINE#         666
  C:4843H         LINE#         667
  C:4845H         LINE#         668
  C:484DH         LINE#         669
  C:484DH         LINE#         670
  C:4852H         LINE#         671
  C:4852H         LINE#         672
  C:4852H         LINE#         674
  C:4855H         LINE#         675
  C:4855H         LINE#         676
  C:485DH         LINE#         677
  C:485DH         LINE#         678
  C:4860H         LINE#         679
  C:4860H         LINE#         680
  C:4862H         LINE#         681
  C:4865H         LINE#         682
  C:4865H         LINE#         683
  C:487EH         LINE#         684
BL51 BANKED LINKER/LOCATER V6.22                                                      06/21/2022  07:40:42  PAGE 37


  C:487EH         LINE#         685
  C:4881H         LINE#         686
  C:4883H         LINE#         687
  C:4888H         LINE#         688
  C:4888H         LINE#         689
  C:488AH         LINE#         691
  C:488AH         LINE#         692
  C:488DH         LINE#         693
  C:488DH         LINE#         694
  C:488FH         LINE#         696
  C:4894H         LINE#         697
  C:4898H         LINE#         698
  C:489CH         LINE#         699
  -------         ENDPROC       _INTERRUPTUARTAPPRX
  -------         PROC          INTERRUPTUARTAPPTX
  C:44D5H         LINE#         708
  C:44D5H         LINE#         709
  C:44D5H         LINE#         710
  C:44E5H         LINE#         711
  C:44E5H         LINE#         712
  C:44FEH         LINE#         713
  C:44FEH         LINE#         714
  C:4500H         LINE#         715
  C:4502H         LINE#         716
  C:4504H         LINE#         717
  C:4508H         LINE#         718
  C:450AH         LINE#         719
  C:450CH         LINE#         720
  C:450EH         LINE#         721
  C:4510H         LINE#         722
  C:4512H         LINE#         724
  C:4512H         LINE#         725
  C:4518H         LINE#         726
  C:4527H         LINE#         727
  C:4527H         LINE#         728
  C:4529H         LINE#         729
  C:4546H         LINE#         730
  C:4546H         LINE#         731
  C:4548H         LINE#         732
  C:454DH         LINE#         733
  C:454FH         LINE#         734
  C:4553H         LINE#         735
  C:4555H         LINE#         736
  C:4557H         LINE#         737
  C:4559H         LINE#         738
  C:455BH         LINE#         739
  C:455DH         LINE#         741
  C:455DH         LINE#         742
  C:4563H         LINE#         743
  C:4572H         LINE#         744
  C:4572H         LINE#         746
  C:4577H         LINE#         747
  C:457BH         LINE#         748
  C:457FH         LINE#         749
  -------         ENDPROC       INTERRUPTUARTAPPTX
  -------         PROC          UARTCHECK
  C:65F2H         LINE#         758
BL51 BANKED LINKER/LOCATER V6.22                                                      06/21/2022  07:40:42  PAGE 38


  C:65F2H         LINE#         759
  C:65F2H         LINE#         760
  C:65FDH         LINE#         761
  C:65FDH         LINE#         762
  C:65FFH         LINE#         763
  C:6603H         LINE#         764
  C:6605H         LINE#         765
  C:6605H         LINE#         766
  -------         ENDPROC       UARTCHECK
  -------         ENDMOD        UARTAPP

  -------         MODULE        MEMORY
  C:0000H         SYMBOL        _ICE_DUMMY_
  B:0020H.2       PUBLIC        bOCRC_EN
  X:00B3H         PUBLIC        E2uiLearnLowTempe
  D:0080H         PUBLIC        P0
  D:0022H         PUBLIC        uiBatStatus
  D:0090H         PUBLIC        P1
  X:00C2H         PUBLIC        E2ulCycleThreshold
  D:00A0H         PUBLIC        P2
  D:00B0H         PUBLIC        P3
  B:0025H.6       PUBLIC        bFastDischarge
  D:00C0H         PUBLIC        P4
  D:0080H         PUBLIC        P5
  B:0023H.0       PUBLIC        bOV
  X:002AH         PUBLIC        E2ucLowPowerDeley
  B:0023H.1       PUBLIC        bUV
  X:00C6H         PUBLIC        E2ulCycleThresholdCount
  B:0025H.5       PUBLIC        bMidDischarge
  B:0020H.6       PUBLIC        bOCPM
  B:0025H.2       PUBLIC        bCHGING
  X:006DH         PUBLIC        E2slOCCCurrent
  X:00D7H         PUBLIC        E2siTS0Offset
  X:0088H         PUBLIC        E2ucLoadRDelay
  X:00D9H         PUBLIC        E2siTS1Offset
  X:0071H         PUBLIC        E2ucOCCDelay
  X:0024H         PUBLIC        E2uiLearnLowTemp
  B:0025H.4       PUBLIC        bSlowDischarge
  B:0021H.3       PUBLIC        bLEDNum0
  B:0021H.4       PUBLIC        bLEDNum1
  X:00CEH         PUBLIC        E2uiAFEOVvol
  X:001EH         PUBLIC        E2ulCycleThreshold_Rsv
  X:002FH         PUBLIC        E2ucRamCheckFlg0
  X:00ADH         PUBLIC        E2siChgEndCurr
  X:0061H         PUBLIC        E2ucRamCheckFlg1
  B:0025H.3       PUBLIC        bDSGING
  X:0074H         PUBLIC        E2ucRamCheckFlg2
  X:008DH         PUBLIC        E2ucDSG1PWMRatioH
  X:0089H         PUBLIC        E2ucRamCheckFlg3
  X:0064H         PUBLIC        E2uiOVRvol
  X:002CH         PUBLIC        E2siChgBKCur
  X:008EH         PUBLIC        E2ucRamCheckFlg5
  X:0053H         PUBLIC        E2ucDeviceChem
  X:0099H         PUBLIC        E2ucRamCheckFlg6
  B:0022H.5       PUBLIC        bAFE_SC
  B:0025H.0       PUBLIC        bCHGMOS
  B:0020H.3       PUBLIC        bBAL_EN
BL51 BANKED LINKER/LOCATER V6.22                                                      06/21/2022  07:40:42  PAGE 39


  X:00B6H         PUBLIC        E2ulFCC
  X:00A2H         PUBLIC        E2ucRamCheckFlg7
  X:008CH         PUBLIC        E2ucDSG1PWMRatioL
  X:00AAH         PUBLIC        E2ucRamCheckFlg8
  X:00CCH         PUBLIC        E2ucRamCheckFlg9
  X:0077H         PUBLIC        E2uiUVRvol
  X:0047H         PUBLIC        E2ucDeviceName
  X:0091H         PUBLIC        E2uiTempOTCR
  X:009CH         PUBLIC        E2uiTempOTDR
  X:0026H         PUBLIC        E2uiNearFCC
  B:0021H.5       PUBLIC        bTempNum
  X:00D5H         PUBLIC        E2siCadcOffset
  X:0098H         PUBLIC        E2ucTempRDelay
  D:0026H         PUBLIC        ucAFEStatus
  X:0095H         PUBLIC        E2uiTempUTCR
  B:0020H.7       PUBLIC        bEnEEPRomBK
  X:00D1H         PUBLIC        E2uiVPackGain
  X:00D0H         PUBLIC        E2ucRamCheckFlgA
  X:00A5H         PUBLIC        E2uiBalanceVolDiff
  X:00A0H         PUBLIC        E2uiTempUTDR
  X:00DCH         PUBLIC        E2ucRamCheckFlgB
  B:0025H.1       PUBLIC        bDSGMOS
  X:01FEH         PUBLIC        E2uiCheckFlag
  X:00A3H         PUBLIC        E2uiBalanceVol
  B:0022H.4       PUBLIC        bAFE_OV
  X:00B5H         PUBLIC        E2ucSOC
  X:00ABH         PUBLIC        E2uiChgEndVol
  X:0035H         PUBLIC        E2ucMNFName
  B:0023H.2       PUBLIC        bOCC
  X:00BEH         PUBLIC        E2ulChgFCC
  D:0020H         PUBLIC        uiPackConfig
  X:0067H         PUBLIC        E2ucOVRDelay
  X:002EH         PUBLIC        E2ucRTCBKDelay
  X:0041H         PUBLIC        E2ulMNFDate
  B:0020H.5       PUBLIC        bCTO_EN
  X:00BAH         PUBLIC        E2ulLastFCC
  X:0002H         PUBLIC        E2uiVOC
  X:007AH         PUBLIC        E2ucUVRDelay
  X:00DBH         PUBLIC        E2ucCalibrated
  X:00B1H         PUBLIC        E2uiDsgEndVol
  B:0026H.4       PUBLIC        bAfeCHG
  X:00D3H         PUBLIC        E2siCadcGain
  X:001AH         PUBLIC        E2ulFCC_Rsv
  B:0026H.2       PUBLIC        bAfeChging
  X:00DDH         PUBLIC        Reserved
  X:0068H         PUBLIC        E2ucReserved0
  X:007BH         PUBLIC        E2ucReserved1
  B:0021H.0       PUBLIC        bCellNum1
  X:007EH         PUBLIC        E2slOCD1Current
  X:0073H         PUBLIC        E2ucReserved2
  B:0022H.6       PUBLIC        bCTO
  B:0022H.0       PUBLIC        bOTC
  B:0021H.1       PUBLIC        bCellNum2
  X:0083H         PUBLIC        E2slOCD2Current
  B:0022H.1       PUBLIC        bOTD
  B:0021H.2       PUBLIC        bCellNum3
  X:0082H         PUBLIC        E2ucOCD1Delay
BL51 BANKED LINKER/LOCATER V6.22                                                      06/21/2022  07:40:42  PAGE 40


  X:0087H         PUBLIC        E2ucOCD2Delay
  B:0024H.2       PUBLIC        bVDQ
  X:00A7H         PUBLIC        E2siBalCurrent
  B:0026H.5       PUBLIC        bAfeDSG
  B:0022H.2       PUBLIC        bUTC
  X:0062H         PUBLIC        E2uiOVvol
  X:0028H         PUBLIC        E2siDfilterCur
  B:0026H.3       PUBLIC        bAfeDsging
  B:0022H.3       PUBLIC        bUTD
  X:0000H         PUBLIC        E2uiPackConfigMap
  X:0075H         PUBLIC        E2uiUVvol
  X:00CAH         PUBLIC        E2uiCycleCount
  X:008FH         PUBLIC        E2uiTempOTC
  X:009AH         PUBLIC        E2uiTempOTD
  B:0021H.6       PUBLIC        bChgerLock
  X:0097H         PUBLIC        E2ucTempDelay
  B:0026H.0       PUBLIC        bAfeChger
  X:0093H         PUBLIC        E2uiTempUTC
  X:009EH         PUBLIC        E2uiTempUTD
  X:0034H         PUBLIC        E2ucID
  X:00CDH         PUBLIC        E2ucAFEProtectConfig
  X:0032H         PUBLIC        E2uiHWVersion
  X:005FH         PUBLIC        E2uiChemID
  X:002BH         PUBLIC        E2ucChgBKDelay
  X:0066H         PUBLIC        E2ucOVDelay
  D:0024H         PUBLIC        uiPackStatus
  B:0023H.3       PUBLIC        bOCD1
  B:0023H.4       PUBLIC        bOCD2
  B:0024H.0       PUBLIC        bFC
  B:0020H.4       PUBLIC        bPF_EN
  X:0072H         PUBLIC        E2ucOCCRDelay
  X:0016H         PUBLIC        E2ulDesignCapacity
  B:0024H.1       PUBLIC        bFD
  B:0020H.0       PUBLIC        bSC_EN
  X:0045H         PUBLIC        E2uiSerialNum
  X:0030H         PUBLIC        E2uiSWVersion
  X:00A9H         PUBLIC        E2ucBalanceDelay
  X:008AH         PUBLIC        E2uiDSG1PWMFreq
  X:0079H         PUBLIC        E2ucUVDelay
  X:00AFH         PUBLIC        E2ucChgEndDelay
  B:0021H.7       PUBLIC        bLoadLock
  B:0026H.1       PUBLIC        bAfeLoad
  X:0022H         PUBLIC        E2uiCycleCount_Rsv
  I:00A0H         PUBLIC        STACK
  B:0020H.1       PUBLIC        bOV_EN
  X:00B0H         PUBLIC        E2ucDsgEndDelay
  -------         ENDMOD        MEMORY

  -------         MODULE        AFE
  C:0000H         SYMBOL        _ICE_DUMMY_
  X:0200H         PUBLIC        uiVadcVmax
  D:000FH         PUBLIC        uiCellVmin
  D:0080H         PUBLIC        P0
  D:0011H         PUBLIC        uiCellVmax
  D:0090H         PUBLIC        P1
  D:00A0H         PUBLIC        P2
  D:00B0H         PUBLIC        P3
BL51 BANKED LINKER/LOCATER V6.22                                                      06/21/2022  07:40:42  PAGE 41


  C:4BECH         PUBLIC        AFEInitReg
  X:0202H         PUBLIC        uiTempeMin
  D:00C0H         PUBLIC        P4
  D:0080H         PUBLIC        P5
  X:0204H         PUBLIC        uiTempeMax
  B:0029H.3       PUBLIC        bCADCFlg
  C:66B3H         PUBLIC        AfeADCEn
  C:6017H         PUBLIC        AFEClrFlg
  C:6599H         PUBLIC        AFERdStatus
  D:0013H         PUBLIC        ucCellNum
  X:0206H         PUBLIC        Info
  C:6712H         PUBLIC        AfeTempADCDis
  X:023CH         PUBLIC        slCadcCurBuf
  B:0029H.4       PUBLIC        bAfeErr
  B:0029H.5       PUBLIC        bVADCFlg
  C:6280H         PUBLIC        AFERdFlg
  C:65B1H         PUBLIC        _AfeAlarmDis
  C:66A0H         PUBLIC        AfeWDTDis
  B:0029H.6       PUBLIC        bAfeI2CRWErrFlg
  C:65C8H         PUBLIC        _AFEMosCtl
  C:66FFH         PUBLIC        AfeTempADCEn
  X:027CH         PUBLIC        ucTempeMiddle
  C:674AH         PUBLIC        _AfeAlarmEn
  C:668DH         PUBLIC        AfeWDTEn
  X:027DH         PUBLIC        slCadcCurrent
  X:0281H         PUBLIC        slCadcCurAverage
  C:66ECH         PUBLIC        AfeCADCDis
  C:6654H         PUBLIC        AFEChgerCheckDis
  C:5FD8H         PUBLIC        _AfeBalCtl
  X:0285H         PUBLIC        AFE
  C:66D9H         PUBLIC        AfeCADCEn
  C:6641H         PUBLIC        AFEChgerCheckEn
  C:5378H         PUBLIC        AFERamCheck
  C:667AH         PUBLIC        AFELoadCheckDis
  D:00C8H         PUBLIC        TWICON
  X:02A3H         PUBLIC        REG
  C:63EEH         PUBLIC        AFEEnterPD
  C:675CH         PUBLIC        AFEInit
  C:657FH         PUBLIC        AFETwiCheck
  C:6667H         PUBLIC        AFELoadCheckEn
  C:4FD9H         PUBLIC        _AFEReadReg
  X:02B1H         PUBLIC        ucAfeI2CErrDelayCnt
  X:02B2H         PUBLIC        ucCadcCnt
  C:66C6H         PUBLIC        AfeADCDis
  D:0014H         PUBLIC        ucCellNumOffset
  C:4376H         PUBLIC        _AFEWriteReg
  B:0029H.7       PUBLIC        bAfeAlarmFlg
  X:02B3H         PUBLIC        uiVadcVmin
  -------         PROC          AFETWICHECK
  C:657FH         LINE#         43
  C:657FH         LINE#         44
  C:657FH         LINE#         45
  C:6582H         LINE#         46
  C:6582H         LINE#         47
  C:658DH         LINE#         48
  C:658DH         LINE#         49
  C:658FH         LINE#         50
BL51 BANKED LINKER/LOCATER V6.22                                                      06/21/2022  07:40:42  PAGE 42


  C:6592H         LINE#         51
  C:6592H         LINE#         52
  C:6593H         LINE#         54
  C:6593H         LINE#         55
  C:6598H         LINE#         56
  C:6598H         LINE#         57
  -------         ENDPROC       AFETWICHECK
  -------         PROC          _AFEWRITEREG
  X:02BDH         SYMBOL        Reg
  X:02BEH         SYMBOL        Length
  X:02BFH         SYMBOL        WrBuf
  -------         DO            
  B:0028H.6       SYMBOL        Result
  X:02C1H         SYMBOL        Times
  X:02C2H         SYMBOL        i
  -------         ENDDO         
  C:4376H         LINE#         67
  C:4384H         LINE#         68
  C:4384H         LINE#         69
  C:4386H         LINE#         70
  C:4389H         LINE#         73
  C:438FH         LINE#         74
  C:438FH         LINE#         75
  C:43A1H         LINE#         76
  C:43A1H         LINE#         77
  C:43AEH         LINE#         78
  C:43AEH         LINE#         79
  C:43D5H         LINE#         80
  C:43D8H         LINE#         81
  C:43D8H         LINE#         82
  C:43DAH         LINE#         83
  C:43DCH         LINE#         85
  C:43DCH         LINE#         86
  C:43DFH         LINE#         87
  C:43E4H         LINE#         88
  C:43E9H         LINE#         89
  C:43EEH         LINE#         90
  C:43EEH         LINE#         91
  C:43F0H         LINE#         92
  C:43F9H         LINE#         93
  C:43F9H         LINE#         94
  C:43FBH         LINE#         95
  C:43FDH         LINE#         97
  C:43FDH         LINE#         98
  C:4402H         LINE#         99
  C:4408H         LINE#         100
  C:4412H         LINE#         101
  C:4412H         LINE#         102
  C:4417H         LINE#         103
  C:4420H         LINE#         104
  C:4420H         LINE#         105
  C:4425H         LINE#         107
  C:4427H         LINE#         108
  -------         ENDPROC       _AFEWRITEREG
  -------         PROC          _AFEREADREG
  X:02C3H         SYMBOL        Reg
  X:02C4H         SYMBOL        Length
BL51 BANKED LINKER/LOCATER V6.22                                                      06/21/2022  07:40:42  PAGE 43


  X:02C5H         SYMBOL        RdBuf
  -------         DO            
  B:0028H.6       SYMBOL        Result
  X:02C7H         SYMBOL        Times
  -------         ENDDO         
  C:4FD9H         LINE#         118
  C:4FE7H         LINE#         119
  C:4FE7H         LINE#         120
  C:4FE9H         LINE#         121
  C:4FECH         LINE#         123
  C:4FEFH         LINE#         124
  C:4FEFH         LINE#         125
  C:4FFCH         LINE#         126
  C:4FFCH         LINE#         127
  C:5025H         LINE#         128
  C:5028H         LINE#         129
  C:5028H         LINE#         130
  C:502AH         LINE#         131
  C:502CH         LINE#         133
  C:502CH         LINE#         134
  C:502FH         LINE#         135
  C:5034H         LINE#         136
  C:5039H         LINE#         137
  C:503EH         LINE#         138
  C:503EH         LINE#         139
  C:5040H         LINE#         140
  C:5040H         LINE#         141
  C:5045H         LINE#         143
  C:5047H         LINE#         144
  -------         ENDPROC       _AFEREADREG
  -------         PROC          AFECLRFLG
  C:6017H         LINE#         153
  C:6017H         LINE#         154
  C:6017H         LINE#         155
  C:6024H         LINE#         156
  C:6024H         LINE#         157
  C:602EH         LINE#         158
  C:602EH         LINE#         159
  C:6035H         LINE#         160
  C:6040H         LINE#         161
  C:6047H         LINE#         162
  C:6052H         LINE#         163
  C:6052H         LINE#         164
  C:6052H         LINE#         165
  -------         ENDPROC       AFECLRFLG
  -------         PROC          AFEINITREG
  -------         DO            
  D:0004H         SYMBOL        TempVar
  -------         ENDDO         
  C:4BECH         LINE#         174
  C:4BECH         LINE#         175
  C:4BECH         LINE#         178
  C:4BF1H         LINE#         179
  C:4BF5H         LINE#         180
  C:4BF8H         LINE#         181
  C:4BFCH         LINE#         182
  C:4BFFH         LINE#         183
BL51 BANKED LINKER/LOCATER V6.22                                                      06/21/2022  07:40:42  PAGE 44


  C:4C01H         LINE#         184
  C:4C05H         LINE#         185
  C:4C09H         LINE#         186
  C:4C0DH         LINE#         187
  C:4C11H         LINE#         188
  C:4C14H         LINE#         190
  C:4C17H         LINE#         191
  C:4C17H         LINE#         192
  C:4C1EH         LINE#         193
  C:4C30H         LINE#         194
  C:4C30H         LINE#         195
  C:4C33H         LINE#         196
  C:4C33H         LINE#         197
  C:4C3AH         LINE#         198
  C:4C4CH         LINE#         199
  C:4C69H         LINE#         200
  C:4C6EH         LINE#         201
  C:4C71H         LINE#         202
  C:4C71H         LINE#         203
  -------         ENDPROC       AFEINITREG
  -------         PROC          AFEINIT
  -------         DO            
  B:0028H.5       SYMBOL        Result
  -------         ENDDO         
  C:675CH         LINE#         213
  C:675CH         LINE#         214
  C:675CH         LINE#         229
  C:6769H         LINE#         230
  C:676BH         LINE#         231
  -------         ENDPROC       AFEINIT
  -------         PROC          AFERDFLG
  C:6280H         LINE#         242
  C:6280H         LINE#         243
  C:6280H         LINE#         244
  C:628DH         LINE#         245
  C:628DH         LINE#         246
  C:6295H         LINE#         247
  C:6295H         LINE#         248
  C:6297H         LINE#         249
  C:6297H         LINE#         251
  C:629BH         LINE#         252
  C:629BH         LINE#         253
  C:629DH         LINE#         254
  C:629DH         LINE#         256
  C:62A4H         LINE#         257
  C:62A4H         LINE#         258
  C:62A6H         LINE#         259
  C:62A8H         LINE#         260
  C:62A8H         LINE#         262
  C:62AFH         LINE#         263
  C:62AFH         LINE#         264
  C:62B2H         LINE#         265
  C:62B2H         LINE#         266
  C:62B2H         LINE#         267
  -------         ENDPROC       AFERDFLG
  -------         PROC          AFERDSTATUS
  -------         DO            
BL51 BANKED LINKER/LOCATER V6.22                                                      06/21/2022  07:40:42  PAGE 45


  X:02B9H         SYMBOL        RegTemp
  -------         ENDDO         
  C:6599H         LINE#         276
  C:6599H         LINE#         277
  C:6599H         LINE#         279
  C:65A6H         LINE#         280
  C:65A6H         LINE#         281
  C:65B0H         LINE#         282
  C:65B0H         LINE#         283
  -------         ENDPROC       AFERDSTATUS
  -------         PROC          AFERAMCHECK
  -------         DO            
  X:02B9H         SYMBOL        RdBuf
  X:02BBH         SYMBOL        i
  -------         ENDDO         
  C:5378H         LINE#         292
  C:5378H         LINE#         293
  C:5378H         LINE#         297
  C:5388H         LINE#         298
  C:5388H         LINE#         299
  C:5391H         LINE#         301
  C:53BFH         LINE#         302
  C:53BFH         LINE#         303
  C:53C7H         LINE#         304
  C:53C7H         LINE#         305
  C:53CAH         LINE#         306
  C:53CBH         LINE#         307
  C:53CBH         LINE#         308
  C:53CBH         LINE#         309
  C:53D4H         LINE#         310
  -------         ENDPROC       AFERAMCHECK
  -------         PROC          AFEENTERPD
  C:63EEH         LINE#         319
  C:63EEH         LINE#         320
  C:63EEH         LINE#         321
  C:63F4H         LINE#         322
  C:6401H         LINE#         323
  C:6401H         LINE#         324
  C:6408H         LINE#         325
  C:6413H         LINE#         326
  C:6413H         LINE#         327
  -------         ENDPROC       AFEENTERPD
  -------         PROC          _AFEMOSCTL
  D:0007H         SYMBOL        MosStatus
  C:65C8H         LINE#         336
  C:65C8H         LINE#         337
  C:65C8H         LINE#         338
  C:65CFH         LINE#         339
  C:65D1H         LINE#         340
  C:65DCH         LINE#         341
  -------         ENDPROC       _AFEMOSCTL
  -------         PROC          AFECHGERCHECKEN
  C:6641H         LINE#         351
  C:6641H         LINE#         352
  C:6641H         LINE#         353
  C:6648H         LINE#         354
  C:6653H         LINE#         355
BL51 BANKED LINKER/LOCATER V6.22                                                      06/21/2022  07:40:42  PAGE 46


  -------         ENDPROC       AFECHGERCHECKEN
  -------         PROC          AFECHGERCHECKDIS
  C:6654H         LINE#         358
  C:6654H         LINE#         359
  C:6654H         LINE#         360
  C:665BH         LINE#         361
  C:6666H         LINE#         362
  -------         ENDPROC       AFECHGERCHECKDIS
  -------         PROC          AFELOADCHECKEN
  C:6667H         LINE#         365
  C:6667H         LINE#         366
  C:6667H         LINE#         367
  C:666EH         LINE#         368
  C:6679H         LINE#         369
  -------         ENDPROC       AFELOADCHECKEN
  -------         PROC          AFELOADCHECKDIS
  C:667AH         LINE#         372
  C:667AH         LINE#         373
  C:667AH         LINE#         374
  C:6681H         LINE#         375
  C:668CH         LINE#         376
  -------         ENDPROC       AFELOADCHECKDIS
  -------         PROC          _AFEBALCTL
  X:02BBH         SYMBOL        BalChTemp
  C:5FD8H         LINE#         385
  C:5FE0H         LINE#         386
  C:5FE0H         LINE#         387
  C:5FF4H         LINE#         388
  C:6001H         LINE#         389
  C:6001H         LINE#         390
  C:600BH         LINE#         391
  C:6016H         LINE#         392
  C:6016H         LINE#         393
  -------         ENDPROC       _AFEBALCTL
  -------         PROC          AFEWDTEN
  C:668DH         LINE#         402
  C:668DH         LINE#         403
  C:668DH         LINE#         404
  C:6694H         LINE#         405
  C:669FH         LINE#         406
  -------         ENDPROC       AFEWDTEN
  -------         PROC          AFEWDTDIS
  C:66A0H         LINE#         409
  C:66A0H         LINE#         410
  C:66A0H         LINE#         411
  C:66A7H         LINE#         412
  C:66B2H         LINE#         413
  -------         ENDPROC       AFEWDTDIS
  -------         PROC          AFEADCEN
  C:66B3H         LINE#         422
  C:66B3H         LINE#         423
  C:66B3H         LINE#         424
  C:66BAH         LINE#         425
  C:66C5H         LINE#         426
  -------         ENDPROC       AFEADCEN
  -------         PROC          AFEADCDIS
  C:66C6H         LINE#         429
BL51 BANKED LINKER/LOCATER V6.22                                                      06/21/2022  07:40:42  PAGE 47


  C:66C6H         LINE#         430
  C:66C6H         LINE#         431
  C:66CDH         LINE#         432
  C:66D8H         LINE#         433
  -------         ENDPROC       AFEADCDIS
  -------         PROC          AFECADCEN
  C:66D9H         LINE#         435
  C:66D9H         LINE#         436
  C:66D9H         LINE#         437
  C:66E0H         LINE#         438
  C:66EBH         LINE#         439
  -------         ENDPROC       AFECADCEN
  -------         PROC          AFECADCDIS
  C:66ECH         LINE#         442
  C:66ECH         LINE#         443
  C:66ECH         LINE#         444
  C:66F3H         LINE#         445
  C:66FEH         LINE#         446
  -------         ENDPROC       AFECADCDIS
  -------         PROC          AFETEMPADCEN
  C:66FFH         LINE#         448
  C:66FFH         LINE#         449
  C:66FFH         LINE#         450
  C:6706H         LINE#         451
  C:6711H         LINE#         452
  -------         ENDPROC       AFETEMPADCEN
  -------         PROC          AFETEMPADCDIS
  C:6712H         LINE#         455
  C:6712H         LINE#         456
  C:6712H         LINE#         457
  C:6719H         LINE#         458
  C:6724H         LINE#         459
  -------         ENDPROC       AFETEMPADCDIS
  -------         PROC          _AFEALARMEN
  D:0007H         SYMBOL        AlarmFlg
  C:674AH         LINE#         468
  C:674AH         LINE#         469
  C:674AH         LINE#         470
  C:6750H         LINE#         471
  C:675BH         LINE#         472
  -------         ENDPROC       _AFEALARMEN
  -------         PROC          _AFEALARMDIS
  D:0007H         SYMBOL        AlarmFlg
  C:65B1H         LINE#         474
  C:65B1H         LINE#         475
  C:65B1H         LINE#         476
  C:65BCH         LINE#         477
  C:65C7H         LINE#         478
  -------         ENDPROC       _AFEALARMDIS
  -------         ENDMOD        AFE

  -------         MODULE        BALANCE
  C:0000H         SYMBOL        _ICE_DUMMY_
  D:0080H         PUBLIC        P0
  D:0090H         PUBLIC        P1
  D:00A0H         PUBLIC        P2
  B:002AH.0       PUBLIC        bBalancingFlg
BL51 BANKED LINKER/LOCATER V6.22                                                      06/21/2022  07:40:42  PAGE 48


  D:00B0H         PUBLIC        P3
  D:00C0H         PUBLIC        P4
  B:002AH.1       PUBLIC        bCellOpenDecFlag
  D:0080H         PUBLIC        P5
  C:6794H         PUBLIC        BalanceProcess
  X:0386H         PUBLIC        ucBalanceStep
  X:0387H         PUBLIC        ucCellOpenDecCnt
  X:0388H         PUBLIC        ucCtoCnt
  B:002AH.2       PUBLIC        bBalanceFlg
  C:6414H         PUBLIC        CTOTurnOnCheck
  X:0389H         PUBLIC        ucBalanceTimeCnt
  B:002AH.3       PUBLIC        bBalanceOddFlg
  X:038AH         PUBLIC        uiBalanceChannel
  B:002AH.4       PUBLIC        bCTOValidFlg
  C:346BH         PUBLIC        BalTurnOnCheck
  C:4209H         PUBLIC        BalProcess
  C:61E2H         PUBLIC        CTOCheckVol
  -------         PROC          BALTURNONCHECK
  -------         DO            
  D:0005H         SYMBOL        i
  -------         ENDDO         
  C:346BH         LINE#         32
  C:346BH         LINE#         33
  C:346BH         LINE#         36
  C:3477H         LINE#         37
  C:3477H         LINE#         38
  C:347DH         LINE#         39
  C:347DH         LINE#         40
  C:3484H         LINE#         41
  C:34B4H         LINE#         44
  C:34B4H         LINE#         45
  C:34B6H         LINE#         46
  C:34BBH         LINE#         47
  C:34BCH         LINE#         49
  C:34BCH         LINE#         50
  C:3506H         LINE#         51
  C:3506H         LINE#         52
  C:3509H         LINE#         53
  C:3509H         LINE#         54
  C:350FH         LINE#         55
  C:350FH         LINE#         56
  C:352BH         LINE#         57
  C:352BH         LINE#         58
  C:3541H         LINE#         59
  C:3541H         LINE#         60
  C:3586H         LINE#         61
  C:3586H         LINE#         62
  C:35A1H         LINE#         63
  C:35A1H         LINE#         64
  C:35A4H         LINE#         65
  C:35A6H         LINE#         66
  C:35A6H         LINE#         67
  C:35A7H         LINE#         69
  C:35A7H         LINE#         70
  C:35A9H         LINE#         71
  C:35AEH         LINE#         72
  C:35AEH         LINE#         73
BL51 BANKED LINKER/LOCATER V6.22                                                      06/21/2022  07:40:42  PAGE 49


  C:35AEH         LINE#         74
  C:35AEH         LINE#         75
  C:35AEH         LINE#         76
  -------         ENDPROC       BALTURNONCHECK
  -------         PROC          CTOCHECKVOL
  -------         DO            
  B:0028H.5       SYMBOL        bResult
  -------         ENDDO         
  C:61E2H         LINE#         87
  C:61E2H         LINE#         88
  C:61E2H         LINE#         89
  C:61E4H         LINE#         91
  C:61E7H         LINE#         92
  C:61E7H         LINE#         93
  C:61EAH         LINE#         94
  C:61EAH         LINE#         95
  C:61EDH         LINE#         96
  C:61EDH         LINE#         97
  C:61FCH         LINE#         98
  C:61FCH         LINE#         99
  C:61FEH         LINE#         100
  C:6209H         LINE#         101
  C:6209H         LINE#         102
  C:620BH         LINE#         103
  C:620BH         LINE#         104
  C:620DH         LINE#         106
  C:620DH         LINE#         107
  C:620FH         LINE#         108
  C:6214H         LINE#         109
  C:6214H         LINE#         110
  C:6214H         LINE#         111
  C:6214H         LINE#         128
  C:6214H         LINE#         130
  C:6216H         LINE#         131
  -------         ENDPROC       CTOCHECKVOL
  -------         PROC          BALPROCESS
  -------         DO            
  X:02B9H         SYMBOL        BalChTemp
  -------         ENDDO         
  C:4209H         LINE#         144
  C:4209H         LINE#         145
  C:4209H         LINE#         150
  C:4227H         LINE#         151
  C:4227H         LINE#         152
  C:4229H         LINE#         153
  C:4229H         LINE#         155
  C:4241H         LINE#         156
  C:4241H         LINE#         157
  C:4241H         LINE#         158
  C:4247H         LINE#         159
  C:4247H         LINE#         160
  C:424AH         LINE#         161
  C:424AH         LINE#         162
  C:425DH         LINE#         163
  C:425FH         LINE#         165
  C:425FH         LINE#         166
  C:4272H         LINE#         167
BL51 BANKED LINKER/LOCATER V6.22                                                      06/21/2022  07:40:42  PAGE 50


  C:4272H         LINE#         168
  C:427DH         LINE#         169
  C:4283H         LINE#         170
  C:4285H         LINE#         171
  C:4285H         LINE#         172
  C:4286H         LINE#         174
  C:4286H         LINE#         175
  C:428CH         LINE#         176
  C:428DH         LINE#         178
  C:428DH         LINE#         179
  C:4292H         LINE#         180
  C:4292H         LINE#         181
  C:4298H         LINE#         182
  C:429EH         LINE#         183
  C:42A0H         LINE#         184
  C:42A0H         LINE#         185
  C:42A1H         LINE#         187
  C:42A1H         LINE#         188
  C:42A6H         LINE#         189
  C:42A6H         LINE#         190
  C:42ACH         LINE#         191
  C:42ADH         LINE#         193
  C:42ADH         LINE#         194
  C:42B3H         LINE#         195
  C:42B5H         LINE#         196
  C:42B5H         LINE#         197
  C:42B6H         LINE#         199
  C:42B6H         LINE#         200
  C:42BCH         LINE#         201
  C:42BEH         LINE#         202
  C:42C0H         LINE#         203
  C:42C2H         LINE#         204
  C:42C2H         LINE#         205
  C:42C2H         LINE#         206
  -------         ENDPROC       BALPROCESS
  -------         PROC          CTOTURNONCHECK
  C:6414H         LINE#         215
  C:6414H         LINE#         216
  C:6414H         LINE#         220
  C:641AH         LINE#         222
  C:641AH         LINE#         223
  C:6425H         LINE#         224
  C:6425H         LINE#         225
  C:6428H         LINE#         226
  C:642BH         LINE#         227
  C:642BH         LINE#         228
  C:642DH         LINE#         229
  C:642FH         LINE#         230
  C:6439H         LINE#         231
  C:6439H         LINE#         232
  C:6439H         LINE#         233
  C:6439H         LINE#         234
  -------         ENDPROC       CTOTURNONCHECK
  -------         PROC          BALANCEPROCESS
  C:6794H         LINE#         242
  C:6794H         LINE#         243
  C:6794H         LINE#         244
BL51 BANKED LINKER/LOCATER V6.22                                                      06/21/2022  07:40:42  PAGE 51


  C:6797H         LINE#         246
  C:679AH         LINE#         248
  C:679DH         LINE#         249
  -------         ENDPROC       BALANCEPROCESS
  -------         ENDMOD        BALANCE

  -------         MODULE        CALCULATE
  C:0000H         SYMBOL        _ICE_DUMMY_
  C:42C3H         PUBLIC        OffsetCalculate
  D:0080H         PUBLIC        P0
  D:0090H         PUBLIC        P1
  D:00A0H         PUBLIC        P2
  D:00B0H         PUBLIC        P3
  C:27C0H         PUBLIC        _CalcuTemp
  D:00C0H         PUBLIC        P4
  D:0080H         PUBLIC        P5
  C:624CH         PUBLIC        siCurTempOffset
  C:2EFDH         PUBLIC        AfeCalcuCurr
  C:382AH         PUBLIC        AfeCalcuVol
  C:5BD2H         PUBLIC        AfeGetTempe
  X:039AH         PUBLIC        ucChgingCheckCnt
  C:6606H         PUBLIC        AFEInfoProcess
  X:039BH         PUBLIC        ucDsgingCheckCnt
  B:00A8H.4       PUBLIC        ES0
  C:5A64H         PUBLIC        AfeGetVol
  C:3A62H         PUBLIC        AfeCalcuTempe
  -------         PROC          _CALCUTEMP
  D:0082H         SYMBOL        getdata
  -------         DO            
  X:02B9H         SYMBOL        i
  X:02BAH         SYMBOL        Temperature
  X:02BCH         SYMBOL        Tempcalcu
  -------         ENDDO         
  C:27C0H         LINE#         22
  C:27C4H         LINE#         23
  C:27C4H         LINE#         31
  C:27F2H         LINE#         32
  C:2804H         LINE#         33
  C:2804H         LINE#         34
  C:2821H         LINE#         35
  C:2821H         LINE#         38
  C:283AH         LINE#         39
  C:283AH         LINE#         40
  C:2844H         LINE#         41
  C:2847H         LINE#         42
  C:2860H         LINE#         43
  C:2860H         LINE#         44
  C:286AH         LINE#         45
  C:286DH         LINE#         47
  C:286DH         LINE#         48
  C:2875H         LINE#         49
  C:2894H         LINE#         50
  C:2894H         LINE#         51
  C:28A7H         LINE#         52
  C:28A7H         LINE#         53
  C:28C7H         LINE#         54
  C:28C7H         LINE#         55
BL51 BANKED LINKER/LOCATER V6.22                                                      06/21/2022  07:40:42  PAGE 52


  C:28C7H         LINE#         56
  C:28C7H         LINE#         57
  C:28CFH         LINE#         58
  C:28CFH         LINE#         60
  C:28CFH         LINE#         61
  C:28E2H         LINE#         62
  C:28E2H         LINE#         63
  C:2902H         LINE#         64
  C:2902H         LINE#         65
  C:2902H         LINE#         66
  C:2902H         LINE#         67
  C:290AH         LINE#         68
  C:2910H         LINE#         69
  C:2910H         LINE#         70
  C:2918H         LINE#         72
  C:29A7H         LINE#         73
  C:29A7H         LINE#         74
  C:29AFH         LINE#         75
  -------         ENDPROC       _CALCUTEMP
  -------         PROC          AFEGETVOL
  -------         DO            
  X:02C2H         SYMBOL        i
  B:0028H.5       SYMBOL        Result
  -------         ENDDO         
  C:5A64H         LINE#         84
  C:5A64H         LINE#         85
  C:5A64H         LINE#         87
  C:5A66H         LINE#         89
  C:5A83H         LINE#         90
  C:5A83H         LINE#         91
  C:5A9EH         LINE#         92
  C:5A9EH         LINE#         93
  C:5AA0H         LINE#         94
  C:5AA3H         LINE#         95
  C:5AA3H         LINE#         96
  C:5AABH         LINE#         98
  C:5AADH         LINE#         99
  -------         ENDPROC       AFEGETVOL
  -------         PROC          AFEGETTEMPE
  -------         DO            
  B:0028H.5       SYMBOL        Result
  -------         ENDDO         
  C:5BD2H         LINE#         101
  C:5BD2H         LINE#         102
  C:5BD2H         LINE#         103
  C:5BD4H         LINE#         105
  C:5BE1H         LINE#         106
  C:5BE1H         LINE#         107
  C:5BE3H         LINE#         108
  C:5BE3H         LINE#         109
  C:5BF0H         LINE#         110
  C:5BF0H         LINE#         111
  C:5BF2H         LINE#         112
  C:5BF2H         LINE#         114
  C:5BFFH         LINE#         115
  C:5BFFH         LINE#         116
  C:5C01H         LINE#         117
BL51 BANKED LINKER/LOCATER V6.22                                                      06/21/2022  07:40:42  PAGE 53


  C:5C01H         LINE#         118
  C:5C08H         LINE#         119
  C:5C08H         LINE#         120
  C:5C15H         LINE#         121
  C:5C15H         LINE#         122
  C:5C17H         LINE#         123
  C:5C17H         LINE#         124
  C:5C17H         LINE#         126
  C:5C19H         LINE#         127
  -------         ENDPROC       AFEGETTEMPE
  -------         PROC          AFECALCUTEMPE
  -------         DO            
  D:0006H         SYMBOL        TempeData
  -------         ENDDO         
  C:3A62H         LINE#         136
  C:3A62H         LINE#         137
  C:3A62H         LINE#         140
  C:3A6AH         LINE#         141
  C:3A6AH         LINE#         142
  C:3A81H         LINE#         143
  C:3A83H         LINE#         144
  C:3A8AH         LINE#         145
  C:3A8CH         LINE#         147
  C:3AB2H         LINE#         148
  C:3AB4H         LINE#         149
  C:3ABCH         LINE#         150
  C:3ABEH         LINE#         152
  C:3AC5H         LINE#         153
  C:3AC5H         LINE#         154
  C:3AEBH         LINE#         155
  C:3AEDH         LINE#         156
  C:3AF5H         LINE#         157
  C:3AF7H         LINE#         158
  C:3AF7H         LINE#         160
  C:3B07H         LINE#         161
  C:3B0FH         LINE#         162
  C:3B12H         LINE#         163
  C:3B12H         LINE#         164
  C:3B29H         LINE#         165
  C:3B2BH         LINE#         166
  C:3B32H         LINE#         167
  C:3B34H         LINE#         169
  C:3B41H         LINE#         170
  C:3B41H         LINE#         171
  C:3B46H         LINE#         172
  C:3B47H         LINE#         174
  C:3B47H         LINE#         175
  C:3B4FH         LINE#         176
  C:3B4FH         LINE#         177
  C:3B4FH         LINE#         178
  C:3B4FH         LINE#         179
  -------         ENDPROC       AFECALCUTEMPE
  -------         PROC          AFECALCUVOL
  -------         DO            
  X:02B9H         SYMBOL        i
  X:02BAH         SYMBOL        TempPackVol
  X:02BEH         SYMBOL        TempCellVol
BL51 BANKED LINKER/LOCATER V6.22                                                      06/21/2022  07:40:42  PAGE 54


  -------         ENDDO         
  C:382AH         LINE#         189
  C:382AH         LINE#         190
  C:382AH         LINE#         192
  C:383EH         LINE#         193
  C:3845H         LINE#         194
  C:384FH         LINE#         196
  C:3857H         LINE#         197
  C:3857H         LINE#         198
  C:3878H         LINE#         199
  C:3878H         LINE#         200
  C:38AFH         LINE#         202
  C:38C6H         LINE#         203
  C:38C6H         LINE#         204
  C:38D4H         LINE#         205
  C:38D4H         LINE#         206
  C:38EBH         LINE#         207
  C:38EBH         LINE#         208
  C:38F9H         LINE#         209
  C:38F9H         LINE#         211
  C:38FCH         LINE#         212
  C:38FCH         LINE#         213
  C:38FEH         LINE#         214
  C:3918H         LINE#         215
  C:391AH         LINE#         216
  C:392FH         LINE#         217
  C:392FH         LINE#         218
  C:3938H         LINE#         220
  C:393BH         LINE#         221
  C:393BH         LINE#         222
  C:3945H         LINE#         223
  C:394FH         LINE#         225
  C:3951H         LINE#         226
  C:395FH         LINE#         227
  C:3961H         LINE#         228
  C:3961H         LINE#         229
  C:3961H         LINE#         230
  -------         ENDPROC       AFECALCUVOL
  -------         PROC          OFFSETCALCULATE
  -------         DO            
  X:02BEH         SYMBOL        siCadcTempOffset
  X:02C0H         SYMBOL        i
  -------         ENDDO         
  C:42C3H         LINE#         251
  C:42C3H         LINE#         252
  C:42C3H         LINE#         253
  C:42CAH         LINE#         256
  C:42D9H         LINE#         257
  C:42D9H         LINE#         258
  C:4345H         LINE#         259
  C:4345H         LINE#         260
  C:4362H         LINE#         261
  C:4364H         LINE#         262
  C:4364H         LINE#         263
  C:436DH         LINE#         264
  C:4375H         LINE#         265
  -------         ENDPROC       OFFSETCALCULATE
BL51 BANKED LINKER/LOCATER V6.22                                                      06/21/2022  07:40:42  PAGE 55


  -------         PROC          AFECALCUCURR
  -------         DO            
  X:02B9H         SYMBOL        i
  X:02BAH         SYMBOL        Tempdata
  -------         ENDDO         
  C:2EFDH         LINE#         273
  C:2EFDH         LINE#         274
  C:2EFDH         LINE#         276
  C:2F07H         LINE#         278
  C:2F12H         LINE#         280
  C:2F1EH         LINE#         281
  C:2F1EH         LINE#         282
  C:2F27H         LINE#         283
  C:2F27H         LINE#         284
  C:2F76H         LINE#         286
  C:2F90H         LINE#         287
  C:2F9BH         LINE#         288
  C:2F9BH         LINE#         289
  C:2F9DH         LINE#         290
  C:2F9DH         LINE#         291
  C:2FACH         LINE#         292
  C:2FACH         LINE#         293
  C:2FCAH         LINE#         294
  C:2FD2H         LINE#         295
  C:2FE7H         LINE#         297
  C:2FE9H         LINE#         298
  C:2FEBH         LINE#         299
  C:300BH         LINE#         300
  C:300BH         LINE#         301
  C:3016H         LINE#         302
  C:3016H         LINE#         303
  C:3019H         LINE#         304
  C:301BH         LINE#         305
  C:301DH         LINE#         306
  C:3029H         LINE#         307
  C:302BH         LINE#         308
  C:302BH         LINE#         309
  C:302CH         LINE#         310
  C:3046H         LINE#         311
  C:3046H         LINE#         312
  C:3050H         LINE#         313
  C:3050H         LINE#         314
  C:3053H         LINE#         315
  C:3055H         LINE#         316
  C:3057H         LINE#         317
  C:3063H         LINE#         318
  C:3065H         LINE#         319
  C:3065H         LINE#         320
  C:3066H         LINE#         322
  C:3066H         LINE#         323
  C:3068H         LINE#         324
  C:3072H         LINE#         325
  C:3074H         LINE#         326
  C:3074H         LINE#         327
  -------         ENDPROC       AFECALCUCURR
  -------         PROC          AFEINFOPROCESS
  C:6606H         LINE#         336
BL51 BANKED LINKER/LOCATER V6.22                                                      06/21/2022  07:40:42  PAGE 56


  C:6606H         LINE#         337
  C:6606H         LINE#         338
  C:6609H         LINE#         340
  C:660BH         LINE#         341
  C:660EH         LINE#         342
  C:6611H         LINE#         344
  C:6614H         LINE#         345
  C:6614H         LINE#         346
  C:6616H         LINE#         347
  C:6619H         LINE#         348
  C:6619H         LINE#         349
  -------         ENDPROC       AFEINFOPROCESS
  -------         ENDMOD        CALCULATE

  -------         MODULE        CALIBRATE
  C:0000H         SYMBOL        _ICE_DUMMY_
  D:0080H         PUBLIC        P0
  D:0090H         PUBLIC        P1
  D:00A0H         PUBLIC        P2
  D:00B0H         PUBLIC        P3
  D:00C0H         PUBLIC        P4
  D:0080H         PUBLIC        P5
  X:0347H         PUBLIC        slExtCur
  C:676CH         PUBLIC        CaliCurZero
  X:034BH         PUBLIC        ucExtcaliSwitch1
  C:5048H         PUBLIC        CaliVoltage
  C:5D7DH         PUBLIC        CaliTS1
  C:5DC2H         PUBLIC        CaliTS2
  X:034CH         PUBLIC        uiExtTemp1
  X:034EH         PUBLIC        uiExtTemp2
  C:583FH         PUBLIC        CaliProcess
  C:608EH         PUBLIC        CaliCurrentGain
  X:0350H         PUBLIC        ulExtVPack
  X:0352H         PUBLIC        ucExtRTC
  C:5E07H         PUBLIC        CaliRTCTime
  B:002EH.3       PUBLIC        bCaliFlg
  -------         PROC          CALIVOLTAGE
  -------         DO            
  D:0007H         SYMBOL        i
  X:02B9H         SYMBOL        VPackTemp
  -------         ENDDO         
  C:5048H         LINE#         26
  C:5048H         LINE#         27
  C:5048H         LINE#         29
  C:504FH         LINE#         31
  C:5067H         LINE#         32
  C:5067H         LINE#         33
  C:5081H         LINE#         34
  C:5084H         LINE#         36
  C:50B4H         LINE#         37
  -------         ENDPROC       CALIVOLTAGE
  -------         PROC          CALICURRENTGAIN
  -------         DO            
  D:0006H         SYMBOL        TempGain
  -------         ENDDO         
  C:608EH         LINE#         46
  C:608EH         LINE#         47
BL51 BANKED LINKER/LOCATER V6.22                                                      06/21/2022  07:40:42  PAGE 57


  C:608EH         LINE#         50
  C:60BCH         LINE#         51
  C:60C0H         LINE#         52
  C:60C0H         LINE#         53
  C:60C8H         LINE#         54
  C:60C8H         LINE#         55
  -------         ENDPROC       CALICURRENTGAIN
  -------         PROC          CALICURZERO
  C:676CH         LINE#         64
  C:676CH         LINE#         65
  C:676CH         LINE#         66
  C:677BH         LINE#         67
  -------         ENDPROC       CALICURZERO
  -------         PROC          CALITS1
  -------         DO            
  D:0006H         SYMBOL        Tempe
  -------         ENDDO         
  C:5D7DH         LINE#         76
  C:5D7DH         LINE#         77
  C:5D7DH         LINE#         80
  C:5D95H         LINE#         81
  C:5DB9H         LINE#         82
  C:5DB9H         LINE#         83
  C:5DC1H         LINE#         84
  C:5DC1H         LINE#         85
  -------         ENDPROC       CALITS1
  -------         PROC          CALITS2
  -------         DO            
  D:0006H         SYMBOL        Tempe
  -------         ENDDO         
  C:5DC2H         LINE#         87
  C:5DC2H         LINE#         88
  C:5DC2H         LINE#         91
  C:5DDAH         LINE#         92
  C:5DFEH         LINE#         93
  C:5DFEH         LINE#         94
  C:5E06H         LINE#         95
  C:5E06H         LINE#         96
  -------         ENDPROC       CALITS2
  -------         PROC          CALIRTCTIME
  C:5E07H         LINE#         106
  C:5E07H         LINE#         107
  C:5E07H         LINE#         108
  C:5E0FH         LINE#         109
  C:5E17H         LINE#         110
  C:5E1FH         LINE#         111
  C:5E27H         LINE#         112
  C:5E2FH         LINE#         113
  C:5E37H         LINE#         114
  C:5E3FH         LINE#         116
  C:5E46H         LINE#         118
  C:5E48H         LINE#         119
  C:5E4AH         LINE#         120
  -------         ENDPROC       CALIRTCTIME
  -------         PROC          CALIPROCESS
  C:583FH         LINE#         131
  C:583FH         LINE#         132
BL51 BANKED LINKER/LOCATER V6.22                                                      06/21/2022  07:40:42  PAGE 58


  C:583FH         LINE#         133
  C:5842H         LINE#         134
  C:5842H         LINE#         135
  C:5844H         LINE#         137
  C:584BH         LINE#         138
  C:584BH         LINE#         139
  C:584EH         LINE#         140
  C:584EH         LINE#         142
  C:5855H         LINE#         143
  C:5855H         LINE#         144
  C:5858H         LINE#         145
  C:5858H         LINE#         147
  C:585FH         LINE#         148
  C:585FH         LINE#         149
  C:5862H         LINE#         150
  C:5862H         LINE#         152
  C:5869H         LINE#         153
  C:5869H         LINE#         154
  C:586CH         LINE#         155
  C:586CH         LINE#         157
  C:5873H         LINE#         158
  C:5873H         LINE#         159
  C:5876H         LINE#         160
  C:5876H         LINE#         162
  C:587DH         LINE#         163
  C:587DH         LINE#         164
  C:5880H         LINE#         165
  C:5880H         LINE#         167
  C:5885H         LINE#         168
  C:5887H         LINE#         169
  C:588DH         LINE#         170
  C:588DH         LINE#         171
  -------         ENDPROC       CALIPROCESS
  -------         ENDMOD        CALIBRATE

  -------         MODULE        CHARGERLOAD
  C:0000H         SYMBOL        _ICE_DUMMY_
  D:0080H         PUBLIC        P0
  D:0090H         PUBLIC        P1
  D:00A0H         PUBLIC        P2
  D:00B0H         PUBLIC        P3
  D:00C0H         PUBLIC        P4
  D:0080H         PUBLIC        P5
  X:039CH         PUBLIC        ucChgerRCnt
  B:002BH.5       PUBLIC        bChgerChkingFlg
  C:5E4BH         PUBLIC        ChgerCheck
  X:039DH         PUBLIC        ucLoadRCnt
  B:002BH.6       PUBLIC        bLoadChkingFlg
  B:002BH.7       PUBLIC        bChgerStartCheckFlg
  C:59CAH         PUBLIC        LoadCheck
  B:002CH.0       PUBLIC        bLoadStartCheckFlg
  -------         PROC          LOADCHECK
  C:59CAH         LINE#         26
  C:59CAH         LINE#         27
  C:59CAH         LINE#         28
  C:59CDH         LINE#         29
  C:59CDH         LINE#         30
BL51 BANKED LINKER/LOCATER V6.22                                                      06/21/2022  07:40:42  PAGE 59


  C:59CFH         LINE#         31
  C:59D1H         LINE#         32
  C:59D6H         LINE#         33
  C:59D9H         LINE#         34
  C:59DAH         LINE#         35
  C:59DDH         LINE#         36
  C:59DDH         LINE#         37
  C:59E0H         LINE#         38
  C:59E3H         LINE#         39
  C:59E3H         LINE#         40
  C:59FFH         LINE#         41
  C:59FFH         LINE#         42
  C:5A01H         LINE#         43
  C:5A03H         LINE#         44
  C:5A06H         LINE#         45
  C:5A09H         LINE#         46
  C:5A09H         LINE#         47
  C:5A0BH         LINE#         48
  C:5A0BH         LINE#         49
  C:5A0DH         LINE#         50
  C:5A0FH         LINE#         51
  C:5A12H         LINE#         52
  C:5A12H         LINE#         53
  C:5A14H         LINE#         54
  C:5A17H         LINE#         55
  C:5A17H         LINE#         56
  C:5A17H         LINE#         57
  C:5A17H         LINE#         58
  C:5A17H         LINE#         59
  -------         ENDPROC       LOADCHECK
  -------         PROC          CHGERCHECK
  C:5E4BH         LINE#         68
  C:5E4BH         LINE#         69
  C:5E4BH         LINE#         70
  C:5E4EH         LINE#         71
  C:5E4EH         LINE#         72
  C:5E50H         LINE#         73
  C:5E52H         LINE#         74
  C:5E57H         LINE#         75
  C:5E5AH         LINE#         76
  C:5E5BH         LINE#         77
  C:5E5EH         LINE#         78
  C:5E5EH         LINE#         79
  C:5E61H         LINE#         80
  C:5E64H         LINE#         81
  C:5E64H         LINE#         82
  C:5E80H         LINE#         83
  C:5E80H         LINE#         84
  C:5E82H         LINE#         85
  C:5E84H         LINE#         86
  C:5E87H         LINE#         87
  C:5E8AH         LINE#         88
  C:5E8AH         LINE#         89
  C:5E8CH         LINE#         90
  C:5E8CH         LINE#         91
  C:5E8EH         LINE#         92
  C:5E8EH         LINE#         93
BL51 BANKED LINKER/LOCATER V6.22                                                      06/21/2022  07:40:42  PAGE 60


  C:5E8EH         LINE#         94
  C:5E8EH         LINE#         95
  -------         ENDPROC       CHGERCHECK
  -------         ENDMOD        CHARGERLOAD

  -------         MODULE        EXTE2PROM
  C:0000H         SYMBOL        _ICE_DUMMY_
  D:0080H         PUBLIC        P0
  D:0090H         PUBLIC        P1
  D:00A0H         PUBLIC        P2
  C:2D4AH         PUBLIC        _E2PRomBKData
  D:00B0H         PUBLIC        P3
  D:00C0H         PUBLIC        P4
  D:0080H         PUBLIC        P5
  C:525BH         PUBLIC        _E2PRomWrite
  C:4DF5H         PUBLIC        E2PRomInit
  C:6529H         PUBLIC        E2PRomTwiCheck
  X:0359H         PUBLIC        ucRTCBKTime1
  B:0027H.0       PUBLIC        bRTCRdTime
  X:035AH         PUBLIC        uiRTCBKTime2
  C:5F58H         PUBLIC        E2PRomBKBoot
  B:0027H.1       PUBLIC        bE2PErase
  X:035CH         PUBLIC        uiE2PDataAddr
  B:0027H.2       PUBLIC        bE2PRErr
  B:0027H.3       PUBLIC        bE2PProcessFlg
  I:002FH         PUBLIC        ucUpDataLimitTime
  D:0099H         PUBLIC        SBUF
  X:035EH         PUBLIC        uiCHGValidTime
  D:00B1H         PUBLIC        RSTSTAT
  C:5CF2H         PUBLIC        UartRdRTC
  X:0360H         PUBLIC        ucE2PTwiRWErrDelayCnt
  C:518CH         PUBLIC        UartRdE2PRom
  B:0027H.4       PUBLIC        bE2PTwiRWErrFlg
  B:0027H.5       PUBLIC        bE2PRdData
  B:0027H.6       PUBLIC        bE2PBKChgStart
  X:0361H         PUBLIC        ucRTCBuf
  B:0027H.7       PUBLIC        bE2PBKRtc
  B:0028H.0       PUBLIC        bE2PBKDsgEndValid
  B:0098H.4       PUBLIC        REN
  C:3B50H         PUBLIC        E2PRomBKCheck
  C:564CH         PUBLIC        E2PRomBKProcess
  C:50B5H         PUBLIC        E2PRomErase
  C:5A18H         PUBLIC        E2PRomBKRTC
  B:0028H.1       PUBLIC        bE2PBKDsgEnd
  B:0028H.2       PUBLIC        bChgToDsgFlg
  B:0028H.3       PUBLIC        bDsgToChgFlg
  B:0028H.4       PUBLIC        bE2PBKChgStop
  C:52BAH         PUBLIC        _E2PRomRead
  -------         PROC          E2PROMTWICHECK
  C:6529H         LINE#         39
  C:6529H         LINE#         40
  C:6529H         LINE#         41
  C:652CH         LINE#         42
  C:652CH         LINE#         43
  C:652FH         LINE#         44
  C:652FH         LINE#         45
  C:653AH         LINE#         46
BL51 BANKED LINKER/LOCATER V6.22                                                      06/21/2022  07:40:42  PAGE 61


  C:653AH         LINE#         47
  C:653CH         LINE#         48
  C:653FH         LINE#         49
  C:653FH         LINE#         50
  C:6540H         LINE#         52
  C:6540H         LINE#         53
  C:6545H         LINE#         54
  C:6545H         LINE#         55
  C:6545H         LINE#         56
  -------         ENDPROC       E2PROMTWICHECK
  -------         PROC          _E2PROMWRITE
  X:02E3H         SYMBOL        WrAddr
  X:02E5H         SYMBOL        Length
  X:02E6H         SYMBOL        WrBuf
  -------         DO            
  B:0028H.5       SYMBOL        Result
  X:02E8H         SYMBOL        i
  -------         ENDDO         
  C:525BH         LINE#         65
  C:526CH         LINE#         66
  C:526CH         LINE#         67
  C:526EH         LINE#         70
  C:5271H         LINE#         71
  C:5271H         LINE#         72
  C:5274H         LINE#         73
  C:5274H         LINE#         74
  C:529DH         LINE#         75
  C:529DH         LINE#         76
  C:529FH         LINE#         77
  C:52A1H         LINE#         78
  C:52A1H         LINE#         79
  C:52A6H         LINE#         80
  C:52B2H         LINE#         81
  C:52B2H         LINE#         82
  C:52B7H         LINE#         84
  C:52B9H         LINE#         85
  -------         ENDPROC       _E2PROMWRITE
  -------         PROC          _E2PROMREAD
  X:02C5H         SYMBOL        RdAddr
  X:02C7H         SYMBOL        Length
  X:02C8H         SYMBOL        RdBuf
  -------         DO            
  B:0028H.6       SYMBOL        Result
  X:02CAH         SYMBOL        i
  -------         ENDDO         
  C:52BAH         LINE#         94
  C:52CBH         LINE#         95
  C:52CBH         LINE#         96
  C:52CDH         LINE#         99
  C:52D0H         LINE#         100
  C:52D0H         LINE#         101
  C:52D3H         LINE#         102
  C:52D3H         LINE#         103
  C:52FCH         LINE#         104
  C:52FCH         LINE#         105
  C:52FEH         LINE#         106
  C:5300H         LINE#         107
BL51 BANKED LINKER/LOCATER V6.22                                                      06/21/2022  07:40:42  PAGE 62


  C:5300H         LINE#         108
  C:5305H         LINE#         109
  C:5311H         LINE#         110
  C:5311H         LINE#         111
  C:5316H         LINE#         113
  C:5318H         LINE#         114
  -------         ENDPROC       _E2PROMREAD
  -------         PROC          E2PROMERASE
  -------         DO            
  X:02BAH         SYMBOL        i
  X:02BCH         SYMBOL        WrBuf
  -------         ENDDO         
  C:50B5H         LINE#         124
  C:50B5H         LINE#         125
  C:50B5H         LINE#         129
  C:50C0H         LINE#         131
  C:50DEH         LINE#         132
  C:50DEH         LINE#         133
  C:50E1H         LINE#         134
  C:5100H         LINE#         135
  C:510CH         LINE#         137
  C:5119H         LINE#         138
  C:5120H         LINE#         139
  -------         ENDPROC       E2PROMERASE
  -------         PROC          E2PROMINIT
  -------         DO            
  B:0028H.5       SYMBOL        Result
  X:02B9H         SYMBOL        RdBuf
  -------         ENDDO         
  C:4DF5H         LINE#         148
  C:4DF5H         LINE#         149
  C:4DF5H         LINE#         150
  C:4DF7H         LINE#         154
  C:4E06H         LINE#         156
  C:4E14H         LINE#         157
  C:4E22H         LINE#         159
  C:4E2EH         LINE#         160
  C:4E2EH         LINE#         161
  C:4E43H         LINE#         162
  C:4E45H         LINE#         163
  C:4E51H         LINE#         164
  C:4E51H         LINE#         165
  C:4E66H         LINE#         166
  C:4E68H         LINE#         168
  C:4E68H         LINE#         169
  C:4E6FH         LINE#         170
  C:4E6FH         LINE#         172
  C:4E71H         LINE#         173
  -------         ENDPROC       E2PROMINIT
  -------         PROC          E2PROMBKRTC
  -------         DO            
  X:02BAH         SYMBOL        WrBuf
  D:0007H         SYMBOL        i
  X:02C3H         SYMBOL        checksum
  -------         ENDDO         
  C:5A18H         LINE#         182
  C:5A18H         LINE#         183
BL51 BANKED LINKER/LOCATER V6.22                                                      06/21/2022  07:40:42  PAGE 63


  C:5A18H         LINE#         185
  C:5A1DH         LINE#         187
  C:5A24H         LINE#         188
  C:5A31H         LINE#         189
  C:5A33H         LINE#         190
  C:5A33H         LINE#         191
  C:5A45H         LINE#         192
  C:5A4AH         LINE#         193
  C:5A52H         LINE#         194
  C:5A56H         LINE#         196
  C:5A63H         LINE#         197
  -------         ENDPROC       E2PROMBKRTC
  -------         PROC          E2PROMBKBOOT
  -------         DO            
  X:02DBH         SYMBOL        WrBuf
  -------         ENDDO         
  C:5F58H         LINE#         206
  C:5F58H         LINE#         207
  C:5F58H         LINE#         210
  C:5F65H         LINE#         211
  C:5F6AH         LINE#         212
  C:5F73H         LINE#         214
  C:5F7BH         LINE#         215
  C:5F83H         LINE#         216
  C:5F8BH         LINE#         218
  C:5F98H         LINE#         219
  -------         ENDPROC       E2PROMBKBOOT
  -------         PROC          _E2PROMBKDATA
  X:02BAH         SYMBOL        BKType
  -------         DO            
  X:02BBH         SYMBOL        WrBuf
  -------         ENDDO         
  C:2D4AH         LINE#         228
  C:2D4FH         LINE#         229
  C:2D4FH         LINE#         232
  C:2D53H         LINE#         233
  C:2D53H         LINE#         234
  C:2D60H         LINE#         235
  C:2D6BH         LINE#         236
  C:2D6DH         LINE#         238
  C:2D6DH         LINE#         239
  C:2D74H         LINE#         240
  C:2D81H         LINE#         241
  C:2D8CH         LINE#         242
  C:2D8CH         LINE#         244
  C:2D99H         LINE#         245
  C:2D9CH         LINE#         246
  C:2DA9H         LINE#         247
  C:2DACH         LINE#         248
  C:2DBCH         LINE#         249
  C:2DCCH         LINE#         250
  C:2DDCH         LINE#         251
  C:2DE7H         LINE#         252
  C:2DF7H         LINE#         253
  C:2E07H         LINE#         254
  C:2E17H         LINE#         255
  C:2E22H         LINE#         256
BL51 BANKED LINKER/LOCATER V6.22                                                      06/21/2022  07:40:42  PAGE 64


  C:2E39H         LINE#         257
  C:2E49H         LINE#         258
  C:2E56H         LINE#         259
  C:2E59H         LINE#         260
  C:2E69H         LINE#         261
  C:2E79H         LINE#         262
  C:2E89H         LINE#         263
  C:2E94H         LINE#         264
  C:2EA1H         LINE#         265
  C:2EA4H         LINE#         266
  C:2EB1H         LINE#         267
  C:2EB4H         LINE#         268
  C:2EBCH         LINE#         269
  C:2EC0H         LINE#         271
  C:2ED1H         LINE#         273
  C:2EDBH         LINE#         274
  C:2EF2H         LINE#         275
  C:2EF2H         LINE#         276
  C:2EF9H         LINE#         277
  C:2EF9H         LINE#         279
  C:2EFCH         LINE#         280
  -------         ENDPROC       _E2PROMBKDATA
  -------         PROC          UARTRDE2PROM
  -------         DO            
  D:0006H         SYMBOL        RdAddr
  -------         ENDDO         
  C:518CH         LINE#         289
  C:518CH         LINE#         290
  C:518CH         LINE#         293
  C:51B7H         LINE#         294
  C:51C3H         LINE#         296
  C:51E2H         LINE#         297
  C:51F4H         LINE#         298
  -------         ENDPROC       UARTRDE2PROM
  -------         PROC          UARTRDRTC
  C:5CF2H         LINE#         307
  C:5CF2H         LINE#         308
  C:5CF2H         LINE#         309
  C:5CF9H         LINE#         310
  C:5D06H         LINE#         312
  C:5D25H         LINE#         313
  C:5D37H         LINE#         314
  -------         ENDPROC       UARTRDRTC
  -------         PROC          E2PROMBKPROCESS
  -------         DO            
  X:02B9H         SYMBOL        BKType
  -------         ENDDO         
  C:564CH         LINE#         323
  C:564CH         LINE#         324
  C:564CH         LINE#         327
  C:5652H         LINE#         328
  C:5652H         LINE#         329
  C:5654H         LINE#         333
  C:5657H         LINE#         334
  C:5657H         LINE#         335
  C:5659H         LINE#         336
  C:565CH         LINE#         337
BL51 BANKED LINKER/LOCATER V6.22                                                      06/21/2022  07:40:42  PAGE 65


  C:565CH         LINE#         339
  C:565FH         LINE#         340
  C:565FH         LINE#         341
  C:5661H         LINE#         342
  C:5664H         LINE#         343
  C:5664H         LINE#         345
  C:5667H         LINE#         346
  C:5667H         LINE#         347
  C:5669H         LINE#         348
  C:566CH         LINE#         349
  C:566CH         LINE#         351
  C:566FH         LINE#         352
  C:566FH         LINE#         353
  C:5671H         LINE#         354
  C:5674H         LINE#         355
  C:5674H         LINE#         357
  C:5677H         LINE#         358
  C:5677H         LINE#         359
  C:5679H         LINE#         360
  C:567FH         LINE#         361
  C:5683H         LINE#         362
  C:5683H         LINE#         364
  C:5686H         LINE#         365
  C:5686H         LINE#         366
  C:5688H         LINE#         367
  C:568EH         LINE#         368
  C:5692H         LINE#         369
  C:5692H         LINE#         371
  C:5695H         LINE#         372
  C:5695H         LINE#         373
  C:5697H         LINE#         374
  C:569DH         LINE#         375
  C:56A1H         LINE#         376
  C:56A1H         LINE#         377
  C:56A1H         LINE#         378
  -------         ENDPROC       E2PROMBKPROCESS
  -------         PROC          E2PROMBKCHECK
  C:3B50H         LINE#         387
  C:3B50H         LINE#         388
  C:3B50H         LINE#         389
  C:3B56H         LINE#         390
  C:3B56H         LINE#         394
  C:3B65H         LINE#         395
  C:3B65H         LINE#         396
  C:3B67H         LINE#         397
  C:3B6EH         LINE#         398
  C:3B6EH         LINE#         400
  C:3B83H         LINE#         401
  C:3B83H         LINE#         402
  C:3B8AH         LINE#         403
  C:3B8CH         LINE#         404
  C:3B8EH         LINE#         405
  C:3B8EH         LINE#         407
  C:3B91H         LINE#         408
  C:3B91H         LINE#         409
  C:3B93H         LINE#         410
  C:3B96H         LINE#         411
BL51 BANKED LINKER/LOCATER V6.22                                                      06/21/2022  07:40:42  PAGE 66


  C:3B96H         LINE#         412
  C:3B98H         LINE#         413
  C:3B9AH         LINE#         414
  C:3B9CH         LINE#         415
  C:3B9CH         LINE#         416
  C:3BA2H         LINE#         417
  C:3BA2H         LINE#         418
  C:3BA4H         LINE#         419
  C:3BA6H         LINE#         420
  C:3BA8H         LINE#         421
  C:3BAAH         LINE#         422
  C:3BADH         LINE#         423
  C:3BADH         LINE#         424
  C:3BAFH         LINE#         425
  C:3BAFH         LINE#         426
  C:3BAFH         LINE#         428
  C:3BCCH         LINE#         429
  C:3BCCH         LINE#         430
  C:3BD6H         LINE#         431
  C:3BD6H         LINE#         432
  C:3BDDH         LINE#         433
  C:3BEAH         LINE#         434
  C:3BEAH         LINE#         436
  C:3C0BH         LINE#         437
  C:3C0BH         LINE#         438
  C:3C12H         LINE#         439
  C:3C14H         LINE#         440
  C:3C16H         LINE#         441
  C:3C18H         LINE#         442
  C:3C1AH         LINE#         443
  C:3C1AH         LINE#         444
  C:3C1BH         LINE#         446
  C:3C1BH         LINE#         447
  C:3C22H         LINE#         448
  C:3C22H         LINE#         449
  C:3C22H         LINE#         450
  -------         ENDPROC       E2PROMBKCHECK
  -------         ENDMOD        EXTE2PROM

  -------         MODULE        INTERRUPT
  C:0000H         SYMBOL        _ICE_DUMMY_
  D:0080H         PUBLIC        P0
  D:0090H         PUBLIC        P1
  D:00A0H         PUBLIC        P2
  D:00B0H         PUBLIC        P3
  D:00C0H         PUBLIC        P4
  D:0080H         PUBLIC        P5
  C:1003H         PUBLIC        InterruptTimer3
  D:0086H         PUBLIC        INSCON
  B:0088H.7       PUBLIC        TF3
  B:00D8H.0       PUBLIC        IF40
  C:5121H         PUBLIC        InterruptINT4
  B:00D8H.1       PUBLIC        IF41
  B:00D8H.2       PUBLIC        IF42
  B:00D8H.3       PUBLIC        IF43
  B:00D8H.4       PUBLIC        IF44
  B:00D8H.5       PUBLIC        IF45
BL51 BANKED LINKER/LOCATER V6.22                                                      06/21/2022  07:40:42  PAGE 67


  B:00D8H.6       PUBLIC        IF46
  B:00D8H.7       PUBLIC        IF47
  -------         PROC          INTERRUPTINT4
  C:5121H         LINE#         18
  C:512CH         LINE#         20
  C:512EH         LINE#         21
  C:5131H         LINE#         23
  C:5134H         LINE#         24
  C:5134H         LINE#         25
  C:5136H         LINE#         26
  C:513BH         LINE#         27
  C:513BH         LINE#         28
  C:513EH         LINE#         29
  C:513EH         LINE#         30
  C:5140H         LINE#         31
  C:5145H         LINE#         32
  C:5145H         LINE#         33
  C:5148H         LINE#         34
  C:5148H         LINE#         35
  C:514AH         LINE#         36
  C:514FH         LINE#         37
  C:514FH         LINE#         38
  C:5152H         LINE#         39
  C:5152H         LINE#         40
  C:5154H         LINE#         41
  C:5159H         LINE#         42
  C:5159H         LINE#         43
  C:515CH         LINE#         44
  C:515CH         LINE#         45
  C:515EH         LINE#         46
  C:5163H         LINE#         47
  C:5163H         LINE#         48
  C:5166H         LINE#         49
  C:5166H         LINE#         50
  C:5168H         LINE#         51
  C:516DH         LINE#         52
  C:516DH         LINE#         53
  C:5170H         LINE#         54
  C:5170H         LINE#         55
  C:5172H         LINE#         56
  C:5177H         LINE#         57
  C:5177H         LINE#         58
  C:517AH         LINE#         59
  C:517AH         LINE#         60
  C:517CH         LINE#         61
  C:5181H         LINE#         62
  C:5181H         LINE#         64
  C:5183H         LINE#         65
  -------         ENDPROC       INTERRUPTINT4
  -------         PROC          INTERRUPTTIMER3
  C:1003H         LINE#         74
  C:100BH         LINE#         76
  C:100DH         LINE#         78
  C:1010H         LINE#         79
  C:1012H         LINE#         80
  C:1015H         LINE#         82
  C:1018H         LINE#         84
BL51 BANKED LINKER/LOCATER V6.22                                                      06/21/2022  07:40:42  PAGE 68


  C:101AH         LINE#         85
  -------         ENDPROC       INTERRUPTTIMER3
  -------         ENDMOD        INTERRUPT

  -------         MODULE        KEYSCAN
  C:0000H         SYMBOL        _ICE_DUMMY_
  D:0080H         PUBLIC        P0
  D:0090H         PUBLIC        P1
  D:00A0H         PUBLIC        P2
  D:00B0H         PUBLIC        P3
  D:00C0H         PUBLIC        P4
  D:0008H         PUBLIC        ucKeyValue
  D:0080H         PUBLIC        P5
  D:0009H         PUBLIC        ucKeyValueBK
  B:00B0H.0       PUBLIC        P3_0
  B:00A0H.7       PUBLIC        P2_7
  D:000AH         PUBLIC        uiKeyValidCnt
  D:000CH         PUBLIC        ucKeyOldValue
  B:002EH.4       PUBLIC        bKeyFlg
  C:4627H         PUBLIC        KeyScan
  D:000DH         PUBLIC        uiKeyInvalidCnt
  -------         PROC          KEYSCAN
  -------         DO            
  C:46BCH         SYMBOL        scanend
  -------         ENDDO         
  C:4627H         LINE#         33
  C:4627H         LINE#         34
  C:4627H         LINE#         35
  C:462DH         LINE#         36
  C:462DH         LINE#         37
  C:4630H         LINE#         46
  C:4633H         LINE#         47
  C:4633H         LINE#         48
  C:4636H         LINE#         49
  C:4638H         LINE#         50
  C:463BH         LINE#         51
  C:463BH         LINE#         52
  C:463EH         LINE#         53
  C:463EH         LINE#         69
  C:4644H         LINE#         70
  C:4644H         LINE#         71
  C:464CH         LINE#         72
  C:4657H         LINE#         73
  C:4657H         LINE#         74
  C:4661H         LINE#         75
  C:4661H         LINE#         76
  C:466BH         LINE#         77
  C:466BH         LINE#         78
  C:4671H         LINE#         79
  C:4673H         LINE#         81
  C:4673H         LINE#         82
  C:4676H         LINE#         83
  C:4676H         LINE#         84
  C:4678H         LINE#         85
  C:467AH         LINE#         86
  C:467AH         LINE#         91
  C:467AH         LINE#         93
BL51 BANKED LINKER/LOCATER V6.22                                                      06/21/2022  07:40:42  PAGE 69


  C:467AH         LINE#         94
  C:467CH         LINE#         95
  C:467CH         LINE#         96
  C:467CH         LINE#         98
  C:467CH         LINE#         99
  C:4682H         LINE#         100
  C:4682H         LINE#         101
  C:4687H         LINE#         102
  C:468FH         LINE#         103
  C:4697H         LINE#         104
  C:4697H         LINE#         105
  C:469DH         LINE#         106
  C:469FH         LINE#         107
  C:46A0H         LINE#         108
  C:46AAH         LINE#         109
  C:46AAH         LINE#         110
  C:46B0H         LINE#         111
  C:46B6H         LINE#         112
  C:46B8H         LINE#         113
  C:46B8H         LINE#         114
  C:46B9H         LINE#         116
  C:46B9H         LINE#         117
  C:46BCH         LINE#         118
  C:46BCH         LINE#         119
  C:46C1H         LINE#         120
  C:46C5H         LINE#         121
  C:46C8H         LINE#         122
  C:46C8H         LINE#         123
  C:46C8H         LINE#         124
  C:46C8H         LINE#         125
  -------         ENDPROC       KEYSCAN
  -------         ENDMOD        KEYSCAN

  -------         MODULE        MCUFLASH
  C:0000H         SYMBOL        _ICE_DUMMY_
  D:00F3H         PUBLIC        IB_CON2
  D:0080H         PUBLIC        P0
  D:00F4H         PUBLIC        IB_CON3
  D:0090H         PUBLIC        P1
  D:00F5H         PUBLIC        IB_CON4
  D:00A0H         PUBLIC        P2
  D:00F6H         PUBLIC        IB_CON5
  D:00B0H         PUBLIC        P3
  D:00C0H         PUBLIC        P4
  X:039EH         PUBLIC        bMcuFlashWrWaitCnt
  D:0080H         PUBLIC        P5
  B:00A8H.7       PUBLIC        EA
  D:00FCH         PUBLIC        IB_DATA
  C:63A0H         PUBLIC        _McuFlashCheckFlg
  C:5319H         PUBLIC        _McuFlashRead
  C:6217H         PUBLIC        _McuFlashWrOneByte
  B:002DH.0       PUBLIC        bMcuFlashErr
  C:489DH         PUBLIC        _McuFlashWrite
  X:039FH         PUBLIC        ucMcuFlashWrValid
  D:00FBH         PUBLIC        IB_OFFSET
  D:00B1H         PUBLIC        RSTSTAT
  D:00A7H         PUBLIC        FLASHCON
BL51 BANKED LINKER/LOCATER V6.22                                                      06/21/2022  07:40:42  PAGE 70


  C:4A52H         PUBLIC        _McuFlashWrSector
  C:65DDH         PUBLIC        McuFlashWrWaitCheck
  B:002DH.1       PUBLIC        bMcuFlashWrFlg
  C:643AH         PUBLIC        _McuFlashBlankCheck
  C:54E7H         PUBLIC        _McuFlashDataCheck
  D:00F7H         PUBLIC        XPAGE
  B:002DH.2       PUBLIC        bMcuFlashWrWaitFlg
  C:3C23H         PUBLIC        McuFlashProcess
  D:00F2H         PUBLIC        IB_CON1
  -------         PROC          _MCUFLASHWRONEBYTE
  D:0002H         SYMBOL        McuFlashAddr
  D:0005H         SYMBOL        WrData
  C:6217H         LINE#         24
  C:621BH         LINE#         25
  C:621BH         LINE#         26
  C:621DH         LINE#         27
  C:6220H         LINE#         29
  C:6223H         LINE#         30
  C:6227H         LINE#         31
  C:622BH         LINE#         33
  C:622EH         LINE#         34
  C:6231H         LINE#         35
  C:6234H         LINE#         36
  C:6237H         LINE#         37
  C:623EH         LINE#         38
  C:623EH         LINE#         39
  C:6241H         LINE#         40
  C:6242H         LINE#         41
  C:6243H         LINE#         42
  C:6244H         LINE#         43
  C:6245H         LINE#         44
  C:6246H         LINE#         45
  C:6246H         LINE#         47
  C:6249H         LINE#         48
  C:624BH         LINE#         49
  -------         ENDPROC       _MCUFLASHWRONEBYTE
  -------         PROC          _MCUFLASHBLANKCHECK
  D:0006H         SYMBOL        McuFlashAddr
  -------         DO            
  B:0029H.0       SYMBOL        Result
  D:0004H         SYMBOL        i
  -------         ENDDO         
  C:643AH         LINE#         58
  C:643AH         LINE#         59
  C:643AH         LINE#         60
  C:643CH         LINE#         63
  C:643FH         LINE#         64
  C:643FH         LINE#         65
  C:644CH         LINE#         66
  C:644CH         LINE#         67
  C:644EH         LINE#         68
  C:6450H         LINE#         69
  C:6450H         LINE#         70
  C:645DH         LINE#         72
  C:645FH         LINE#         73
  -------         ENDPROC       _MCUFLASHBLANKCHECK
  -------         PROC          _MCUFLASHDATACHECK
BL51 BANKED LINKER/LOCATER V6.22                                                      06/21/2022  07:40:42  PAGE 71


  X:02BFH         SYMBOL        McuFlashAddr
  D:0004H         SYMBOL        XramAddr
  -------         DO            
  B:0029H.0       SYMBOL        Result
  D:0006H         SYMBOL        ptr
  X:02C1H         SYMBOL        i
  -------         ENDDO         
  C:54E7H         LINE#         82
  C:54EFH         LINE#         83
  C:54EFH         LINE#         84
  C:54F1H         LINE#         85
  C:54F5H         LINE#         88
  C:5508H         LINE#         89
  C:5508H         LINE#         90
  C:552EH         LINE#         91
  C:552EH         LINE#         92
  C:5530H         LINE#         93
  C:5532H         LINE#         94
  C:5532H         LINE#         95
  C:553EH         LINE#         97
  C:5540H         LINE#         98
  -------         ENDPROC       _MCUFLASHDATACHECK
  -------         PROC          _MCUFLASHWRSECTOR
  X:02BFH         SYMBOL        McuFlashAddr
  D:0004H         SYMBOL        XramAddr
  -------         DO            
  B:0029H.0       SYMBOL        Result
  D:0004H         SYMBOL        i
  X:02C1H         SYMBOL        ptr
  -------         ENDDO         
  C:4A52H         LINE#         107
  C:4A5AH         LINE#         108
  C:4A5AH         LINE#         109
  C:4A5CH         LINE#         111
  C:4A64H         LINE#         113
  C:4A67H         LINE#         114
  C:4A67H         LINE#         115
  C:4A72H         LINE#         116
  C:4A78H         LINE#         117
  C:4A87H         LINE#         118
  C:4A8AH         LINE#         119
  C:4A8DH         LINE#         120
  C:4A8DH         LINE#         121
  C:4A90H         LINE#         122
  C:4A94H         LINE#         123
  C:4A94H         LINE#         124
  C:4A97H         LINE#         125
  C:4A9FH         LINE#         126
  C:4A9FH         LINE#         127
  C:4AA2H         LINE#         128
  C:4AB2H         LINE#         129
  C:4AB2H         LINE#         130
  C:4AB5H         LINE#         131
  C:4AB6H         LINE#         132
  C:4AB7H         LINE#         133
  C:4AB8H         LINE#         134
  C:4AB9H         LINE#         135
BL51 BANKED LINKER/LOCATER V6.22                                                      06/21/2022  07:40:42  PAGE 72


  C:4ABAH         LINE#         136
  C:4ABCH         LINE#         137
  C:4ABEH         LINE#         139
  C:4ABEH         LINE#         140
  C:4AC0H         LINE#         141
  C:4AC2H         LINE#         142
  C:4AC2H         LINE#         143
  C:4AC2H         LINE#         145
  C:4AC2H         LINE#         146
  C:4AC4H         LINE#         147
  C:4AC6H         LINE#         148
  C:4AC6H         LINE#         149
  C:4AC6H         LINE#         151
  C:4AC6H         LINE#         152
  C:4AC8H         LINE#         153
  C:4ACAH         LINE#         154
  C:4ACAH         LINE#         155
  C:4ACAH         LINE#         157
  C:4ACAH         LINE#         158
  C:4ACCH         LINE#         159
  C:4ACEH         LINE#         160
  C:4ACEH         LINE#         161
  C:4ADBH         LINE#         163
  C:4ADDH         LINE#         164
  -------         ENDPROC       _MCUFLASHWRSECTOR
  -------         PROC          _MCUFLASHWRITE
  X:02BBH         SYMBOL        McuFlashAddr
  X:02BDH         SYMBOL        XramAddr
  -------         DO            
  B:0028H.7       SYMBOL        Result
  -------         ENDDO         
  C:489DH         LINE#         177
  C:48ABH         LINE#         178
  C:48ABH         LINE#         179
  C:48ADH         LINE#         181
  C:48B0H         LINE#         182
  C:48B2H         LINE#         183
  C:48B5H         LINE#         185
  C:48BEH         LINE#         186
  C:48C1H         LINE#         187
  C:48C4H         LINE#         188
  C:48C4H         LINE#         189
  C:48C7H         LINE#         190
  C:48CBH         LINE#         191
  C:48CBH         LINE#         192
  C:48CEH         LINE#         193
  C:48D6H         LINE#         194
  C:48D6H         LINE#         195
  C:48D9H         LINE#         196
  C:48E2H         LINE#         197
  C:48E2H         LINE#         198
  C:48E5H         LINE#         199
  C:48E6H         LINE#         200
  C:48E7H         LINE#         201
  C:48E8H         LINE#         202
  C:48E9H         LINE#         203
  C:48EAH         LINE#         205
BL51 BANKED LINKER/LOCATER V6.22                                                      06/21/2022  07:40:42  PAGE 73


  C:48F7H         LINE#         206
  C:48F7H         LINE#         207
  C:490AH         LINE#         208
  C:490AH         LINE#         209
  C:491DH         LINE#         210
  C:491DH         LINE#         211
  C:491FH         LINE#         212
  C:491FH         LINE#         213
  C:491FH         LINE#         214
  C:491FH         LINE#         215
  C:491FH         LINE#         216
  C:491FH         LINE#         217
  C:491FH         LINE#         218
  C:491FH         LINE#         220
  C:4922H         LINE#         221
  C:4924H         LINE#         222
  C:4926H         LINE#         223
  C:4928H         LINE#         224
  C:492AH         LINE#         226
  C:492DH         LINE#         227
  C:492FH         LINE#         228
  C:4931H         LINE#         230
  C:4933H         LINE#         231
  -------         ENDPROC       _MCUFLASHWRITE
  -------         PROC          MCUFLASHPROCESS
  -------         DO            
  B:0028H.5       SYMBOL        McuFlashBk1WrFailFlg
  B:0028H.6       SYMBOL        McuFlashBk2WrFailFlg
  X:02B9H         SYMBOL        VoltageMin
  -------         ENDDO         
  C:3C23H         LINE#         244
  C:3C23H         LINE#         245
  C:3C23H         LINE#         246
  C:3C27H         LINE#         249
  C:3C2DH         LINE#         250
  C:3C2DH         LINE#         251
  C:3C2FH         LINE#         253
  C:3C35H         LINE#         254
  C:3C3CH         LINE#         255
  C:3C3CH         LINE#         256
  C:3C46H         LINE#         257
  C:3C48H         LINE#         259
  C:3C48H         LINE#         260
  C:3C52H         LINE#         261
  C:3C52H         LINE#         263
  C:3C75H         LINE#         264
  C:3C75H         LINE#         265
  C:3C7EH         LINE#         266
  C:3C7EH         LINE#         267
  C:3C88H         LINE#         268
  C:3C88H         LINE#         269
  C:3C8AH         LINE#         270
  C:3C92H         LINE#         271
  C:3C9AH         LINE#         272
  C:3CA1H         LINE#         273
  C:3CA1H         LINE#         274
  C:3CA1H         LINE#         276
BL51 BANKED LINKER/LOCATER V6.22                                                      06/21/2022  07:40:42  PAGE 74


  C:3CACH         LINE#         277
  C:3CACH         LINE#         278
  C:3CB7H         LINE#         279
  C:3CB7H         LINE#         280
  C:3CB9H         LINE#         281
  C:3CC1H         LINE#         282
  C:3CC9H         LINE#         283
  C:3CD0H         LINE#         284
  C:3CD0H         LINE#         285
  C:3CD0H         LINE#         286
  C:3CD2H         LINE#         288
  C:3CD2H         LINE#         289
  C:3CD4H         LINE#         290
  C:3CD6H         LINE#         291
  C:3CD6H         LINE#         292
  C:3CDBH         LINE#         294
  C:3CE1H         LINE#         295
  C:3CE1H         LINE#         296
  C:3CE3H         LINE#         297
  C:3CE3H         LINE#         298
  C:3CE3H         LINE#         299
  -------         ENDPROC       MCUFLASHPROCESS
  -------         PROC          _MCUFLASHREAD
  X:02B9H         SYMBOL        SourceAddr
  D:0004H         SYMBOL        TargetAddr
  X:02BBH         SYMBOL        Length
  -------         DO            
  D:0006H         SYMBOL        i
  B:0028H.5       SYMBOL        Result
  D:0015H         SYMBOL        TargetAddr1
  -------         ENDDO         
  C:5319H         LINE#         308
  C:5327H         LINE#         309
  C:5327H         LINE#         311
  C:5329H         LINE#         312
  C:5331H         LINE#         314
  C:5333H         LINE#         315
  C:5336H         LINE#         316
  C:5339H         LINE#         317
  C:5349H         LINE#         318
  C:5349H         LINE#         319
  C:5361H         LINE#         320
  C:5369H         LINE#         321
  C:5370H         LINE#         322
  C:5373H         LINE#         323
  C:5375H         LINE#         325
  C:5377H         LINE#         326
  -------         ENDPROC       _MCUFLASHREAD
  -------         PROC          MCUFLASHWRWAITCHECK
  C:65DDH         LINE#         335
  C:65DDH         LINE#         336
  C:65DDH         LINE#         337
  C:65E0H         LINE#         338
  C:65E0H         LINE#         339
  C:65EBH         LINE#         340
  C:65EBH         LINE#         341
  C:65EDH         LINE#         342
BL51 BANKED LINKER/LOCATER V6.22                                                      06/21/2022  07:40:42  PAGE 75


  C:65EFH         LINE#         343
  C:65F1H         LINE#         344
  C:65F1H         LINE#         345
  C:65F1H         LINE#         346
  -------         ENDPROC       MCUFLASHWRWAITCHECK
  -------         PROC          _MCUFLASHCHECKFLG
  D:0006H         SYMBOL        McuFlashAddr
  -------         DO            
  B:0028H.5       SYMBOL        Result
  -------         ENDDO         
  C:63A0H         LINE#         355
  C:63A0H         LINE#         356
  C:63A0H         LINE#         357
  C:63A2H         LINE#         359
  C:63A5H         LINE#         360
  C:63BFH         LINE#         361
  C:63BFH         LINE#         362
  C:63C1H         LINE#         363
  C:63C1H         LINE#         364
  C:63C4H         LINE#         366
  C:63C6H         LINE#         367
  -------         ENDPROC       _MCUFLASHCHECKFLG
  -------         ENDMOD        MCUFLASH

  -------         MODULE        MCULIB
  C:0000H         SYMBOL        _ICE_DUMMY_
  D:0080H         PUBLIC        P0
  D:0090H         PUBLIC        P1
  D:00A0H         PUBLIC        P2
  D:00B0H         PUBLIC        P3
  D:00C0H         PUBLIC        P4
  C:5C1AH         PUBLIC        _Delay1ms
  D:009DH         PUBLIC        SBRTH
  D:0080H         PUBLIC        P5
  B:00A8H.7       PUBLIC        EA
  D:00C7H         PUBLIC        PWM0CON
  D:00B6H         PUBLIC        PWM1CON
  D:00B7H         PUBLIC        PWM2CON
  D:009CH         PUBLIC        SBRTL
  C:36F1H         PUBLIC        _McuTimer3Set
  D:00A8H         PUBLIC        IEN0
  D:00A9H         PUBLIC        IEN1
  D:00E8H         PUBLIC        EXF0
  D:008EH         PUBLIC        SUSLO
  C:62E6H         PUBLIC        _MemoryCopy
  C:6376H         PUBLIC        _MemorySet
  D:0087H         PUBLIC        PCON
  D:00CFH         PUBLIC        PWM0DH
  D:00A5H         PUBLIC        PWM1DH
  D:00BFH         PUBLIC        PWM2DH
  D:0098H         PUBLIC        SCON
  D:0088H         PUBLIC        TCON
  D:00CEH         PUBLIC        PWM0DL
  D:00A4H         PUBLIC        PWM1DL
  D:00BEH         PUBLIC        PWM2DL
  D:00B2H         PUBLIC        CLKCON
  D:00CDH         PUBLIC        PWM0PH
BL51 BANKED LINKER/LOCATER V6.22                                                      06/21/2022  07:40:42  PAGE 76


  D:00AFH         PUBLIC        PWM1PH
  D:00BDH         PUBLIC        PWM2PH
  D:00CCH         PUBLIC        PWM0PL
  D:00AEH         PUBLIC        PWM1PL
  C:677CH         PUBLIC        McuIntoIdle
  C:579DH         PUBLIC        _McuClockSet
  C:62B3H         PUBLIC        ClrRam
  D:00BCH         PUBLIC        PWM2PL
  D:0086H         PUBLIC        INSCON
  D:008DH         PUBLIC        TH3
  D:008CH         PUBLIC        TL3
  C:6788H         PUBLIC        McuIntoPD
  B:0088H.2       PUBLIC        TR3
  C:51F5H         PUBLIC        RamCheckProcess
  D:0088H         PUBLIC        T3CON
  C:6460H         PUBLIC        SystemResetProcess
  C:4C72H         PUBLIC        _McuPWM0Set
  C:4CF3H         PUBLIC        _McuPWM1Set
  C:4D74H         PUBLIC        _McuPWM2Set
  -------         PROC          _MCUTIMER3SET
  X:02B9H         SYMBOL        ClkSource
  X:02BAH         SYMBOL        XmS
  -------         DO            
  X:02BCH         SYMBOL        TempVal
  -------         ENDDO         
  C:36F1H         LINE#         20
  C:36FEH         LINE#         21
  C:36FEH         LINE#         24
  C:3701H         LINE#         26
  C:3706H         LINE#         27
  C:3706H         LINE#         28
  C:3714H         LINE#         29
  C:3714H         LINE#         30
  C:3717H         LINE#         31
  C:3729H         LINE#         32
  C:372CH         LINE#         34
  C:372CH         LINE#         35
  C:372FH         LINE#         36
  C:3754H         LINE#         37
  C:3754H         LINE#         38
  C:3757H         LINE#         39
  C:375FH         LINE#         40
  C:375FH         LINE#         41
  C:376DH         LINE#         42
  C:376DH         LINE#         43
  C:3770H         LINE#         44
  C:378DH         LINE#         45
  C:3790H         LINE#         47
  C:3790H         LINE#         48
  C:3793H         LINE#         49
  C:37B8H         LINE#         50
  C:37B8H         LINE#         51
  C:37BAH         LINE#         52
  C:37C0H         LINE#         53
  C:37C0H         LINE#         54
  C:37CEH         LINE#         55
  C:37CEH         LINE#         56
BL51 BANKED LINKER/LOCATER V6.22                                                      06/21/2022  07:40:42  PAGE 77


  C:37D1H         LINE#         57
  C:37EEH         LINE#         58
  C:37F0H         LINE#         60
  C:37F0H         LINE#         61
  C:37F3H         LINE#         62
  C:3818H         LINE#         63
  C:3818H         LINE#         64
  C:3818H         LINE#         66
  C:3821H         LINE#         67
  C:3824H         LINE#         68
  C:3826H         LINE#         70
  C:3829H         LINE#         71
  -------         ENDPROC       _MCUTIMER3SET
  -------         PROC          _MCUCLOCKSET
  D:0007H         SYMBOL        SysClock
  -------         DO            
  D:0006H         SYMBOL        ea
  -------         ENDDO         
  C:579DH         LINE#         80
  C:579DH         LINE#         81
  C:579DH         LINE#         84
  C:57A2H         LINE#         85
  C:57A4H         LINE#         87
  C:57B4H         LINE#         89
  C:57B4H         LINE#         90
  C:57B9H         LINE#         91
  C:57BBH         LINE#         92
  C:57C4H         LINE#         93
  C:57C4H         LINE#         94
  C:57C7H         LINE#         95
  C:57C8H         LINE#         96
  C:57CBH         LINE#         97
  C:57CBH         LINE#         98
  C:57CCH         LINE#         99
  C:57CDH         LINE#         100
  C:57CEH         LINE#         101
  C:57CFH         LINE#         102
  C:57D0H         LINE#         103
  C:57D1H         LINE#         104
  C:57D2H         LINE#         105
  C:57D3H         LINE#         106
  C:57E3H         LINE#         108
  C:57E3H         LINE#         109
  C:57E6H         LINE#         110
  C:57E6H         LINE#         112
  C:57EDH         LINE#         113
  -------         ENDPROC       _MCUCLOCKSET
  -------         PROC          _MCUPWM0SET
  X:0392H         SYMBOL        PwmFreq
  X:0394H         SYMBOL        DutyRatio
  C:4C72H         LINE#         122
  C:4C7DH         LINE#         123
  C:4C7DH         LINE#         124
  C:4C80H         LINE#         125
  C:4C9AH         LINE#         126
  C:4CB9H         LINE#         127
  C:4CD7H         LINE#         128
BL51 BANKED LINKER/LOCATER V6.22                                                      06/21/2022  07:40:42  PAGE 78


  C:4CF2H         LINE#         129
  -------         ENDPROC       _MCUPWM0SET
  -------         PROC          _MCUPWM1SET
  X:0395H         SYMBOL        PwmFreq
  X:0397H         SYMBOL        DutyRatio
  C:4CF3H         LINE#         131
  C:4CFEH         LINE#         132
  C:4CFEH         LINE#         133
  C:4D01H         LINE#         134
  C:4D1BH         LINE#         135
  C:4D3AH         LINE#         136
  C:4D58H         LINE#         137
  C:4D73H         LINE#         138
  -------         ENDPROC       _MCUPWM1SET
  -------         PROC          _MCUPWM2SET
  X:02B9H         SYMBOL        PwmFreq
  X:02BBH         SYMBOL        DutyRatio
  C:4D74H         LINE#         140
  C:4D7FH         LINE#         141
  C:4D7FH         LINE#         142
  C:4D82H         LINE#         143
  C:4D9CH         LINE#         144
  C:4DBBH         LINE#         145
  C:4DD9H         LINE#         146
  C:4DF4H         LINE#         147
  -------         ENDPROC       _MCUPWM2SET
  -------         PROC          _DELAY1MS
  D:0007H         SYMBOL        Xms
  -------         DO            
  D:0006H         SYMBOL        i
  D:0002H         SYMBOL        j
  D:0004H         SYMBOL        Tcnt
  -------         ENDDO         
  C:5C1AH         LINE#         160
  C:5C1AH         LINE#         161
  C:5C1AH         LINE#         165
  C:5C20H         LINE#         166
  C:5C20H         LINE#         167
  C:5C24H         LINE#         168
  C:5C26H         LINE#         169
  C:5C2EH         LINE#         170
  C:5C2EH         LINE#         171
  C:5C32H         LINE#         172
  C:5C34H         LINE#         173
  C:5C3CH         LINE#         174
  C:5C3CH         LINE#         175
  C:5C40H         LINE#         176
  C:5C42H         LINE#         178
  C:5C42H         LINE#         179
  C:5C46H         LINE#         180
  C:5C46H         LINE#         183
  C:5C4DH         LINE#         184
  C:5C4DH         LINE#         185
  C:5C57H         LINE#         186
  C:5C57H         LINE#         187
  C:5C5EH         LINE#         188
  C:5C61H         LINE#         189
BL51 BANKED LINKER/LOCATER V6.22                                                      06/21/2022  07:40:42  PAGE 79


  -------         ENDPROC       _DELAY1MS
  -------         PROC          CLRRAM
  -------         DO            
  D:0000H         SYMBOL        ptr1
  D:0006H         SYMBOL        ptr2
  D:0007H         SYMBOL        i
  I:001EH         SYMBOL        j
  -------         ENDDO         
  C:62B3H         LINE#         199
  C:62B3H         LINE#         200
  C:62B3H         LINE#         206
  C:62B5H         LINE#         207
  C:62B5H         LINE#         208
  C:62B9H         LINE#         209
  C:62BBH         LINE#         210
  C:62C2H         LINE#         212
  C:62D7H         LINE#         213
  C:62D7H         LINE#         214
  C:62D7H         LINE#         215
  C:62DDH         LINE#         216
  C:62E5H         LINE#         217
  -------         ENDPROC       CLRRAM
  -------         PROC          RAMCHECKPROCESS
  C:51F5H         LINE#         226
  C:51F5H         LINE#         227
  C:51F5H         LINE#         228
  C:5257H         LINE#         240
  C:5257H         LINE#         241
  C:5259H         LINE#         242
  C:5259H         LINE#         244
  C:5259H         LINE#         245
  C:525AH         LINE#         246
  C:525AH         LINE#         247
  -------         ENDPROC       RAMCHECKPROCESS
  -------         PROC          _MEMORYSET
  X:02C5H         SYMBOL        pt
  D:0005H         SYMBOL        setval
  D:0003H         SYMBOL        length
  -------         DO            
  D:0007H         SYMBOL        i
  -------         ENDDO         
  C:6376H         LINE#         258
  C:637EH         LINE#         259
  C:637EH         LINE#         261
  C:6385H         LINE#         262
  C:6385H         LINE#         263
  C:6392H         LINE#         264
  C:639CH         LINE#         265
  C:639FH         LINE#         266
  -------         ENDPROC       _MEMORYSET
  -------         PROC          _MEMORYCOPY
  X:02DBH         SYMBOL        source
  D:0004H         SYMBOL        target
  D:0003H         SYMBOL        length
  -------         DO            
  D:0007H         SYMBOL        i
  -------         ENDDO         
BL51 BANKED LINKER/LOCATER V6.22                                                      06/21/2022  07:40:42  PAGE 80


  C:62E6H         LINE#         277
  C:62EEH         LINE#         278
  C:62EEH         LINE#         280
  C:62F5H         LINE#         281
  C:62F5H         LINE#         282
  C:6306H         LINE#         283
  C:630BH         LINE#         284
  C:6315H         LINE#         285
  C:6318H         LINE#         286
  -------         ENDPROC       _MEMORYCOPY
  -------         PROC          MCUINTOIDLE
  C:677CH         LINE#         295
  C:677CH         LINE#         296
  C:677CH         LINE#         297
  C:677FH         LINE#         298
  C:6782H         LINE#         299
  C:6783H         LINE#         300
  C:6784H         LINE#         301
  C:6785H         LINE#         302
  C:6786H         LINE#         303
  C:6787H         LINE#         304
  -------         ENDPROC       MCUINTOIDLE
  -------         PROC          MCUINTOPD
  C:6788H         LINE#         306
  C:6788H         LINE#         307
  C:6788H         LINE#         308
  C:678BH         LINE#         309
  C:678EH         LINE#         310
  C:678FH         LINE#         311
  C:6790H         LINE#         312
  C:6791H         LINE#         313
  C:6792H         LINE#         314
  C:6793H         LINE#         315
  -------         ENDPROC       MCUINTOPD
  -------         PROC          SYSTEMRESETPROCESS
  C:6460H         LINE#         324
  C:6460H         LINE#         325
  C:6460H         LINE#         326
  C:6471H         LINE#         328
  C:6471H         LINE#         329
  C:6473H         LINE#         330
  C:6475H         LINE#         331
  C:6477H         LINE#         332
  C:6479H         LINE#         333
  C:647BH         LINE#         335
  C:647DH         LINE#         336
  C:647FH         LINE#         337
  C:6481H         LINE#         339
  C:6484H         LINE#         340
  C:6484H         LINE#         341
  -------         ENDPROC       SYSTEMRESETPROCESS
  -------         ENDMOD        MCULIB

  -------         MODULE        MOSCTRL
  C:0000H         SYMBOL        _ICE_DUMMY_
  D:0080H         PUBLIC        P0
  D:0090H         PUBLIC        P1
BL51 BANKED LINKER/LOCATER V6.22                                                      06/21/2022  07:40:42  PAGE 81


  D:00A0H         PUBLIC        P2
  D:00B0H         PUBLIC        P3
  D:00C0H         PUBLIC        P4
  D:0080H         PUBLIC        P5
  C:5AAEH         PUBLIC        MosStatusCheck
  C:6349H         PUBLIC        MosCtrl
  B:002DH.5       PUBLIC        bCHGMOSBk
  B:002DH.6       PUBLIC        bDSGMOSBk
  -------         PROC          MOSSTATUSCHECK
  C:5AAEH         LINE#         20
  C:5AAEH         LINE#         21
  C:5AAEH         LINE#         22
  C:5AB0H         LINE#         23
  C:5AB2H         LINE#         25
  C:5AB8H         LINE#         26
  C:5AB8H         LINE#         27
  C:5ABAH         LINE#         28
  C:5ABAH         LINE#         30
  C:5ACCH         LINE#         31
  C:5ACCH         LINE#         32
  C:5ACEH         LINE#         33
  C:5ACEH         LINE#         35
  C:5AD1H         LINE#         36
  C:5AD1H         LINE#         37
  C:5ADDH         LINE#         38
  C:5ADDH         LINE#         39
  C:5ADFH         LINE#         40
  C:5ADFH         LINE#         41
  C:5ADFH         LINE#         43
  C:5AE2H         LINE#         44
  C:5AE2H         LINE#         45
  C:5AE5H         LINE#         46
  C:5AE5H         LINE#         47
  C:5AE7H         LINE#         48
  C:5AE7H         LINE#         49
  C:5AE7H         LINE#         51
  C:5AF0H         LINE#         52
  C:5AF0H         LINE#         53
  C:5AF2H         LINE#         54
  C:5AF2H         LINE#         56
  C:5AF5H         LINE#         57
  C:5AF5H         LINE#         58
  C:5AF7H         LINE#         59
  C:5AF7H         LINE#         60
  -------         ENDPROC       MOSSTATUSCHECK
  -------         PROC          MOSCTRL
  C:6349H         LINE#         70
  C:6349H         LINE#         71
  C:6349H         LINE#         72
  C:634CH         LINE#         74
  C:635CH         LINE#         75
  C:635CH         LINE#         76
  C:6360H         LINE#         77
  C:6364H         LINE#         79
  C:6375H         LINE#         80
  C:6375H         LINE#         81
  -------         ENDPROC       MOSCTRL
BL51 BANKED LINKER/LOCATER V6.22                                                      06/21/2022  07:40:42  PAGE 82


  -------         ENDMOD        MOSCTRL

  -------         MODULE        PORSELFTEST
  C:0000H         SYMBOL        _ICE_DUMMY_
  D:0080H         PUBLIC        P0
  C:588EH         PUBLIC        PorProtectOTC
  D:0090H         PUBLIC        P1
  C:592CH         PUBLIC        PorProtectOTD
  D:00A0H         PUBLIC        P2
  D:00B0H         PUBLIC        P3
  D:00C0H         PUBLIC        P4
  D:0080H         PUBLIC        P5
  C:58DDH         PUBLIC        PorProtectUTC
  C:597BH         PUBLIC        PorProtectUTD
  C:5C62H         PUBLIC        PorProtectOV
  C:5CAAH         PUBLIC        PorProtectUV
  X:03A1H         PUBLIC        ucPorSelfTestDelayCnt
  B:002EH.5       PUBLIC        bPorSelfTestFlg
  C:60C9H         PUBLIC        PorSelfTest
  -------         PROC          PORPROTECTOV
  C:5C62H         LINE#         20
  C:5C62H         LINE#         21
  C:5C62H         LINE#         22
  C:5C65H         LINE#         23
  C:5C65H         LINE#         24
  C:5C74H         LINE#         25
  C:5C74H         LINE#         26
  C:5C89H         LINE#         27
  C:5C89H         LINE#         28
  C:5C8BH         LINE#         29
  C:5C92H         LINE#         30
  C:5C92H         LINE#         31
  C:5C93H         LINE#         32
  C:5CA2H         LINE#         33
  C:5CA2H         LINE#         34
  C:5CA9H         LINE#         35
  C:5CA9H         LINE#         36
  C:5CA9H         LINE#         37
  -------         ENDPROC       PORPROTECTOV
  -------         PROC          PORPROTECTUV
  C:5CAAH         LINE#         46
  C:5CAAH         LINE#         47
  C:5CAAH         LINE#         48
  C:5CADH         LINE#         49
  C:5CADH         LINE#         50
  C:5CBCH         LINE#         51
  C:5CBCH         LINE#         52
  C:5CD1H         LINE#         53
  C:5CD1H         LINE#         54
  C:5CD3H         LINE#         55
  C:5CDAH         LINE#         56
  C:5CDAH         LINE#         57
  C:5CDBH         LINE#         58
  C:5CEAH         LINE#         59
  C:5CEAH         LINE#         60
  C:5CF1H         LINE#         61
  C:5CF1H         LINE#         62
BL51 BANKED LINKER/LOCATER V6.22                                                      06/21/2022  07:40:42  PAGE 83


  C:5CF1H         LINE#         63
  -------         ENDPROC       PORPROTECTUV
  -------         PROC          PORPROTECTOTC
  C:588EH         LINE#         72
  C:588EH         LINE#         73
  C:588EH         LINE#         74
  C:5891H         LINE#         75
  C:5891H         LINE#         76
  C:58A7H         LINE#         77
  C:58A7H         LINE#         78
  C:58BCH         LINE#         79
  C:58BCH         LINE#         80
  C:58BEH         LINE#         81
  C:58C5H         LINE#         82
  C:58C5H         LINE#         83
  C:58C6H         LINE#         84
  C:58D5H         LINE#         85
  C:58D5H         LINE#         86
  C:58DCH         LINE#         87
  C:58DCH         LINE#         88
  C:58DCH         LINE#         89
  -------         ENDPROC       PORPROTECTOTC
  -------         PROC          PORPROTECTUTC
  C:58DDH         LINE#         98
  C:58DDH         LINE#         99
  C:58DDH         LINE#         100
  C:58E0H         LINE#         101
  C:58E0H         LINE#         102
  C:58F6H         LINE#         103
  C:58F6H         LINE#         104
  C:590BH         LINE#         105
  C:590BH         LINE#         106
  C:590DH         LINE#         107
  C:5914H         LINE#         108
  C:5914H         LINE#         109
  C:5915H         LINE#         110
  C:5924H         LINE#         111
  C:5924H         LINE#         112
  C:592BH         LINE#         113
  C:592BH         LINE#         114
  C:592BH         LINE#         115
  -------         ENDPROC       PORPROTECTUTC
  -------         PROC          PORPROTECTOTD
  C:592CH         LINE#         124
  C:592CH         LINE#         125
  C:592CH         LINE#         126
  C:592FH         LINE#         127
  C:592FH         LINE#         128
  C:5945H         LINE#         129
  C:5945H         LINE#         130
  C:595AH         LINE#         131
  C:595AH         LINE#         132
  C:595CH         LINE#         133
  C:5963H         LINE#         134
  C:5963H         LINE#         135
  C:5964H         LINE#         136
  C:5973H         LINE#         137
BL51 BANKED LINKER/LOCATER V6.22                                                      06/21/2022  07:40:42  PAGE 84


  C:5973H         LINE#         138
  C:597AH         LINE#         139
  C:597AH         LINE#         140
  C:597AH         LINE#         141
  -------         ENDPROC       PORPROTECTOTD
  -------         PROC          PORPROTECTUTD
  C:597BH         LINE#         150
  C:597BH         LINE#         151
  C:597BH         LINE#         152
  C:597EH         LINE#         153
  C:597EH         LINE#         154
  C:5994H         LINE#         155
  C:5994H         LINE#         156
  C:59A9H         LINE#         157
  C:59A9H         LINE#         158
  C:59ABH         LINE#         159
  C:59B2H         LINE#         160
  C:59B2H         LINE#         161
  C:59B3H         LINE#         162
  C:59C2H         LINE#         163
  C:59C2H         LINE#         164
  C:59C9H         LINE#         165
  C:59C9H         LINE#         166
  C:59C9H         LINE#         167
  -------         ENDPROC       PORPROTECTUTD
  -------         PROC          PORSELFTEST
  C:60C9H         LINE#         176
  C:60C9H         LINE#         177
  C:60C9H         LINE#         178
  C:60CCH         LINE#         179
  C:60CCH         LINE#         180
  C:60CFH         LINE#         181
  C:60D2H         LINE#         182
  C:60D5H         LINE#         183
  C:60D8H         LINE#         185
  C:60DBH         LINE#         186
  C:60DEH         LINE#         187
  C:60E1H         LINE#         188
  C:60E4H         LINE#         190
  C:60EFH         LINE#         191
  C:60EFH         LINE#         192
  C:60F1H         LINE#         193
  C:60FDH         LINE#         194
  C:60FDH         LINE#         195
  C:60FFH         LINE#         196
  C:6100H         LINE#         198
  C:6100H         LINE#         199
  C:6103H         LINE#         200
  C:6103H         LINE#         201
  C:6103H         LINE#         202
  C:6103H         LINE#         203
  -------         ENDPROC       PORSELFTEST
  -------         ENDMOD        PORSELFTEST

  -------         MODULE        PROTECT
  C:0000H         SYMBOL        _ICE_DUMMY_
  D:0080H         PUBLIC        P0
BL51 BANKED LINKER/LOCATER V6.22                                                      06/21/2022  07:40:42  PAGE 85


  D:0090H         PUBLIC        P1
  X:0325H         PUBLIC        uiOCD1DelayCnt
  D:00A0H         PUBLIC        P2
  X:0327H         PUBLIC        uiOCD2DelayCnt
  D:00B0H         PUBLIC        P3
  D:00C0H         PUBLIC        P4
  D:0080H         PUBLIC        P5
  C:3DA1H         PUBLIC        ProtectOV
  C:3E5DH         PUBLIC        ProtectUV
  B:002DH.7       PUBLIC        bOVLock
  B:002EH.0       PUBLIC        bUVLock
  X:0329H         PUBLIC        uiOVDelayCnt
  X:032BH         PUBLIC        uiUVDelayCnt
  X:032DH         PUBLIC        uiOTCRDelayCnt
  X:032FH         PUBLIC        uiOTDRDelayCnt
  X:0331H         PUBLIC        uiUTCRDelayCnt
  X:0333H         PUBLIC        uiUTDRDelayCnt
  C:5541H         PUBLIC        ProtectOCC
  C:64ECH         PUBLIC        ProtectProcess
  C:3F19H         PUBLIC        ProtectOTC
  C:4091H         PUBLIC        ProtectOTD
  X:0335H         PUBLIC        uiOCCRcnt
  X:0337H         PUBLIC        uiOCCDelayCnt
  X:0339H         PUBLIC        uiOCDRcnt
  C:3FD5H         PUBLIC        ProtectUTC
  C:414DH         PUBLIC        ProtectUTD
  C:4F63H         PUBLIC        ProtectOCRecover
  X:033BH         PUBLIC        uiOTCDelayCnt
  X:033DH         PUBLIC        uiOTDDelayCnt
  X:033FH         PUBLIC        uiUTCDelayCnt
  X:0341H         PUBLIC        uiUTDDelayCnt
  C:559AH         PUBLIC        ProtectOCD1
  C:55F3H         PUBLIC        ProtectOCD2
  X:0343H         PUBLIC        uiOVRDelayCnt
  X:0345H         PUBLIC        uiUVRDelayCnt
  -------         PROC          PROTECTOV
  C:3DA1H         LINE#         39
  C:3DA1H         LINE#         40
  C:3DA1H         LINE#         41
  C:3DA4H         LINE#         42
  C:3DA4H         LINE#         43
  C:3DB3H         LINE#         44
  C:3DB3H         LINE#         45
  C:3DD4H         LINE#         46
  C:3DD4H         LINE#         47
  C:3DD6H         LINE#         48
  C:3DD8H         LINE#         49
  C:3DDFH         LINE#         50
  C:3DE5H         LINE#         51
  C:3DE5H         LINE#         52
  C:3DE6H         LINE#         53
  C:3DF5H         LINE#         54
  C:3DF5H         LINE#         55
  C:3DFCH         LINE#         56
  C:3DFCH         LINE#         57
  C:3DFDH         LINE#         58
  C:3E00H         LINE#         59
BL51 BANKED LINKER/LOCATER V6.22                                                      06/21/2022  07:40:42  PAGE 86


  C:3E00H         LINE#         60
  C:3E0FH         LINE#         61
  C:3E0FH         LINE#         62
  C:3E2DH         LINE#         63
  C:3E2DH         LINE#         64
  C:3E30H         LINE#         65
  C:3E30H         LINE#         66
  C:3E32H         LINE#         67
  C:3E34H         LINE#         68
  C:3E36H         LINE#         70
  C:3E36H         LINE#         71
  C:3E38H         LINE#         72
  C:3E38H         LINE#         73
  C:3E3FH         LINE#         74
  C:3E45H         LINE#         75
  C:3E45H         LINE#         76
  C:3E46H         LINE#         77
  C:3E55H         LINE#         78
  C:3E55H         LINE#         79
  C:3E5CH         LINE#         80
  C:3E5CH         LINE#         81
  C:3E5CH         LINE#         82
  -------         ENDPROC       PROTECTOV
  -------         PROC          PROTECTUV
  C:3E5DH         LINE#         90
  C:3E5DH         LINE#         91
  C:3E5DH         LINE#         92
  C:3E60H         LINE#         93
  C:3E60H         LINE#         94
  C:3E6FH         LINE#         95
  C:3E6FH         LINE#         96
  C:3E90H         LINE#         97
  C:3E90H         LINE#         98
  C:3E92H         LINE#         99
  C:3E94H         LINE#         100
  C:3E9BH         LINE#         101
  C:3EA1H         LINE#         102
  C:3EA1H         LINE#         103
  C:3EA2H         LINE#         104
  C:3EB1H         LINE#         105
  C:3EB1H         LINE#         106
  C:3EB8H         LINE#         107
  C:3EB8H         LINE#         108
  C:3EB9H         LINE#         109
  C:3EBCH         LINE#         110
  C:3EBCH         LINE#         111
  C:3ECBH         LINE#         112
  C:3ECBH         LINE#         113
  C:3EE9H         LINE#         114
  C:3EE9H         LINE#         115
  C:3EECH         LINE#         116
  C:3EECH         LINE#         117
  C:3EEEH         LINE#         118
  C:3EF0H         LINE#         119
  C:3EF2H         LINE#         121
  C:3EF2H         LINE#         122
  C:3EF4H         LINE#         123
BL51 BANKED LINKER/LOCATER V6.22                                                      06/21/2022  07:40:42  PAGE 87


  C:3EF4H         LINE#         124
  C:3EFBH         LINE#         125
  C:3F01H         LINE#         126
  C:3F01H         LINE#         127
  C:3F02H         LINE#         128
  C:3F11H         LINE#         129
  C:3F11H         LINE#         130
  C:3F18H         LINE#         131
  C:3F18H         LINE#         132
  C:3F18H         LINE#         133
  -------         ENDPROC       PROTECTUV
  -------         PROC          PROTECTOTC
  C:3F19H         LINE#         141
  C:3F19H         LINE#         142
  C:3F19H         LINE#         143
  C:3F1CH         LINE#         144
  C:3F1CH         LINE#         145
  C:3F32H         LINE#         146
  C:3F32H         LINE#         147
  C:3F53H         LINE#         148
  C:3F53H         LINE#         149
  C:3F55H         LINE#         150
  C:3F5CH         LINE#         151
  C:3F62H         LINE#         152
  C:3F62H         LINE#         153
  C:3F63H         LINE#         154
  C:3F72H         LINE#         155
  C:3F72H         LINE#         156
  C:3F79H         LINE#         157
  C:3F79H         LINE#         158
  C:3F7AH         LINE#         160
  C:3F7AH         LINE#         161
  C:3F90H         LINE#         162
  C:3F90H         LINE#         163
  C:3FAEH         LINE#         164
  C:3FAEH         LINE#         165
  C:3FB0H         LINE#         166
  C:3FB7H         LINE#         167
  C:3FBDH         LINE#         168
  C:3FBDH         LINE#         169
  C:3FBEH         LINE#         170
  C:3FCDH         LINE#         171
  C:3FCDH         LINE#         172
  C:3FD4H         LINE#         173
  C:3FD4H         LINE#         174
  C:3FD4H         LINE#         175
  -------         ENDPROC       PROTECTOTC
  -------         PROC          PROTECTUTC
  C:3FD5H         LINE#         184
  C:3FD5H         LINE#         185
  C:3FD5H         LINE#         186
  C:3FD8H         LINE#         187
  C:3FD8H         LINE#         188
  C:3FEEH         LINE#         189
  C:3FEEH         LINE#         190
  C:400FH         LINE#         191
  C:400FH         LINE#         192
BL51 BANKED LINKER/LOCATER V6.22                                                      06/21/2022  07:40:42  PAGE 88


  C:4011H         LINE#         193
  C:4018H         LINE#         194
  C:401EH         LINE#         195
  C:401EH         LINE#         196
  C:401FH         LINE#         197
  C:402EH         LINE#         198
  C:402EH         LINE#         199
  C:4035H         LINE#         200
  C:4035H         LINE#         201
  C:4036H         LINE#         203
  C:4036H         LINE#         204
  C:404CH         LINE#         205
  C:404CH         LINE#         206
  C:406AH         LINE#         207
  C:406AH         LINE#         208
  C:406CH         LINE#         209
  C:4073H         LINE#         210
  C:4079H         LINE#         211
  C:4079H         LINE#         212
  C:407AH         LINE#         213
  C:4089H         LINE#         214
  C:4089H         LINE#         215
  C:4090H         LINE#         216
  C:4090H         LINE#         217
  C:4090H         LINE#         218
  -------         ENDPROC       PROTECTUTC
  -------         PROC          PROTECTOTD
  C:4091H         LINE#         227
  C:4091H         LINE#         228
  C:4091H         LINE#         229
  C:4094H         LINE#         230
  C:4094H         LINE#         231
  C:40AAH         LINE#         232
  C:40AAH         LINE#         233
  C:40CBH         LINE#         234
  C:40CBH         LINE#         235
  C:40CDH         LINE#         236
  C:40D4H         LINE#         237
  C:40DAH         LINE#         238
  C:40DAH         LINE#         239
  C:40DBH         LINE#         240
  C:40EAH         LINE#         241
  C:40EAH         LINE#         242
  C:40F1H         LINE#         243
  C:40F1H         LINE#         244
  C:40F2H         LINE#         246
  C:40F2H         LINE#         247
  C:4108H         LINE#         248
  C:4108H         LINE#         249
  C:4126H         LINE#         250
  C:4126H         LINE#         251
  C:4128H         LINE#         252
  C:412FH         LINE#         253
  C:4135H         LINE#         254
  C:4135H         LINE#         255
  C:4136H         LINE#         256
  C:4145H         LINE#         257
BL51 BANKED LINKER/LOCATER V6.22                                                      06/21/2022  07:40:42  PAGE 89


  C:4145H         LINE#         258
  C:414CH         LINE#         259
  C:414CH         LINE#         260
  C:414CH         LINE#         261
  -------         ENDPROC       PROTECTOTD
  -------         PROC          PROTECTUTD
  C:414DH         LINE#         270
  C:414DH         LINE#         271
  C:414DH         LINE#         272
  C:4150H         LINE#         273
  C:4150H         LINE#         274
  C:4166H         LINE#         275
  C:4166H         LINE#         276
  C:4187H         LINE#         277
  C:4187H         LINE#         278
  C:4189H         LINE#         279
  C:4190H         LINE#         280
  C:4196H         LINE#         281
  C:4196H         LINE#         282
  C:4197H         LINE#         283
  C:41A6H         LINE#         284
  C:41A6H         LINE#         285
  C:41ADH         LINE#         286
  C:41ADH         LINE#         287
  C:41AEH         LINE#         289
  C:41AEH         LINE#         290
  C:41C4H         LINE#         291
  C:41C4H         LINE#         292
  C:41E2H         LINE#         293
  C:41E2H         LINE#         294
  C:41E4H         LINE#         295
  C:41EBH         LINE#         296
  C:41F1H         LINE#         297
  C:41F1H         LINE#         298
  C:41F2H         LINE#         299
  C:4201H         LINE#         300
  C:4201H         LINE#         301
  C:4208H         LINE#         302
  C:4208H         LINE#         303
  C:4208H         LINE#         304
  -------         ENDPROC       PROTECTUTD
  -------         PROC          PROTECTOCC
  C:5541H         LINE#         314
  C:5541H         LINE#         315
  C:5541H         LINE#         316
  C:5544H         LINE#         317
  C:5544H         LINE#         318
  C:5556H         LINE#         319
  C:5556H         LINE#         320
  C:5574H         LINE#         321
  C:5574H         LINE#         322
  C:5576H         LINE#         323
  C:5578H         LINE#         324
  C:557FH         LINE#         325
  C:557FH         LINE#         326
  C:5580H         LINE#         327
  C:5583H         LINE#         328
BL51 BANKED LINKER/LOCATER V6.22                                                      06/21/2022  07:40:42  PAGE 90


  C:5583H         LINE#         329
  C:5592H         LINE#         330
  C:5592H         LINE#         331
  C:5599H         LINE#         332
  C:5599H         LINE#         333
  C:5599H         LINE#         334
  C:5599H         LINE#         335
  -------         ENDPROC       PROTECTOCC
  -------         PROC          PROTECTOCD1
  C:559AH         LINE#         344
  C:559AH         LINE#         345
  C:559AH         LINE#         346
  C:559DH         LINE#         347
  C:559DH         LINE#         348
  C:55AFH         LINE#         349
  C:55AFH         LINE#         350
  C:55CDH         LINE#         351
  C:55CDH         LINE#         352
  C:55D4H         LINE#         353
  C:55D6H         LINE#         354
  C:55D8H         LINE#         355
  C:55D8H         LINE#         356
  C:55D9H         LINE#         357
  C:55DCH         LINE#         358
  C:55DCH         LINE#         359
  C:55EBH         LINE#         360
  C:55EBH         LINE#         361
  C:55F2H         LINE#         362
  C:55F2H         LINE#         363
  C:55F2H         LINE#         364
  C:55F2H         LINE#         365
  -------         ENDPROC       PROTECTOCD1
  -------         PROC          PROTECTOCD2
  C:55F3H         LINE#         374
  C:55F3H         LINE#         375
  C:55F3H         LINE#         376
  C:55F6H         LINE#         377
  C:55F6H         LINE#         378
  C:5608H         LINE#         379
  C:5608H         LINE#         380
  C:5626H         LINE#         381
  C:5626H         LINE#         382
  C:562DH         LINE#         383
  C:562FH         LINE#         384
  C:5631H         LINE#         385
  C:5631H         LINE#         386
  C:5632H         LINE#         387
  C:5635H         LINE#         388
  C:5635H         LINE#         389
  C:5644H         LINE#         390
  C:5644H         LINE#         391
  C:564BH         LINE#         392
  C:564BH         LINE#         393
  C:564BH         LINE#         394
  C:564BH         LINE#         395
  -------         ENDPROC       PROTECTOCD2
  -------         PROC          PROTECTPROCESS
BL51 BANKED LINKER/LOCATER V6.22                                                      06/21/2022  07:40:42  PAGE 91


  C:64ECH         LINE#         404
  C:64ECH         LINE#         405
  C:64ECH         LINE#         406
  C:64EFH         LINE#         407
  C:64EFH         LINE#         408
  C:64F2H         LINE#         409
  C:64F5H         LINE#         411
  C:64F8H         LINE#         412
  C:64FBH         LINE#         413
  C:64FEH         LINE#         414
  C:6501H         LINE#         416
  C:6504H         LINE#         417
  C:6507H         LINE#         418
  C:650AH         LINE#         419
  C:650AH         LINE#         420
  -------         ENDPROC       PROTECTPROCESS
  -------         PROC          PROTECTOCRECOVER
  C:4F63H         LINE#         429
  C:4F63H         LINE#         430
  C:4F63H         LINE#         431
  C:4F66H         LINE#         432
  C:4F66H         LINE#         433
  C:4F6FH         LINE#         434
  C:4F6FH         LINE#         435
  C:4F8DH         LINE#         436
  C:4F8DH         LINE#         437
  C:4F92H         LINE#         438
  C:4F98H         LINE#         439
  C:4F9AH         LINE#         440
  C:4F9CH         LINE#         441
  C:4F9EH         LINE#         442
  C:4FA0H         LINE#         443
  C:4FA3H         LINE#         444
  C:4FA3H         LINE#         445
  C:4FA5H         LINE#         446
  C:4FA8H         LINE#         447
  C:4FA8H         LINE#         448
  C:4FA8H         LINE#         449
  C:4FA8H         LINE#         451
  C:4FABH         LINE#         452
  C:4FABH         LINE#         453
  C:4FC9H         LINE#         454
  C:4FC9H         LINE#         455
  C:4FD0H         LINE#         456
  C:4FD2H         LINE#         457
  C:4FD6H         LINE#         458
  C:4FD8H         LINE#         459
  C:4FD8H         LINE#         460
  C:4FD8H         LINE#         461
  C:4FD8H         LINE#         462
  -------         ENDPROC       PROTECTOCRECOVER
  -------         ENDMOD        PROTECT

  -------         MODULE        RTC
  C:0000H         SYMBOL        _ICE_DUMMY_
  D:0080H         PUBLIC        P0
  D:0090H         PUBLIC        P1
BL51 BANKED LINKER/LOCATER V6.22                                                      06/21/2022  07:40:42  PAGE 92


  C:6546H         PUBLIC        RTCTwiCheck
  D:00A0H         PUBLIC        P2
  D:00B0H         PUBLIC        P3
  D:00C0H         PUBLIC        P4
  D:0080H         PUBLIC        P5
  C:49C5H         PUBLIC        _RTCInitTime
  B:002EH.1       PUBLIC        bRTCTwiRWErr
  C:548CH         PUBLIC        _RTCRead
  C:476AH         PUBLIC        _RTCModifyTime
  X:0377H         PUBLIC        ucRTCTwiRWErrDelayCnt
  X:0378H         PUBLIC        RTC
  B:002EH.2       PUBLIC        bRTCErr
  C:5431H         PUBLIC        _RTCWrite
  C:2B88H         PUBLIC        _RTCReadTime
  -------         PROC          RTCTWICHECK
  C:6546H         LINE#         23
  C:6546H         LINE#         24
  C:6546H         LINE#         25
  C:6549H         LINE#         26
  C:6549H         LINE#         27
  C:654CH         LINE#         28
  C:654CH         LINE#         29
  C:6557H         LINE#         30
  C:6557H         LINE#         31
  C:6559H         LINE#         32
  C:655CH         LINE#         33
  C:655CH         LINE#         34
  C:655DH         LINE#         36
  C:655DH         LINE#         37
  C:6562H         LINE#         38
  C:6562H         LINE#         39
  C:6562H         LINE#         40
  -------         ENDPROC       RTCTWICHECK
  -------         PROC          _RTCWRITE
  X:02F0H         SYMBOL        WrAddr
  X:02F1H         SYMBOL        Length
  X:02F2H         SYMBOL        WrBuf
  -------         DO            
  B:0029H.0       SYMBOL        Result
  X:02F4H         SYMBOL        i
  -------         ENDDO         
  C:5431H         LINE#         49
  C:543FH         LINE#         50
  C:543FH         LINE#         51
  C:5441H         LINE#         54
  C:5444H         LINE#         55
  C:5444H         LINE#         56
  C:5447H         LINE#         57
  C:5447H         LINE#         58
  C:546FH         LINE#         59
  C:546FH         LINE#         60
  C:5471H         LINE#         61
  C:5473H         LINE#         62
  C:5473H         LINE#         63
  C:5478H         LINE#         64
  C:5484H         LINE#         65
  C:5484H         LINE#         66
BL51 BANKED LINKER/LOCATER V6.22                                                      06/21/2022  07:40:42  PAGE 93


  C:5489H         LINE#         68
  C:548BH         LINE#         69
  -------         ENDPROC       _RTCWRITE
  -------         PROC          _RTCREAD
  X:02E6H         SYMBOL        RdAddr
  X:02E7H         SYMBOL        Length
  X:02E8H         SYMBOL        RdBuf
  -------         DO            
  B:0028H.7       SYMBOL        Result
  X:02EAH         SYMBOL        i
  -------         ENDDO         
  C:548CH         LINE#         78
  C:549AH         LINE#         79
  C:549AH         LINE#         80
  C:549CH         LINE#         83
  C:549FH         LINE#         84
  C:549FH         LINE#         85
  C:54A2H         LINE#         86
  C:54A2H         LINE#         87
  C:54CAH         LINE#         88
  C:54CAH         LINE#         89
  C:54CCH         LINE#         90
  C:54CEH         LINE#         91
  C:54CEH         LINE#         92
  C:54D3H         LINE#         93
  C:54DFH         LINE#         94
  C:54DFH         LINE#         95
  C:54E4H         LINE#         97
  C:54E6H         LINE#         98
  -------         ENDPROC       _RTCREAD
  -------         PROC          _RTCREADTIME
  X:02DBH         SYMBOL        RtcRdVal
  -------         DO            
  X:02DDH         SYMBOL        rtcbuf
  B:0028H.6       SYMBOL        Result
  -------         ENDDO         
  C:2B88H         LINE#         106
  C:2B90H         LINE#         107
  C:2B90H         LINE#         109
  C:2B92H         LINE#         111
  C:2BA2H         LINE#         112
  C:2BA2H         LINE#         113
  C:2BACH         LINE#         114
  C:2BACH         LINE#         115
  C:2C59H         LINE#         123
  C:2C59H         LINE#         124
  C:2C6AH         LINE#         125
  C:2C74H         LINE#         126
  C:2C85H         LINE#         127
  C:2C91H         LINE#         128
  C:2CA4H         LINE#         129
  C:2CB2H         LINE#         130
  C:2CC5H         LINE#         132
  C:2CCEH         LINE#         133
  C:2CD0H         LINE#         135
  C:2CD0H         LINE#         136
  C:2CE3H         LINE#         137
BL51 BANKED LINKER/LOCATER V6.22                                                      06/21/2022  07:40:42  PAGE 94


  C:2CEDH         LINE#         138
  C:2CFAH         LINE#         139
  C:2D06H         LINE#         140
  C:2D16H         LINE#         141
  C:2D26H         LINE#         142
  C:2D36H         LINE#         144
  C:2D38H         LINE#         145
  C:2D38H         LINE#         146
  C:2D3AH         LINE#         148
  C:2D3AH         LINE#         149
  C:2D47H         LINE#         150
  C:2D47H         LINE#         151
  C:2D47H         LINE#         153
  C:2D49H         LINE#         154
  -------         ENDPROC       _RTCREADTIME
  -------         PROC          _RTCMODIFYTIME
  X:02E6H         SYMBOL        RtcMdyVal
  -------         DO            
  B:0028H.7       SYMBOL        Result
  X:02E8H         SYMBOL        rtcdata
  X:02E9H         SYMBOL        rtctemp
  -------         ENDDO         
  C:476AH         LINE#         163
  C:4772H         LINE#         164
  C:4772H         LINE#         165
  C:4774H         LINE#         169
  C:4778H         LINE#         170
  C:4785H         LINE#         172
  C:4796H         LINE#         173
  C:47A0H         LINE#         174
  C:47B5H         LINE#         175
  C:47C1H         LINE#         176
  C:47D5H         LINE#         177
  C:47E3H         LINE#         178
  C:47F6H         LINE#         180
  C:4803H         LINE#         182
  C:4805H         LINE#         183
  -------         ENDPROC       _RTCMODIFYTIME
  -------         PROC          _RTCINITTIME
  X:02B9H         SYMBOL        RtcInitVal
  -------         DO            
  B:0028H.5       SYMBOL        Result
  X:02BBH         SYMBOL        rtcbuf
  D:0007H         SYMBOL        i
  X:02C4H         SYMBOL        checksum
  -------         ENDDO         
  C:49C5H         LINE#         192
  C:49CDH         LINE#         193
  C:49CDH         LINE#         194
  C:49CFH         LINE#         197
  C:49D4H         LINE#         199
  C:49DEH         LINE#         201
  C:49EBH         LINE#         202
  C:49EDH         LINE#         203
  C:49EDH         LINE#         204
  C:49FFH         LINE#         205
  C:4A04H         LINE#         207
BL51 BANKED LINKER/LOCATER V6.22                                                      06/21/2022  07:40:42  PAGE 95


  C:4A16H         LINE#         208
  C:4A16H         LINE#         209
  C:4A1BH         LINE#         210
  C:4A1DH         LINE#         211
  C:4A21H         LINE#         212
  C:4A25H         LINE#         213
  C:4A29H         LINE#         214
  C:4A2DH         LINE#         215
  C:4A31H         LINE#         216
  C:4A31H         LINE#         218
  C:4A42H         LINE#         219
  C:4A4FH         LINE#         221
  C:4A51H         LINE#         222
  -------         ENDPROC       _RTCINITTIME
  -------         ENDMOD        RTC

  -------         MODULE        TWI
  C:0000H         SYMBOL        _ICE_DUMMY_
  D:0080H         PUBLIC        P0
  D:0090H         PUBLIC        P1
  D:00A0H         PUBLIC        P2
  D:00B0H         PUBLIC        P3
  D:00C0H         PUBLIC        P4
  D:0080H         PUBLIC        P5
  D:008AH         PUBLIC        TWIBR
  D:00C6H         PUBLIC        TWICR
  D:0089H         PUBLIC        TWTFREE
  C:29B0H         PUBLIC        _TwiRead
  D:00B1H         PUBLIC        RSTSTAT
  C:6563H         PUBLIC        _CRC8cal
  D:00E6H         PUBLIC        TWITOUT
  C:3324H         PUBLIC        _TwiWrite
  C:6104H         PUBLIC        _TwiInit
  D:008DH         PUBLIC        TWIDAT
  D:00C8H         PUBLIC        TWICON
  D:00D1H         PUBLIC        TWISTA
  C:63C7H         PUBLIC        _TWICheckStatus
  C:3962H         PUBLIC        CRC8Table
  -------         PROC          _CRC8CAL
  D:0001H         SYMBOL        p
  D:0005H         SYMBOL        counter
  -------         DO            
  D:0007H         SYMBOL        crc8
  -------         ENDDO         
  C:6563H         LINE#         37
  C:6563H         LINE#         38
  C:6563H         LINE#         39
  C:6565H         LINE#         41
  C:656BH         LINE#         42
  C:656BH         LINE#         43
  C:6574H         LINE#         44
  C:657BH         LINE#         45
  C:657EH         LINE#         46
  C:657EH         LINE#         47
  -------         ENDPROC       _CRC8CAL
  -------         PROC          _TWICHECKSTATUS
  D:0007H         SYMBOL        Status
BL51 BANKED LINKER/LOCATER V6.22                                                      06/21/2022  07:40:42  PAGE 96


  -------         DO            
  B:0029H.2       SYMBOL        Result
  D:0004H         SYMBOL        timeoutcount
  -------         ENDDO         
  C:63C7H         LINE#         58
  C:63C7H         LINE#         59
  C:63C7H         LINE#         60
  C:63C9H         LINE#         61
  C:63CDH         LINE#         63
  C:63D2H         LINE#         64
  C:63D2H         LINE#         65
  C:63D5H         LINE#         66
  C:63D9H         LINE#         67
  C:63D9H         LINE#         68
  C:63DEH         LINE#         69
  C:63E0H         LINE#         71
  C:63E0H         LINE#         72
  C:63E0H         LINE#         73
  C:63E0H         LINE#         74
  C:63E2H         LINE#         75
  C:63E9H         LINE#         76
  C:63E9H         LINE#         77
  C:63EBH         LINE#         78
  C:63EBH         LINE#         80
  C:63EDH         LINE#         81
  -------         ENDPROC       _TWICHECKSTATUS
  -------         PROC          _TWIWRITE
  X:02F5H         SYMBOL        SlaveID
  X:02F6H         SYMBOL        WrAddr
  X:02F8H         SYMBOL        AddrType
  X:02F9H         SYMBOL        Length
  X:02FAH         SYMBOL        CrcFlg
  X:02FBH         SYMBOL        WrBuf
  -------         DO            
  D:0006H         SYMBOL        i
  X:02FDH         SYMBOL        TempBuf
  B:0029H.1       SYMBOL        Result
  X:0301H         SYMBOL        timeoutcount
  C:3445H         SYMBOL        WrErr
  -------         ENDDO         
  C:3324H         LINE#         97
  C:3334H         LINE#         98
  C:3334H         LINE#         101
  C:3336H         LINE#         102
  C:3340H         LINE#         104
  C:3345H         LINE#         105
  C:3348H         LINE#         106
  C:3358H         LINE#         107
  C:3368H         LINE#         109
  C:3374H         LINE#         110
  C:3374H         LINE#         111
  C:337DH         LINE#         112
  C:3380H         LINE#         113
  C:338EH         LINE#         114
  C:338EH         LINE#         115
  C:3390H         LINE#         116
  C:3393H         LINE#         117
BL51 BANKED LINKER/LOCATER V6.22                                                      06/21/2022  07:40:42  PAGE 97


  C:3393H         LINE#         119
  C:3399H         LINE#         120
  C:339CH         LINE#         121
  C:33A3H         LINE#         122
  C:33A3H         LINE#         123
  C:33A5H         LINE#         124
  C:33A8H         LINE#         125
  C:33A8H         LINE#         127
  C:33AFH         LINE#         128
  C:33AFH         LINE#         129
  C:33B5H         LINE#         130
  C:33B8H         LINE#         131
  C:33BFH         LINE#         132
  C:33BFH         LINE#         133
  C:33C1H         LINE#         134
  C:33C4H         LINE#         135
  C:33C4H         LINE#         136
  C:33C4H         LINE#         138
  C:33CCH         LINE#         139
  C:33CFH         LINE#         140
  C:33D6H         LINE#         141
  C:33D6H         LINE#         142
  C:33D8H         LINE#         143
  C:33DAH         LINE#         144
  C:33DAH         LINE#         146
  C:33E2H         LINE#         147
  C:33E2H         LINE#         148
  C:33EEH         LINE#         149
  C:33F1H         LINE#         150
  C:33F8H         LINE#         151
  C:33F8H         LINE#         152
  C:33FAH         LINE#         153
  C:33FCH         LINE#         154
  C:33FCH         LINE#         156
  C:3402H         LINE#         157
  C:3405H         LINE#         158
  C:340CH         LINE#         159
  C:340CH         LINE#         160
  C:340EH         LINE#         161
  C:3410H         LINE#         162
  C:3410H         LINE#         163
  C:3410H         LINE#         165
  C:3410H         LINE#         166
  C:341CH         LINE#         167
  C:341CH         LINE#         168
  C:342AH         LINE#         169
  C:342DH         LINE#         170
  C:3434H         LINE#         171
  C:3434H         LINE#         172
  C:3436H         LINE#         173
  C:3438H         LINE#         174
  C:3438H         LINE#         175
  C:3442H         LINE#         176
  C:3445H         LINE#         177
  C:3445H         LINE#         178
  C:3445H         LINE#         179
  C:3448H         LINE#         180
BL51 BANKED LINKER/LOCATER V6.22                                                      06/21/2022  07:40:42  PAGE 98


  C:344DH         LINE#         181
  C:344DH         LINE#         182
  C:3450H         LINE#         183
  C:345AH         LINE#         184
  C:345AH         LINE#         185
  C:3464H         LINE#         186
  C:3466H         LINE#         188
  C:3466H         LINE#         189
  C:3466H         LINE#         190
  C:3466H         LINE#         191
  C:3468H         LINE#         192
  C:3468H         LINE#         194
  C:346AH         LINE#         195
  -------         ENDPROC       _TWIWRITE
  -------         PROC          _TWIREAD
  D:0002H         SYMBOL        SlaveID
  X:02ECH         SYMBOL        RdAddr
  D:0003H         SYMBOL        AddrType
  X:02EFH         SYMBOL        Length
  X:02F0H         SYMBOL        CrcFlg
  X:02F1H         SYMBOL        RdBuf
  -------         DO            
  B:0029H.0       SYMBOL        Result
  X:02F3H         SYMBOL        i
  X:02F4H         SYMBOL        TempBuf
  X:0322H         SYMBOL        RdCrc
  X:0323H         SYMBOL        timeoutcount
  C:2B62H         SYMBOL        RdErr
  -------         ENDDO         
  C:29B0H         LINE#         209
  C:29BAH         LINE#         210
  C:29BAH         LINE#         211
  C:29BCH         LINE#         214
  C:29C1H         LINE#         215
  C:29C9H         LINE#         217
  C:29CEH         LINE#         218
  C:29D1H         LINE#         219
  C:29DAH         LINE#         220
  C:29DFH         LINE#         222
  C:29E8H         LINE#         223
  C:29E8H         LINE#         224
  C:29F1H         LINE#         225
  C:29F4H         LINE#         226
  C:2A02H         LINE#         227
  C:2A02H         LINE#         228
  C:2A04H         LINE#         229
  C:2A07H         LINE#         230
  C:2A07H         LINE#         232
  C:2A09H         LINE#         233
  C:2A0CH         LINE#         234
  C:2A13H         LINE#         235
  C:2A13H         LINE#         236
  C:2A15H         LINE#         237
  C:2A18H         LINE#         238
  C:2A18H         LINE#         240
  C:2A1CH         LINE#         241
  C:2A1CH         LINE#         242
BL51 BANKED LINKER/LOCATER V6.22                                                      06/21/2022  07:40:42  PAGE 99


  C:2A22H         LINE#         243
  C:2A25H         LINE#         244
  C:2A2CH         LINE#         245
  C:2A2CH         LINE#         246
  C:2A2EH         LINE#         247
  C:2A31H         LINE#         248
  C:2A31H         LINE#         249
  C:2A31H         LINE#         251
  C:2A39H         LINE#         252
  C:2A3CH         LINE#         253
  C:2A43H         LINE#         254
  C:2A43H         LINE#         255
  C:2A45H         LINE#         256
  C:2A48H         LINE#         257
  C:2A48H         LINE#         259
  C:2A4CH         LINE#         260
  C:2A4CH         LINE#         261
  C:2A52H         LINE#         262
  C:2A55H         LINE#         263
  C:2A5CH         LINE#         264
  C:2A5CH         LINE#         265
  C:2A5EH         LINE#         266
  C:2A61H         LINE#         267
  C:2A61H         LINE#         268
  C:2A61H         LINE#         270
  C:2A64H         LINE#         271
  C:2A72H         LINE#         272
  C:2A72H         LINE#         273
  C:2A74H         LINE#         274
  C:2A77H         LINE#         275
  C:2A77H         LINE#         277
  C:2A7CH         LINE#         278
  C:2A7FH         LINE#         279
  C:2A86H         LINE#         280
  C:2A86H         LINE#         281
  C:2A88H         LINE#         282
  C:2A8BH         LINE#         283
  C:2A8BH         LINE#         285
  C:2A9EH         LINE#         286
  C:2A9EH         LINE#         287
  C:2AA4H         LINE#         288
  C:2AA4H         LINE#         289
  C:2AA9H         LINE#         290
  C:2AA9H         LINE#         291
  C:2AACH         LINE#         292
  C:2AB1H         LINE#         293
  C:2AB3H         LINE#         295
  C:2AB3H         LINE#         296
  C:2AB6H         LINE#         297
  C:2ABBH         LINE#         298
  C:2ABBH         LINE#         299
  C:2AC9H         LINE#         300
  C:2AD3H         LINE#         301
  C:2AD5H         LINE#         303
  C:2AD5H         LINE#         304
  C:2AD8H         LINE#         305
  C:2ADDH         LINE#         306
BL51 BANKED LINKER/LOCATER V6.22                                                      06/21/2022  07:40:42  PAGE 100


  C:2AEDH         LINE#         307
  C:2AEDH         LINE#         308
  C:2AF5H         LINE#         310
  C:2AFDH         LINE#         311
  C:2AFDH         LINE#         312
  C:2B00H         LINE#         313
  C:2B05H         LINE#         314
  C:2B0BH         LINE#         315
  C:2B22H         LINE#         316
  C:2B22H         LINE#         317
  C:2B35H         LINE#         318
  C:2B35H         LINE#         319
  C:2B4EH         LINE#         320
  C:2B58H         LINE#         321
  C:2B60H         LINE#         322
  C:2B60H         LINE#         324
  C:2B60H         LINE#         325
  C:2B62H         LINE#         326
  C:2B62H         LINE#         327
  C:2B62H         LINE#         328
  C:2B62H         LINE#         329
  C:2B62H         LINE#         330
  C:2B65H         LINE#         331
  C:2B6AH         LINE#         332
  C:2B6AH         LINE#         333
  C:2B6DH         LINE#         334
  C:2B77H         LINE#         335
  C:2B77H         LINE#         336
  C:2B81H         LINE#         337
  C:2B83H         LINE#         339
  C:2B83H         LINE#         340
  C:2B83H         LINE#         341
  C:2B83H         LINE#         342
  C:2B85H         LINE#         343
  C:2B85H         LINE#         345
  C:2B87H         LINE#         346
  -------         ENDPROC       _TWIREAD
  -------         PROC          _TWIINIT
  D:0007H         SYMBOL        FreqKHz
  C:6104H         LINE#         355
  C:6104H         LINE#         356
  C:6104H         LINE#         357
  C:6107H         LINE#         358
  C:610AH         LINE#         359
  C:6130H         LINE#         360
  C:6133H         LINE#         361
  C:6136H         LINE#         362
  C:6139H         LINE#         363
  C:613CH         LINE#         364
  -------         ENDPROC       _TWIINIT
  -------         ENDMOD        TWI

  -------         MODULE        UART
  C:0000H         SYMBOL        _ICE_DUMMY_
  D:0080H         PUBLIC        P0
  D:0090H         PUBLIC        P1
  D:00A0H         PUBLIC        P2
BL51 BANKED LINKER/LOCATER V6.22                                                      06/21/2022  07:40:42  PAGE 101


  D:00B0H         PUBLIC        P3
  D:00C4H         PUBLIC        UART0CR
  D:00C0H         PUBLIC        P4
  C:4934H         PUBLIC        _UART0Init
  D:009DH         PUBLIC        SBRTH
  D:0080H         PUBLIC        P5
  D:009CH         PUBLIC        SBRTL
  B:0098H.0       PUBLIC        RI
  B:0098H.1       PUBLIC        TI
  C:57EEH         PUBLIC        InterruptUart0
  D:0099H         PUBLIC        SBUF
  D:0087H         PUBLIC        PCON
  D:0098H         PUBLIC        SCON
  D:0086H         PUBLIC        INSCON
  D:009BH         PUBLIC        SADEN
  D:009AH         PUBLIC        SADDR
  D:009EH         PUBLIC        SFINE
  -------         PROC          _UART0INIT
  X:02B9H         SYMBOL        Bps
  -------         DO            
  D:0004H         SYMBOL        TempVal
  -------         ENDDO         
  C:4934H         LINE#         19
  C:493CH         LINE#         20
  C:493CH         LINE#         23
  C:493FH         LINE#         24
  C:4942H         LINE#         25
  C:4945H         LINE#         26
  C:495FH         LINE#         27
  C:4961H         LINE#         28
  C:4963H         LINE#         29
  C:49BBH         LINE#         30
  C:49BEH         LINE#         31
  C:49C1H         LINE#         32
  C:49C4H         LINE#         33
  -------         ENDPROC       _UART0INIT
  -------         PROC          INTERRUPTUART0
  -------         DO            
  D:0007H         SYMBOL        RxData
  -------         ENDDO         
  C:57EEH         LINE#         44
  C:580BH         LINE#         48
  C:580DH         LINE#         49
  C:5810H         LINE#         51
  C:5813H         LINE#         52
  C:5813H         LINE#         53
  C:5815H         LINE#         54
  C:5817H         LINE#         55
  C:581AH         LINE#         56
  C:581AH         LINE#         58
  C:581DH         LINE#         59
  C:581DH         LINE#         60
  C:581FH         LINE#         61
  C:5822H         LINE#         62
  C:5822H         LINE#         64
  C:5824H         LINE#         65
  -------         ENDPROC       INTERRUPTUART0
BL51 BANKED LINKER/LOCATER V6.22                                                      06/21/2022  07:40:42  PAGE 102


  -------         ENDMOD        UART

  -------         MODULE        THERMISTOR
  C:0000H         SYMBOL        _ICE_DUMMY_
  D:0080H         PUBLIC        P0
  D:0090H         PUBLIC        P1
  D:00A0H         PUBLIC        P2
  D:00B0H         PUBLIC        P3
  D:00C0H         PUBLIC        P4
  D:0080H         PUBLIC        P5
  C:35AFH         PUBLIC        NTC103AT
  -------         ENDMOD        THERMISTOR

  -------         MODULE        ?C_STARTUP
  C:661AH         SEGMENT       ?C_C51STARTUP
  C:1000H         PUBLIC        ?C_STARTUP
  N:00B2H         SYMBOL        CLKCON
  D:0081H         SYMBOL        SP
  C:661AH         SYMBOL        STARTUP1
  C:1000H         LINE#         12
  C:661AH         LINE#         18
  C:661DH         LINE#         19
  C:6620H         LINE#         20
  C:6621H         LINE#         21
  C:6622H         LINE#         22
  C:6623H         LINE#         23
  C:6624H         LINE#         24
  C:6625H         LINE#         25
  C:6626H         LINE#         26
  C:6627H         LINE#         27
  C:6628H         LINE#         28
  C:662BH         LINE#         29
  -------         ENDMOD        ?C_STARTUP

  -------         MODULE        GASGAUGE
  C:0000H         SYMBOL        _ICE_DUMMY_
  D:0080H         PUBLIC        P0
  D:0090H         PUBLIC        P1
  D:00A0H         PUBLIC        P2
  D:00B0H         PUBLIC        P3
  D:00C0H         PUBLIC        P4
  D:0080H         PUBLIC        P5
  I:0017H         PUBLIC        uiRCDischarge
  I:0019H         PUBLIC        uiTempBK
  X:0368H         PUBLIC        slCur
  C:230FH         PUBLIC        GasGaugeInit
  X:036CH         PUBLIC        uiDfRC
  B:002CH.1       PUBLIC        bRSOCFast
  B:002CH.2       PUBLIC        bDsgEndFlg
  X:036EH         PUBLIC        ucCHGEndDelay
  X:036FH         PUBLIC        ucRSOCCnt
  I:001BH         PUBLIC        uiRCCharge
  B:002CH.3       PUBLIC        bRSOCSlow
  X:0370H         PUBLIC        uiDfRSOC
  X:0372H         PUBLIC        ucDSGEndDelay
  B:00A8H.4       PUBLIC        ES0
  I:001DH         PUBLIC        ucCycleGain
BL51 BANKED LINKER/LOCATER V6.22                                                      06/21/2022  07:40:42  PAGE 103


  C:1FE9H         PUBLIC        GasGaugeManage
  X:0373H         PUBLIC        uiDfFCC
  X:0375H         PUBLIC        ucDSGDelay1
  X:0376H         PUBLIC        ucDSGDelay2
  B:002CH.4       PUBLIC        bCHGEndFlg
  -------         PROC          GASGAUGEINIT
  -------         DO            
  X:02B9H         SYMBOL        i
  D:0006H         SYMBOL        RSOCtemp
  -------         ENDDO         
  C:230FH         LINE#         40
  C:230FH         LINE#         41
  C:230FH         LINE#         43
  C:2313H         LINE#         46
  C:2315H         LINE#         47
  C:231BH         LINE#         48
  C:2320H         LINE#         49
  C:2324H         LINE#         50
  C:2327H         LINE#         51
  C:232DH         LINE#         52
  C:2333H         LINE#         53
  C:2339H         LINE#         54
  C:233BH         LINE#         55
  C:233FH         LINE#         56
  C:2343H         LINE#         57
  C:2345H         LINE#         58
  C:2347H         LINE#         59
  C:2349H         LINE#         61
  C:235AH         LINE#         62
  C:235AH         LINE#         63
  C:2375H         LINE#         64
  C:2375H         LINE#         65
  C:237BH         LINE#         66
  C:237BH         LINE#         67
  C:238EH         LINE#         68
  C:238EH         LINE#         69
  C:2391H         LINE#         70
  C:2394H         LINE#         72
  C:2394H         LINE#         73
  C:23CAH         LINE#         74
  C:23CAH         LINE#         75
  C:23CDH         LINE#         76
  C:23CDH         LINE#         78
  C:23CDH         LINE#         79
  C:2447H         LINE#         80
  C:2449H         LINE#         81
  C:2449H         LINE#         82
  C:2449H         LINE#         83
  C:2452H         LINE#         85
  C:2461H         LINE#         86
  C:2461H         LINE#         87
  C:2465H         LINE#         88
  C:2465H         LINE#         90
  C:2473H         LINE#         91
  C:2473H         LINE#         92
  C:2477H         LINE#         93
  C:2479H         LINE#         95
BL51 BANKED LINKER/LOCATER V6.22                                                      06/21/2022  07:40:42  PAGE 104


  C:2479H         LINE#         96
  C:2489H         LINE#         97
  C:2489H         LINE#         98
  C:248EH         LINE#         99
  C:2490H         LINE#         101
  C:2490H         LINE#         102
  C:2497H         LINE#         103
  C:2497H         LINE#         104
  C:2497H         LINE#         106
  C:249FH         LINE#         107
  C:24ABH         LINE#         108
  C:24CEH         LINE#         110
  C:24DCH         LINE#         111
  C:24EAH         LINE#         112
  C:2501H         LINE#         114
  C:2511H         LINE#         115
  C:2511H         LINE#         116
  C:2515H         LINE#         117
  C:2517H         LINE#         118
  C:2520H         LINE#         119
  C:2520H         LINE#         120
  C:252EH         LINE#         121
  C:2530H         LINE#         122
  C:2540H         LINE#         123
  C:2540H         LINE#         124
  C:254EH         LINE#         125
  C:2550H         LINE#         127
  C:2550H         LINE#         128
  C:2554H         LINE#         129
  C:2554H         LINE#         131
  C:255AH         LINE#         132
  C:255EH         LINE#         133
  C:2562H         LINE#         134
  C:2564H         LINE#         135
  C:2566H         LINE#         136
  C:256AH         LINE#         137
  -------         ENDPROC       GASGAUGEINIT
  -------         PROC          GASGAUGEMANAGE
  -------         DO            
  X:02B9H         SYMBOL        chgdffcc
  -------         ENDDO         
  C:1FE9H         LINE#         146
  C:1FE9H         LINE#         147
  C:1FE9H         LINE#         148
  C:1FF0H         LINE#         150
  C:1FFAH         LINE#         152
  C:2017H         LINE#         153
  C:2017H         LINE#         154
  C:201CH         LINE#         155
  C:2020H         LINE#         156
  C:2022H         LINE#         157
  C:2024H         LINE#         159
  C:2046H         LINE#         161
  C:2052H         LINE#         162
  C:2052H         LINE#         163
  C:2074H         LINE#         164
  C:2076H         LINE#         165
BL51 BANKED LINKER/LOCATER V6.22                                                      06/21/2022  07:40:42  PAGE 105


  C:207FH         LINE#         166
  C:2081H         LINE#         167
  C:2081H         LINE#         168
  C:2090H         LINE#         170
  C:209FH         LINE#         171
  C:20ABH         LINE#         172
  C:20ABH         LINE#         173
  C:20B5H         LINE#         174
  C:20CAH         LINE#         175
  C:20CAH         LINE#         176
  C:20D1H         LINE#         177
  C:20D3H         LINE#         179
  C:20D3H         LINE#         180
  C:20DBH         LINE#         181
  C:20E1H         LINE#         182
  C:20E1H         LINE#         183
  C:20E3H         LINE#         185
  C:20F9H         LINE#         186
  C:20F9H         LINE#         187
  C:2121H         LINE#         188
  C:2123H         LINE#         190
  C:2123H         LINE#         191
  C:212DH         LINE#         192
  C:212DH         LINE#         194
  C:2147H         LINE#         195
  C:2147H         LINE#         196
  C:2156H         LINE#         197
  C:2156H         LINE#         198
  C:2165H         LINE#         199
  C:2165H         LINE#         200
  C:2167H         LINE#         201
  C:2169H         LINE#         202
  C:2169H         LINE#         203
  C:2169H         LINE#         204
  C:2169H         LINE#         206
  C:216CH         LINE#         208
  C:216FH         LINE#         209
  C:2192H         LINE#         210
  C:2192H         LINE#         211
  C:2197H         LINE#         212
  C:2199H         LINE#         214
  C:21A5H         LINE#         215
  C:21AFH         LINE#         216
  C:21AFH         LINE#         217
  C:21B9H         LINE#         218
  C:21B9H         LINE#         219
  C:21C5H         LINE#         220
  C:21C5H         LINE#         221
  C:21D1H         LINE#         222
  C:21D1H         LINE#         223
  C:21DBH         LINE#         224
  C:21F4H         LINE#         225
  C:2203H         LINE#         226
  C:2203H         LINE#         227
  C:220AH         LINE#         228
  C:220AH         LINE#         229
  C:220CH         LINE#         230
BL51 BANKED LINKER/LOCATER V6.22                                                      06/21/2022  07:40:42  PAGE 106


  C:221EH         LINE#         231
  C:221EH         LINE#         232
  C:2233H         LINE#         233
  C:223DH         LINE#         234
  C:223DH         LINE#         235
  C:223DH         LINE#         237
  C:2240H         LINE#         238
  C:2240H         LINE#         240
  C:2243H         LINE#         241
  C:2243H         LINE#         242
  C:2245H         LINE#         243
  C:2255H         LINE#         244
  C:225EH         LINE#         245
  C:226AH         LINE#         246
  C:2273H         LINE#         247
  C:2275H         LINE#         248
  C:2275H         LINE#         250
  C:228BH         LINE#         251
  C:228BH         LINE#         252
  C:2293H         LINE#         253
  C:2295H         LINE#         254
  C:22AAH         LINE#         255
  C:22AAH         LINE#         256
  C:22B2H         LINE#         257
  C:22B2H         LINE#         258
  C:22E2H         LINE#         260
  C:22E5H         LINE#         262
  C:22E7H         LINE#         263
  C:22F1H         LINE#         264
  C:22FDH         LINE#         265
  C:230CH         LINE#         266
  C:230EH         LINE#         267
  -------         ENDPROC       GASGAUGEMANAGE
  -------         ENDMOD        GASGAUGE

  -------         MODULE        GASGAUGELIB
  C:0000H         SYMBOL        _ICE_DUMMY_
  D:0080H         PUBLIC        P0
  D:0090H         PUBLIC        P1
  D:00A0H         PUBLIC        P2
  D:00B0H         PUBLIC        P3
  D:00C0H         PUBLIC        P4
  D:0080H         PUBLIC        P5
  C:256BH         PUBLIC        CorrectCHGSOC
  C:1B8BH         PUBLIC        CorrectDSGSOC
  C:16B1H         PUBLIC        DataFilter
  -------         PROC          CORRECTCHGSOC
  -------         DO            
  X:02BBH         SYMBOL        i
  -------         ENDDO         
  C:256BH         LINE#         17
  C:256BH         LINE#         18
  C:256BH         LINE#         20
  C:257AH         LINE#         21
  C:257AH         LINE#         22
  C:2592H         LINE#         23
  C:2592H         LINE#         24
BL51 BANKED LINKER/LOCATER V6.22                                                      06/21/2022  07:40:42  PAGE 107


  C:2592H         LINE#         25
  C:2592H         LINE#         26
  C:259AH         LINE#         27
  C:259DH         LINE#         28
  C:259DH         LINE#         29
  C:25ACH         LINE#         30
  C:25ACH         LINE#         31
  C:25BAH         LINE#         32
  C:25F5H         LINE#         33
  C:25F5H         LINE#         34
  C:25F5H         LINE#         35
  C:25FBH         LINE#         36
  C:25FBH         LINE#         37
  C:260DH         LINE#         38
  C:260DH         LINE#         39
  C:2614H         LINE#         40
  C:2614H         LINE#         41
  C:2615H         LINE#         42
  C:263FH         LINE#         43
  C:263FH         LINE#         44
  C:2650H         LINE#         45
  C:2650H         LINE#         46
  C:2699H         LINE#         47
  C:26BEH         LINE#         48
  C:26BEH         LINE#         49
  C:26BFH         LINE#         50
  C:26C5H         LINE#         51
  C:26C5H         LINE#         52
  C:26F4H         LINE#         53
  C:26F4H         LINE#         54
  C:2723H         LINE#         55
  C:2723H         LINE#         56
  C:279AH         LINE#         57
  C:27BFH         LINE#         58
  C:27BFH         LINE#         59
  C:27BFH         LINE#         60
  C:27BFH         LINE#         61
  -------         ENDPROC       CORRECTCHGSOC
  -------         PROC          CORRECTDSGSOC
  -------         DO            
  X:02BBH         SYMBOL        DfRCtemp
  X:02BDH         SYMBOL        j
  X:02BFH         SYMBOL        c_cur
  X:02C0H         SYMBOL        vol5per
  X:02C2H         SYMBOL        tempfcc
  -------         ENDDO         
  C:1B8BH         LINE#         70
  C:1B8BH         LINE#         71
  C:1B8BH         LINE#         73
  C:1B92H         LINE#         74
  C:1B96H         LINE#         75
  C:1B98H         LINE#         76
  C:1B9CH         LINE#         77
  C:1BA0H         LINE#         79
  C:1BCCH         LINE#         80
  C:1BCCH         LINE#         81
  C:1BDBH         LINE#         82
BL51 BANKED LINKER/LOCATER V6.22                                                      06/21/2022  07:40:42  PAGE 108


  C:1BE9H         LINE#         83
  C:1C4EH         LINE#         84
  C:1C65H         LINE#         85
  C:1C65H         LINE#         86
  C:1C78H         LINE#         87
  C:1C7AH         LINE#         88
  C:1CB7H         LINE#         89
  C:1CB7H         LINE#         90
  C:1CDFH         LINE#         91
  C:1CDFH         LINE#         92
  C:1D01H         LINE#         94
  C:1D0FH         LINE#         95
  C:1D0FH         LINE#         96
  C:1D28H         LINE#         97
  C:1D2AH         LINE#         98
  C:1D4CH         LINE#         99
  C:1D4CH         LINE#         100
  C:1D56H         LINE#         101
  C:1D58H         LINE#         103
  C:1D58H         LINE#         104
  C:1D74H         LINE#         105
  C:1D74H         LINE#         106
  C:1D83H         LINE#         107
  C:1D83H         LINE#         108
  C:1D92H         LINE#         109
  C:1D92H         LINE#         110
  C:1D92H         LINE#         111
  C:1DDFH         LINE#         112
  C:1DDFH         LINE#         113
  C:1DFBH         LINE#         114
  C:1E2BH         LINE#         115
  C:1E5AH         LINE#         117
  C:1E90H         LINE#         118
  C:1E90H         LINE#         119
  C:1EA2H         LINE#         120
  C:1EA2H         LINE#         121
  C:1EA4H         LINE#         122
  C:1EA6H         LINE#         123
  C:1EA8H         LINE#         124
  C:1EA8H         LINE#         125
  C:1EABH         LINE#         126
  C:1EE2H         LINE#         127
  C:1EE2H         LINE#         128
  C:1EF4H         LINE#         129
  C:1EF4H         LINE#         130
  C:1EF6H         LINE#         131
  C:1EF8H         LINE#         132
  C:1EFAH         LINE#         133
  C:1EFAH         LINE#         134
  C:1EFDH         LINE#         135
  C:1F2CH         LINE#         136
  C:1F2CH         LINE#         137
  C:1F3BH         LINE#         138
  C:1F3BH         LINE#         139
  C:1F3DH         LINE#         140
  C:1F3FH         LINE#         141
  C:1F41H         LINE#         142
BL51 BANKED LINKER/LOCATER V6.22                                                      06/21/2022  07:40:42  PAGE 109


  C:1F41H         LINE#         143
  C:1F43H         LINE#         144
  C:1F78H         LINE#         145
  C:1F78H         LINE#         146
  C:1F87H         LINE#         147
  C:1F87H         LINE#         148
  C:1F89H         LINE#         149
  C:1F8BH         LINE#         150
  C:1F8DH         LINE#         151
  C:1F8DH         LINE#         152
  C:1F8FH         LINE#         154
  C:1F8FH         LINE#         155
  C:1F91H         LINE#         156
  C:1F93H         LINE#         157
  C:1F93H         LINE#         159
  C:1FA2H         LINE#         160
  C:1FA2H         LINE#         161
  C:1FB0H         LINE#         162
  C:1FB0H         LINE#         163
  C:1FB2H         LINE#         164
  C:1FB4H         LINE#         165
  C:1FBCH         LINE#         166
  C:1FBCH         LINE#         167
  C:1FD8H         LINE#         168
  C:1FD9H         LINE#         170
  C:1FD9H         LINE#         171
  C:1FE8H         LINE#         172
  C:1FE8H         LINE#         173
  C:1FE8H         LINE#         174
  C:1FE8H         LINE#         175
  C:1FE8H         LINE#         176
  -------         ENDPROC       CORRECTDSGSOC
  -------         PROC          DATAFILTER
  -------         DO            
  X:02BBH         SYMBOL        dsoc
  X:02BCH         SYMBOL        Filter_dsoc
  X:02C0H         SYMBOL        k
  X:02C4H         SYMBOL        difvol
  D:0003H         SYMBOL        difsoc
  D:0004H         SYMBOL        curspeed
  D:0006H         SYMBOL        ucrsocdectime
  X:02C5H         SYMBOL        curratio
  -------         ENDDO         
  C:16B1H         LINE#         184
  C:16B1H         LINE#         185
  C:16B1H         LINE#         187
  C:16BBH         LINE#         188
  C:16C5H         LINE#         195
  C:16D9H         LINE#         197
  C:16F0H         LINE#         198
  C:16F0H         LINE#         199
  C:1721H         LINE#         200
  C:1721H         LINE#         201
  C:1740H         LINE#         202
  C:1740H         LINE#         203
  C:1756H         LINE#         204
  C:1785H         LINE#         205
BL51 BANKED LINKER/LOCATER V6.22                                                      06/21/2022  07:40:42  PAGE 110


  C:17B3H         LINE#         206
  C:17C4H         LINE#         207
  C:180CH         LINE#         208
  C:180CH         LINE#         209
  C:183CH         LINE#         210
  C:183CH         LINE#         211
  C:183FH         LINE#         213
  C:183FH         LINE#         214
  C:1850H         LINE#         215
  C:1861H         LINE#         216
  C:186EH         LINE#         217
  C:186EH         LINE#         218
  C:1871H         LINE#         219
  C:189EH         LINE#         220
  C:189EH         LINE#         221
  C:18ADH         LINE#         222
  C:18ADH         LINE#         223
  C:18BEH         LINE#         224
  C:18CFH         LINE#         225
  C:18D9H         LINE#         226
  C:18D9H         LINE#         227
  C:18ECH         LINE#         228
  C:18ECH         LINE#         229
  C:191AH         LINE#         230
  C:191AH         LINE#         231
  C:1952H         LINE#         232
  C:1952H         LINE#         233
  C:1985H         LINE#         234
  C:1987H         LINE#         236
  C:1987H         LINE#         237
  C:198FH         LINE#         238
  C:198FH         LINE#         239
  C:199FH         LINE#         240
  C:199FH         LINE#         241
  C:19B4H         LINE#         242
  C:19B6H         LINE#         244
  C:19B6H         LINE#         245
  C:19BCH         LINE#         246
  C:19BCH         LINE#         247
  C:1A0FH         LINE#         248
  C:1A20H         LINE#         249
  C:1A3BH         LINE#         251
  C:1A47H         LINE#         252
  C:1A47H         LINE#         253
  C:1A55H         LINE#         254
  C:1A5AH         LINE#         255
  C:1A5AH         LINE#         256
  C:1A71H         LINE#         257
  C:1A96H         LINE#         258
  C:1A98H         LINE#         260
  C:1A98H         LINE#         261
  C:1AA6H         LINE#         262
  C:1AABH         LINE#         263
  C:1AABH         LINE#         264
  C:1AABH         LINE#         265
  C:1ABCH         LINE#         266
  C:1AE7H         LINE#         267
BL51 BANKED LINKER/LOCATER V6.22                                                      06/21/2022  07:40:42  PAGE 111


  C:1AE9H         LINE#         268
  C:1AFBH         LINE#         269
  C:1AFBH         LINE#         270
  C:1B0CH         LINE#         271
  C:1B1DH         LINE#         272
  C:1B25H         LINE#         273
  C:1B27H         LINE#         275
  C:1B27H         LINE#         276
  C:1B38H         LINE#         277
  C:1B63H         LINE#         278
  C:1B63H         LINE#         279
  C:1B63H         LINE#         280
  C:1B73H         LINE#         281
  C:1B73H         LINE#         282
  C:1B7CH         LINE#         283
  C:1B7DH         LINE#         284
  C:1B83H         LINE#         285
  C:1B83H         LINE#         286
  C:1B8AH         LINE#         287
  C:1B8AH         LINE#         288
  -------         ENDPROC       DATAFILTER
  -------         ENDMOD        GASGAUGELIB

  -------         MODULE        BOOTAPP
  C:0000H         SYMBOL        _ICE_DUMMY_
  D:0080H         PUBLIC        P0
  D:0090H         PUBLIC        P1
  D:00A0H         PUBLIC        P2
  D:00B0H         PUBLIC        P3
  D:00C0H         PUBLIC        P4
  D:0080H         PUBLIC        P5
  B:00A8H.7       PUBLIC        EA
  C:6725H         PUBLIC        ISPProcess
  -------         PROC          ISPPROCESS
  C:6725H         LINE#         18
  C:6725H         LINE#         19
  C:6725H         LINE#         20
  C:672BH         LINE#         21
  C:672BH         LINE#         22
  C:672DH         LINE#         23
  C:672FH         LINE#         24
  C:6731H         LINE#         25
  C:6734H         LINE#         26
  C:6737H         LINE#         27
  C:6737H         LINE#         28
  -------         ENDPROC       ISPPROCESS
  -------         ENDMOD        BOOTAPP

  -------         MODULE        DATAFLASH
  C:0000H         SYMBOL        _ICE_DUMMY_
  C:8400H         PUBLIC        dataflash
  -------         ENDMOD        DATAFLASH

  -------         MODULE        ?C?FPADD
  C:105DH         PUBLIC        ?C?FPADD
  C:1059H         PUBLIC        ?C?FPSUB
  -------         ENDMOD        ?C?FPADD
BL51 BANKED LINKER/LOCATER V6.22                                                      06/21/2022  07:40:42  PAGE 112



  -------         MODULE        ?C?FPMUL
  C:114EH         PUBLIC        ?C?FPMUL
  -------         ENDMOD        ?C?FPMUL

  -------         MODULE        ?C?FPDIV
  C:1257H         PUBLIC        ?C?FPDIV
  -------         ENDMOD        ?C?FPDIV

  -------         MODULE        ?C?FCAST
  C:12FEH         PUBLIC        ?C?FCASTC
  C:12F9H         PUBLIC        ?C?FCASTI
  C:12F4H         PUBLIC        ?C?FCASTL
  -------         ENDMOD        ?C?FCAST

  -------         MODULE        ?C?CASTF
  C:1332H         PUBLIC        ?C?CASTF
  -------         ENDMOD        ?C?CASTF

  -------         MODULE        ?C?CLDPTR
  C:13B3H         PUBLIC        ?C?CLDPTR
  -------         ENDMOD        ?C?CLDPTR

  -------         MODULE        ?C?IMUL
  C:13CCH         PUBLIC        ?C?IMUL
  -------         ENDMOD        ?C?IMUL

  -------         MODULE        ?C?UIDIV
  C:13DEH         PUBLIC        ?C?UIDIV
  -------         ENDMOD        ?C?UIDIV

  -------         MODULE        ?C?IILDX
  C:1433H         PUBLIC        ?C?IILDX
  -------         ENDMOD        ?C?IILDX

  -------         MODULE        ?C?LADD
  C:1449H         PUBLIC        ?C?LADD
  -------         ENDMOD        ?C?LADD

  -------         MODULE        ?C?LSUB
  C:1456H         PUBLIC        ?C?LSUB
  -------         ENDMOD        ?C?LSUB

  -------         MODULE        ?C?LMUL
  C:1464H         PUBLIC        ?C?LMUL
  -------         ENDMOD        ?C?LMUL

  -------         MODULE        ?C?ULDIV
  C:14EFH         PUBLIC        ?C?ULDIV
  -------         ENDMOD        ?C?ULDIV

  -------         MODULE        ?C?SLDIV
  C:5E8FH         PUBLIC        ?C?SLDIV
  -------         ENDMOD        ?C?SLDIV

  -------         MODULE        ?C?LOR
  C:1581H         PUBLIC        ?C?LOR
BL51 BANKED LINKER/LOCATER V6.22                                                      06/21/2022  07:40:42  PAGE 113


  -------         ENDMOD        ?C?LOR

  -------         MODULE        ?C?LNEG
  C:158EH         PUBLIC        ?C?LNEG
  -------         ENDMOD        ?C?LNEG

  -------         MODULE        ?C?SLCMP
  C:159CH         PUBLIC        ?C?SLCMP
  -------         ENDMOD        ?C?SLCMP

  -------         MODULE        ?C?ULCMP
  C:15B2H         PUBLIC        ?C?ULCMP
  -------         ENDMOD        ?C?ULCMP

  -------         MODULE        ?C?ULSHR
  C:15C3H         PUBLIC        ?C?ULSHR
  -------         ENDMOD        ?C?ULSHR

  -------         MODULE        ?C?SLSHR
  C:15D6H         PUBLIC        ?C?SLSHR
  -------         ENDMOD        ?C?SLSHR

  -------         MODULE        ?C?LSHL
  C:15EAH         PUBLIC        ?C?LSHL
  -------         ENDMOD        ?C?LSHL

  -------         MODULE        ?C?LLDXDATA
  C:15FDH         PUBLIC        ?C?LLDXDATA
  -------         ENDMOD        ?C?LLDXDATA

  -------         MODULE        ?C?LLDXDATA0
  C:1609H         PUBLIC        ?C?LLDXDATA0
  -------         ENDMOD        ?C?LLDXDATA0

  -------         MODULE        ?C?LSTXDATA
  C:1615H         PUBLIC        ?C?LSTXDATA
  -------         ENDMOD        ?C?LSTXDATA

  -------         MODULE        ?C?LSTKXDATA
  C:1621H         PUBLIC        ?C?LSTKXDATA
  -------         ENDMOD        ?C?LSTKXDATA

  -------         MODULE        ?C?OFFXADD
  C:1652H         PUBLIC        ?C?OFFXADD
  -------         ENDMOD        ?C?OFFXADD

  -------         MODULE        ?C?CCASE
  C:165EH         PUBLIC        ?C?CCASE
  -------         ENDMOD        ?C?CCASE

  -------         MODULE        ?C?LIMUL
  C:1684H         PUBLIC        ?C?LIMUL
  -------         ENDMOD        ?C?LIMUL

  -------         MODULE        LABS
  C:679EH         PUBLIC        _LABS
  -------         ENDMOD        LABS
BL51 BANKED LINKER/LOCATER V6.22                                                      06/21/2022  07:40:42  PAGE 114





FUNCTION REGISTER MASKS


FUNCTION . . . . . . . . . REG MASK
-----------------------------------

AFEADCDIS. . . . . . . . . @0xf7ff
AFEADCEN . . . . . . . . . @0xf7ff
AFECADCDIS . . . . . . . . @0xf7ff
AFECADCEN. . . . . . . . . @0xf7ff
AFECHGERCHECKDIS . . . . . @0xf7ff
AFECHGERCHECKEN. . . . . . @0xf7ff
AFECLRFLG. . . . . . . . . @0xf7ff
AFEENTERPD . . . . . . . . @0xf7ff
AFEGETTEMPE. . . . . . . . @0xf7ff
AFEGETVOL. . . . . . . . . @0xf7ff
AFEINIT. . . . . . . . . . @0xf7ff
AFELOADCHECKDIS. . . . . . @0xf7ff
AFELOADCHECKEN . . . . . . @0xf7ff
AFERAMCHECK. . . . . . . . @0xf7ff
AFERDFLG . . . . . . . . . @0xf7ff
AFERDSTATUS. . . . . . . . @0xf7ff
AFETEMPADCDIS. . . . . . . @0xf7ff
AFETEMPADCEN . . . . . . . @0xf7ff
AFETWICHECK. . . . . . . . @0xf300
AFEWDTDIS. . . . . . . . . @0xf7ff
AFEWDTEN . . . . . . . . . @0xf7ff
BALPROCESS . . . . . . . . @0xf7ff
CALICURZERO. . . . . . . . @0xe301
CALIRTCTIME. . . . . . . . @0xf7ff
CHGERCHECK . . . . . . . . @0xf7ff
CLRRAM . . . . . . . . . . @0xf383
CTOCHECKVOL. . . . . . . . @0xf300
CTOTURNONCHECK . . . . . . @0xf300
E2PROMBKBOOT . . . . . . . @0xf7ff
E2PROMINIT . . . . . . . . @0xf7ff
E2PROMTWICHECK . . . . . . @0xf300
IAPCHECKHANDSHAKE. . . . . @0xf7bf
INITGPIO . . . . . . . . . @0x8000
INITIRQ. . . . . . . . . . @0xe000
INITVAR. . . . . . . . . . @0xf797
INTERRUPTINT4. . . . . . . @0xf003
INTERRUPTTIMER3. . . . . . @0xf300
INTERRUPTTIMER3APP . . . . @0xf300
INTERRUPTUARTAPPTX . . . . @0xf38f
KEYSCAN. . . . . . . . . . @0xf000
LEDAUTOOFF . . . . . . . . @0xf300
LEDDISPLAY . . . . . . . . @0xf303
LOADCHECK. . . . . . . . . @0xf7ff
LOWPOWERCHECK. . . . . . . @0xf301
LOWPOWERPROCESS. . . . . . @0xf7ff
MCUFLASHPROCESS. . . . . . @0xf7bf
MCUFLASHWRWAITCHECK. . . . @0xf300
MCUINTOIDLE. . . . . . . . @0xc000
BL51 BANKED LINKER/LOCATER V6.22                                                      06/21/2022  07:40:42  PAGE 115


MCUINTOPD. . . . . . . . . @0xc000
MOSCTRL. . . . . . . . . . @0xf7ff
MOSSTATUSCHECK . . . . . . @0xc000
PORPROTECTOTC. . . . . . . @0xf78f
PORPROTECTOTD. . . . . . . @0xf78f
PORPROTECTOV . . . . . . . @0xf782
PORPROTECTUTC. . . . . . . @0xf78f
PORPROTECTUTD. . . . . . . @0xf78f
PORPROTECTUV . . . . . . . @0xf782
PROTECTOCRECOVER . . . . . @0xf7ff
PROTECTOTC . . . . . . . . @0xf7af
PROTECTOTD . . . . . . . . @0xf7af
PROTECTOV. . . . . . . . . @0xf78b
PROTECTUTC . . . . . . . . @0xf7af
PROTECTUTD . . . . . . . . @0xf7af
PROTECTUV. . . . . . . . . @0xf78b
RAMCHECKPROCESS. . . . . . @0xf300
READSUBCLASSID . . . . . . @0xf375
RTCTWICHECK. . . . . . . . @0xf300
SYSPARAINIT. . . . . . . . @0xffbf
SYSTEMINTOPD . . . . . . . @0xf7ff
SYSTEMINTOSLEEP. . . . . . @0xf7ff
UARTCALICUROFFSET. . . . . @0xf375
UARTCALIRTC. . . . . . . . @0xf377
UARTCALITS1. . . . . . . . @0xf377
UARTCALITS2. . . . . . . . @0xf377
UARTCALIVOLTAGE. . . . . . @0xf377
UARTCHECK. . . . . . . . . @0xf300
UARTHANDSHAKE. . . . . . . @0xe300
UARTRDCMDPROCESS . . . . . @0xf3ff
UARTRDE2PROM . . . . . . . @0xf7ff
WAKEUPPROCESS. . . . . . . @0xf7ff
WRITEMANUFACTURE . . . . . @0xf375
_AFEALARMDIS . . . . . . . @0xf7ff
_AFEALARMEN. . . . . . . . @0xf7ff
_AFEBALCTL . . . . . . . . @0xf7ff
_AFEMOSCTL . . . . . . . . @0xf7ff
_AFEREADREG. . . . . . . . @0xf7ff
_AFEWRITEREG . . . . . . . @0xf7ff
_CRC8CAL . . . . . . . . . @0xf365
_DELAY1MS. . . . . . . . . @0xf03e
_E2PROMREAD. . . . . . . . @0xf7ff
_E2PROMWRITE . . . . . . . @0xf7ff
_INTERRUPTINT4APP. . . . . @0xf003
_LEDGETDISNUM. . . . . . . @0xf001
_MCUCLOCKSET . . . . . . . @0xf003
_MCUFLASHBLANKCHECK. . . . @0xf31c
_MCUFLASHCHECKFLG. . . . . @0xf303
_MCUFLASHDATACHECK . . . . @0xf7af
_MCUFLASHREAD. . . . . . . @0xf307
_MCUFLASHWRITE . . . . . . @0xf7bf
_MCUFLASHWRONEBYTE . . . . @0xf035
_MCUFLASHWRSECTOR. . . . . @0xf33f
_MEMORYCOPY. . . . . . . . @0xf78d
_MEMORYSET . . . . . . . . @0xf781
_RTCMODIFYTIME . . . . . . @0xf7ff
_RTCREAD . . . . . . . . . @0xf7ff
BL51 BANKED LINKER/LOCATER V6.22                                                      06/21/2022  07:40:42  PAGE 116


_RTCWRITE. . . . . . . . . @0xf7ff
_TWICHECKSTATUS. . . . . . @0xf00c
_TWIINIT . . . . . . . . . @0xf48f
_TWIREAD . . . . . . . . . @0xf7ff
_TWIWRITE. . . . . . . . . @0xf7ff
_UARTREADINFO. . . . . . . @0xf37f
_UARTWRITEINFO . . . . . . @0xf7ff

Program Size: data=143.6 xdata=1080 code=23457
LINK/LOCATE RUN COMPLETE.  0 WARNING(S),  0 ERROR(S)
